:020000040002F8
:10600000F8B40020DD630200E56302004588020069
:10601000E9630200EB630200ED6302000000000090
:10602000000000000000000000000000EF6302001C
:10603000F163020000000000F3630200F563020058
:10604000C1A10200F7630200F7630200F9B4020085
:106050000DB50200F7630200F7630200D5B002003D
:10606000F7630200F7630200F7630200F7630200C0
:10607000F7630200F7630200F7630200F7630200B0
:1060800079C7020049AC0200F7630200F76302001F
:10609000F7630200F763020085B50200F7630200B0
:1060A000F7630200F7630200F7630200F763020080
:1060B00081A20200F763020000000000000000005F
:1060C000F7630200F7630200F763020021B50200E4
:1060D00061AC0200F7630200F763020000000000F9
:1060E00000000000000000000000000000000000B0
:1060F00000000000000000000000000000000000A0
:10610000000000000000000000000000000000008F
:10611000000000000000000000000000000000007F
:10612000000000000000000000000000000000006F
:10613000000000000000000000000000000000005F
:10614000000000000000000000000000000000004F
:10615000000000000000000000000000000000003F
:10616000000000000000000000000000000000002F
:10617000000000000000000000000000000000001F
:10618000000000000000000000000000000000000F
:1061900000000000000000000000000000000000FF
:1061A00000000000000000000000000000000000EF
:1061B00000000000000000000000000000000000DF
:1061C00000000000000000000000000000000000CF
:1061D00000000000000000000000000000000000BF
:1061E00000000000000000000000000000000000AF
:1061F000000000000000000000000000000000009F
:10620000DFF80CD000F0F4FC004800476DCD03002F
:10621000F8B4002000B583B002900091019244F2DE
:10622000010071466A460AF039F803B000BD00006B
:1062300030B450E8012F93B2C48923448489A34227
:1062400028BF1B1B0489A34202BFBFF32F8F00206E
:1062500007E0C3EA020340E80134002CE9D14FF023
:1062600001000A6030BC704750E8012FC2EA0242C8
:1062700040E801210029F7D1704730B450E8022FDF
:106280001FFAA2F3C488A34202BFBFF32F8F0020DE
:106290000DE0C48923448489A34228BF1B1BC2EAA2
:1062A000034340E80234002CE8D14FF001000A60BB
:1062B00030BC704750E8022FC2EA224240E8022177
:1062C0000029F7D17047034653E8022FD988B2EB73
:1062D000324F4FF0000017BF92B241EA014142EA4B
:1062E000014104E05A68B2EB324F08BF012043E895
:1062F0000212002AE8D1704730B4044654E8000F77
:106300000D4644E80053002BF8D1156030BC7047AF
:1063100030B4044654E8000F40EA010544E8005355
:10632000002BF7D1156030BC704730B4044654E8F8
:10633000000F00EA010544E80053002BF7D1156077
:1063400030BC704730B4044654E8000F80EA0105C1
:1063500044E80053002BF7D1156030BC704730B4CF
:10636000044654E8000F00EB010544E80053002BFD
:10637000F7D1156030BC704730B4044654E8000FC4
:10638000A0EB010544E80053002BF7D1156030BCA9
:10639000704770B404464FF0000054E8006F0D6879
:1063A000AE4207BF44E80023012044E800630E60CA
:1063B000002B1CBF0020F0E770BC704730B40446CF
:1063C00054E8000F88422CBF451A054644E80053A4
:1063D000002BF5D1156030BC70470000064880479F
:1063E00006480047FEE7FEE7FEE7FEE7FEE7FEE7BA
:1063F000FEE7FEE7FEE7FEE73DC2020001620200A3
:106400002DE9F05F0546002092469B4688460646E9
:10641000814640241BE0284641464746224600F07C
:10642000C8FA53465A46C01A914110D3114618462D
:10643000224600F0AFFA2D1A67EB01084F462246BC
:106440000120002100F0A6FA17EB00094E41201EA2
:10645000A4F10104DFDC484631462A464346BDE844
:10646000F09F40EA01039B0703D009E008C9121F0F
:1064700008C0042AFAD203E011F8013B00F8013BFE
:10648000521EF9D27047D2B201E000F8012B491E2A
:10649000FBD270470022F6E710B513460A460446C1
:1064A0001946FFF7F0FF204610BD421C10F8011BF3
:1064B0000029FBD1801A704710B5002200E0521C61
:1064C000835C8C5CA34201D1002BF8D1D8B2E1B23D
:1064D000401A10BD30B504460020034600E05B1CA6
:1064E000934203D2E05CCD5C401BF8D030BD2DE977
:1064F000FE4F804681EA0300C00F0C46009021F059
:10650000004123F00045B8EB0200A94105D2404606
:10651000214690461C460B46024623F0004010439D
:1065200047D0270DC7F30A00C3F30A510290401A5F
:10653000019040286BDAC3F3130040F4801B0098ED
:10654000924620B10023D2EB030A63EB0B0B0198B8
:106550005946C0F14002504600F01CFA06460D466E
:1065600050465946019A00F034FA10EB0800614198
:10657000002487EA115284EAE7731A4340D0009A54
:1065800062B3019A012A4FEA075215DC001B61EB46
:1065900002014FF0004202EA0752CDE90042001C1E
:1065A00041F5801132462B4600F06BFA03B0BDE88E
:1065B000F08F40462146F9E7001B61EB0201001C09
:1065C00041F5801300185B412018A2F5001747EB36
:1065D000030140EAD570B6196D4111E06D084FEA2C
:1065E000360645EAC0754FEA0752001B61EB02010F
:1065F000001C41F5801149084FEA30000019514153
:1066000032462B4603B0BDE8F04F00F02BBA00989D
:10661000012240000023D0EB020263EBE0730098FC
:1066200021464FEAE074B8EB000061EB0401E9E7B2
:1066300083F000435BE781F0004158E72DE9FE4F0E
:1066400081EA030404F0004421F0004100944FF07B
:10665000000B23F0004350EA01045ED052EA030429
:106660005BD0C3F30A54C1F30A552C44A4F2F334AB
:106670000194A0FB0254C1F3130141F48011C3F350
:10668000130343F4801301FB024400FB034E840A0E
:10669000970A44EA815447EA8357A4FB07680295A6
:1066A0008D0A05FB07854FEA932C04FB0C54270544
:1066B000029D4FEA065847EA1637B5EB08056EEB20
:1066C000070C870E920E47EA811742EA8312A7FB56
:1066D0000201B6EB0B0164EB00042B0D43EA0C3313
:1066E0005E1844EB1C50DA465146E7FB0201C5F345
:1066F00013044FEA0B3343EA14534FEA0432019C6C
:1067000043EA0603A4F10C040294009CCDE900B412
:1067100000F0B7F903B0BDE8F08F00200146F9E7BB
:106720002DE9F04D81EA030404F0004B21F000450F
:1067300014464FF0000A23F0004150EA050220D031
:1067400054EA01021DD0C5F30A570246C5F31303EC
:10675000C1F31300C1F30A5640F4801543F48013CB
:10676000A7EB0608101BD64608F2FD3873EB0500B0
:1067700002D308F1010801E092185B41B8F1000F63
:1067800003DA00200146BDE8F08D00204FF48011AF
:10679000064684460EE0171B73EB050705D3121B54
:1067A00063EB050306434CEA010C49084FEA30004D
:1067B00092185B4150EA0107EDD152EA030012D072
:1067C00082EA040083EA0501084305D0101BAB41AF
:1067D00006D20122002306E000224FF0004302E02F
:1067E0006FF0010253101AEB06004CEB085110EB4E
:1067F0000A0041EB0B01BDE8F04D00F033B90EB5D6
:10680000C10F80EAE0700844CA07002140F2334318
:106810008DE80E000A460B4600F033F903B000BDC8
:106820000EB540F2334102910021CDE900110A4634
:106830000B4600F026F903B000BD70B5C1F30A5253
:1068400001F000450024C1F3130140F2FF3341F48D
:1068500080119A4201DA002070BD40F233439A421F
:10686000A2F2334203DC524200F0A3F800E0904071
:106870002C43F1D0404270BDC1F30A5210B5C1F3B0
:10688000130140F2FF3341F480119A4201DA0020F3
:1068900010BD40F233439A42A2F2334203DC52422B
:1068A00000F087F810BD904010BD00F0004230F0BD
:1068B00000400AD0C10D01F56071C0F3160042EA34
:1068C0000151C2084007114370470020014670473C
:1068D00030B5041E71F1000404DB4FF00044404267
:1068E00064EB0101141E73F1000405DB1C464FF03C
:1068F0000043524263EB04038B4208BF824230BD27
:1069000030B5041E71F1000404DB4FF00044404236
:1069100064EB0101141E73F1000405DB1C464FF00B
:106920000043524263EB0403994208BF904230BDDA
:1069300001F0004330B421F0004150EA010206D0DA
:106940000A0DA2F56072C1F31301002A02DC30BC0B
:1069500000207047440F44EAC104C100E01830BC75
:1069600000EBC25000F047B830B50B46014600209E
:106970002022012409E021FA02F59D4205D303FA01
:1069800002F5491B04FA02F52844151EA2F1010282
:10699000F1DC30BD202A04DB203A00FA02F10020AD
:1069A00070479140C2F1200320FA03F3194390404D
:1069B0007047202A04DB203A21FA02F000217047B8
:1069C00021FA02F3D040C2F1200291400843194657
:1069D0007047202A06DBCB17203A41FA02F043EA3F
:1069E000E07306E041FA02F3D040C2F12002914088
:1069F0000843194670470029A8BF7047401C49004A
:106A000008BF20F00100704710B4B0FA80FC00FA13
:106A10000CF050EA010404BF10BC704749B1CCF13E
:106A2000200421FA04F411FA0CF118BF01212143CA
:106A30000843A3EB0C01CB1D4FEA00614FEA102085
:106A400042BF002010BC704700EBC3501044002927
:106A5000A4BF10BC7047401C490008BF20F00100D3
:106A600010BC704710B5141E73F1000408DA401C06
:106A700041F1000192185B411A4301D120F001005D
:106A800010BD2DE9F04D92469B4611B1B1FA81F24D
:106A900002E0B0FA80F220329046FFF77BFF044616
:106AA0000F4640EA0A0041EA0B0153465A460843A2
:106AB00013D0114653EA010019D0C8F140025046E4
:106AC000FFF777FF05460E46504659464246FFF708
:106AD00061FF084305D0012004E020463946BDE8A7
:106AE000F08D0020054346EAE0762C4337430A98B0
:106AF0006305E40AA0EB08000022FD0A44EA4754BB
:106B00000A3002D500200146E9E701051019694164
:106B1000DDE9084500196941BDE8F04DA2E72DE91E
:106B2000F04D00231A461B1A8A4103DB0020014660
:106B3000BDE8F08DC1F30A52C1F3130141F4801591
:106B40004FF0000BD10702D100186D41521E0027F3
:106B5000044640F2FF11384601EB620A3E46804689
:106B6000024600204FF48011FFF723FFC219714144
:106B7000BB1846EB0100B4EB030C75EB000C04D31F
:106B8000E41A65EB000517460E46241908F10100CA
:106B90006D4180463428E3DDF91946EB0600091BF8
:106BA000A84103D24FF0FF32134601E00022134602
:106BB0001BEB070046EB0A51BDE8F04DFFF752BF53
:106BC000C1F30A52C1F3130140F2FF3341F48011C3
:106BD0009A4202DA00200146704740F233439A425B
:106BE000A2F2334202DC5242FFF7E3BEFFF7D2BE0D
:106BF000064C074D06E0E06840F0010394E807000A
:106C000098471034AC42F6D3FFF7FEFA186F040031
:106C1000386F040070B58C1810F8015B15F007038D
:106C200001D110F8013B2A1106D110F8012B03E025
:106C300010F8016B01F8016B5B1EF9D12B0705D42D
:106C40000023521E0DD401F8013BFAE710F8013B76
:106C5000CB1A921C03E013F8015B01F8015B521E92
:106C6000F9D5A142D8D3002070BD10B519F0D8FED7
:106C700010BD10B500F002F810BD0000F8B50027F7
:106C80001D480068009003208DF802006C461B4EE2
:106C900004B91B4C3146204619F0D6FD0DB14FF01A
:106CA000FF37002419E0174850F83400FF2813D0AC
:106CB000144800EBC4004068FF280DD0114A02EBD5
:106CC000C402526802EBC2020F4BD1180D4A02EB0C
:106CD000C402107919F020FD641C082CE3DB0B487A
:106CE000006840B10948008881B2094819F0B4FC35
:106CF0000DB14FF0FF37F8BD34680400F1EA02002F
:106D0000306804002C410020AC7900206C41002048
:106D1000F479002070B505460E4600242CE0184892
:106D200050F83400A84226D1154800EBC400406852
:106D3000B04220D1124901EBC401087919F058FD85
:106D400000200F4901EBC401496801EBC1010D4A64
:106D50001144C871FF200A4941F8340001EBC40115
:106D600048600948006820B107480068401E06498D
:106D70000860002070BD641C082CD0DB0420F9E7FB
:106D80002C410020AC7900206C41002070B50446F5
:106D900094B10A48006808B9052070BDFFF765FF87
:106DA000FFF767FF19F024FE05460DB10820F4E750
:106DB000034804600020F0E70820EEE76C41002063
:106DC000704100202DE9FC5F05468946164649467C
:106DD0002846FFF79FFF0024D0E06B4850F83400AE
:106DE000FF287DD1684800EBC4004068FF28F8D137
:106DF000FF2D75D0FFF739FF634840F8345000EBA2
:106E0000C400C0F80490604951F8340000BF4FF04E
:106E1000A042114601F5E06252F8202002F0010282
:106E20009246594850F8348000200090334602467C
:106E300001460190404618F0A0F900BF00205249D9
:106E400001EBC401496801EBC101504A50544E495D
:106E500001EBC401496801EBC101114448704A4982
:106E600001EBC401496801EBC10111448870464936
:106E700001EBC401496801EBC1011144C870022053
:106E8000414901EBC401496801EBC101114408719A
:106E900000203D4901EBC401496801EBC1011144E7
:106EA0004871394901EBC401496801EBC101114442
:106EB0008871354800EBC4000079401C324901EB71
:106EC000C401496801EBC1011144C87100202E4979
:106ED00001EBC401496801EBC1011144087200E0F3
:106EE0004BE0294A02EBC402526802EBC202274B74
:106EF000D118254A02EBC402107919F00DFC07469F
:106F00008FB30020204901EBC401496801EBC101A6
:106F10001E4A1144C871FF201B4941F8340001EB9F
:106F2000C4014860184850F83480D346BBF1000FC4
:106F300009D10020009003460246014601904046D8
:106F400018F01BF909E000BF4FF0A04108460121ED
:106F500001FA08F1C0F8181500BF00BFFFF789FE5D
:106F60000320BDE8FC9FFFE709480068401C084972
:106F70000860FFF77EFE0020F3E7641C082CFFF694
:106F80002CAF0320EDE700002C410020AC7900205D
:106F90006C4100202DE9F04106460F461446984604
:106FA000069DB0EE000A84ED000A95ED020AB1EEEE
:106FB000400A84ED010A95ED010A84ED020A95ED7F
:106FC000020A84ED030AB0EE000A84ED040A95ED8E
:106FD000000AB1EE400A84ED050A95ED010AB1EE12
:106FE000400A84ED060A95ED000A84ED070AB0EE2A
:106FF000000A84ED080A4146204614F0F5FBB0EE85
:10700000000A84ED000A95ED020A84ED010A95ED6F
:10701000010AB1EE400A84ED020A95ED020AB1EED2
:10702000400A84ED030AB0EE000A84ED040A95EDEF
:10703000000A84ED050A95ED010A84ED060A95ED36
:10704000000AB1EE400A84ED070AB0EE000A84EDB2
:10705000080A3A464146204616F095FF2422394652
:107060002046FFF7FEF93A463146204616F08BFFE0
:10707000242239463046FFF7F4F9BDE8F0810000DC
:1070800010B5054A05A1002003F054FC074A08A1E9
:10709000012003F04FFC10BD15710200424C455F0A
:1070A000436C69656E745F527800000015730200CE
:1070B000424C455F436C69656E745F547800000014
:1070C00030B50346104A1068002900DC30BD0022AC
:1070D00014E00D4C2468601C0C4CA04201D3A4F5B4
:1070E00080600B4C2468A04206D09C5C064D2D6845
:1070F0002C70054C206000E002E0521C8A42E8DB64
:1071000000BF00BFE2E7000044400020105900200B
:107110004840002070B565E03348007810B1012880
:107120005BD12BE000F058FC032800D270BD00209A
:1071300000F032FCAA2803D0012000F0B9FC1CE0CA
:10714000022000F029FC0446E043C4B2012000F014
:1071500023FC2649087008460078844209D1084675
:107160000078052805DB20480078401C1E4908707F
:1071700002E0012000F09CFC00BF32E000F02CFC9B
:107180001A490978884200D2D0E70025002406E099
:10719000204600F001FC2844C5B2601CC4B213486C
:1071A0000078401EA042F3DC10490978491E88B2DD
:1071B00000F0F2FBA84208D10C48007803F066FC0E
:1071C0000A48007800F074FC02E0012000F070FC36
:1071D00000200549087000BF03E000200249087044
:1071E00000BF00BF98E70000544000205540002039
:1071F00010B5024610480068122802D34FF0FF3045
:1072000010BD0E480C4B1B6800EB0310C1600B480F
:10721000094B1B6800EB031002700948074B064C32
:10722000246803EB0413586003480068401C024BB9
:1072300018600020E4E700004C40002010590020B6
:10724000305A00202DE9F047C0B0804689461646E6
:1072500000250024701D00F0FF0AFA2E03DD601ED9
:1072600040B0BDE8F087AA200DF804002046611C5C
:10727000CCB21DF800002844C5B20DF804A0204689
:10728000611CCCB21DF800002844C5B26FEA0A00A8
:10729000C0B20DF804002046611CCCB21DF80000FD
:1072A0002844C5B20DF804802046611CCCB21DF8FC
:1072B00000002844C5B200270CE019F807000DF8BB
:1072C00004002046611CCCB21DF800002844C5B261
:1072D000781CC7B2B742F0DB2046611CCCB20DF877
:1072E0000050214668461DF017FFB9E708490AE03B
:1072F0000A68824204D100234376136A0B6001E0DE
:1073000002F1200100BF0A68002AF1D17047000095
:107310005040002070B5002600251E48046831E06A
:10732000E06800282BD005F0D9F81B490968451AF8
:1073300005F0D4F81849086005B90125E068A842AD
:1073400003D3E068401BE06001E00020E060E068FB
:10735000A8B9207A00280ADD207A401E20726068D1
:10736000E060227E207C6169FFF76CFF07E0204629
:10737000FFF7BCFFE06910B12046E1698847607EF5
:107380000643246A002CCBD13146AFF2770003F0DC
:10739000ABFA70BD50400020584000202DE9F0416C
:1073A0000446884615461E4613480768ECB184F823
:1073B0001080656126766068E0602078002803DD33
:1073C0002078401E207201E00020207201206076AB
:1073D00004E0A74201D1BDE8F0813F6A002FF8D157
:1073E0000548006820620448046032462946404649
:1073F000FFF728FF00BFEEE75040002010B5054A18
:1074000005A1002003F096FA064A07A1012003F027
:1074100091FA10BDBD740200424C455F486F737411
:107420005F527800CD760200424C455F486F73741E
:107430005F5478002DE9F04104460D461B4806686C
:10744000052D01DABDE8F0816778A078C04300F02F
:10745000FF082078AA280CD147450AD1AF4208D1AD
:10746000E078052805DAE9B22046114A126890470B
:1074700019E0002014E00D4909684E1C0D498E42A8
:1074800001D3A1F580660C4909688E4206D0215CC3
:10749000064A1268117005490E6000E002E0401CC7
:1074A000A842E8DB00BF00BFCCE700005C40002042
:1074B00064400020305F00206040002070B565E02F
:1074C0003348007810B101285BD12BE000F094FA2A
:1074D000032800D270BD002000F06EFAAA2803D065
:1074E000012000F009FB1CE0022000F065FA0446D0
:1074F000E043C4B2012000F05FFA26490870084654
:107500000078844209D108460078052805DB204828
:107510000078401C1E49087002E0012000F0ECFADF
:1075200000BF32E000F068FA1A490978884200D2B8
:10753000D0E70025002406E0204600F03DFA28446C
:10754000C5B2601CC4B213480078401EA042F3DCF0
:1075500010490978491E88B200F02EFAA84208D1D5
:107560000C48007803F0D2FA0A48007800F0C4FA18
:1075700002E0012000F0C0FA00200549087000BFB9
:1075800003E000200249087000BF00BF98E7000038
:10759000704000207140002010B50246104800687D
:1075A000122802D34FF0FF3010BD0E480C4B1B6861
:1075B00000EB0310C1600B48094B1B6800EB031084
:1075C00002700948074B064C246803EB041358600B
:1075D00003480068401C024B18600020E4E70000EC
:1075E00068400020305F00205060002001460248C3
:1075F0000160002070470000644000202DE9F04742
:10760000C0B080468946164600250024701D00F053
:10761000FF0AFA2E02DD40B0BDE8F087AA200DF87F
:1076200004002046611CCCB21DF800002844C5B2FD
:107630000DF804A02046611CCCB21DF800002844BF
:10764000C5B26FEA0A00C0B20DF804002046611C02
:10765000CCB21DF800002844C5B20DF804802046C5
:10766000611CCCB21DF800002844C5B200270CE014
:1076700019F807000DF804002046611CCCB21DF873
:1076800000002844C5B2781CC7B2B742F0DB2046E0
:10769000611CCCB20DF80050214668461DF056FD25
:1076A00000BFB8E708490AE00A68824204D1002313
:1076B0004376136A0B6001E002F1200100BF0A6803
:1076C000002AF1D1704700006C40002070B5002600
:1076D00000251E48046831E0E06800282BD004F043
:1076E000FDFE1B490968451A04F0F8FE18490860B8
:1076F00005B90125E068A84203D3E068401BE060BB
:1077000001E00020E060E068A8B9207A00280ADDE6
:10771000207A401E20726068E060227E207C6169D1
:10772000FFF76CFF07E02046FFF7BCFFE06910B1F0
:107730002046E1698847607E0643246A002CCBD14D
:107740003146AFF2770003F0CFF870BD6C400020F7
:10775000744000202DE9F0410446884615461E4637
:1077600013480768ECB184F810806561267660687C
:10777000E0602078002803DD2078401E207201E0C0
:10778000002020720120607604E0A74201D1BDE80C
:10779000F0813F6A002FF8D1054800682062044854
:1077A0000460324629464046FFF728FF00BFEEE757
:1077B0006C4000200246002116E00E4850F82100DF
:1077C000904202D14FF0FF3070470A4850F8210034
:1077D00048B909480078401C074B1870054840F824
:1077E00021200020F0E7491C0329E6DB6FF00100AF
:1077F000EAE70000488200204848002002460021B5
:1078000016E00E4850F82100904202D14FF0FF30B0
:1078100070470A4850F8210048B909480078401CD0
:10782000074B1870054840F821200020F0E7491C5C
:107830001029E6DB6FF00100EAE70000B07F0020CE
:107840000E42002030B52DED048B83B0B0EE408A9F
:10785000F0EE608A3148007800285CD018EE900A7B
:10786000FFF723F841EC190B9FED2D0B53EC102B78
:10787000FFF746F804D3F4EEC88AF1EE10FA04D20A
:10788000032003B0BDEC048B30BDB1EE0E0AB4EEA4
:10789000C08AF1EE10FA01D20320F2E79FED220A2E
:1078A00028EE800ADFED210A80EE201ABCEEC10A24
:1078B00010EE100A80B2ADF806009FED1B0A28EE0C
:1078C000000ADFED1A0A80EE201ABCEEC10A10EEA3
:1078D000100A80B2ADF804004FF4C870ADF80A0089
:1078E0000020ADF808001249088901A975DF044697
:1078F000082C0ED0112C0CD05CB100BF25463DB138
:1079000000BF0CA24FF428712846FEF783FC00BF8D
:1079100000BF2046B5E70120B3E700003E48002045
:1079200000000000003B9F4000007A4400409C445F
:10793000308000202E2E5C2E2E5C2E2E5C626C651C
:107940005F6366675C686F73742E63009FED0E2A39
:10795000C0EE022A9FED0D2A22EE822AB0EE421AD4
:107960009FED0B2A21EE022A22EE202ADFED092AC2
:1079700082EE223AF0EE431A90ED002A32EE212AEE
:1079800080ED002A7047000000803B45CDCC8C3F45
:1079900000007A44000061450246054800688118ED
:1079A0000448814201D3A1F5806108787047000046
:1079B0004840002010590020024605480068811800
:1079C0000448814201D3A1F5806108787047000026
:1079D00060400020305F0020054B1A68054B196895
:1079E0008A4201D3501A02E002F58063581A7047A8
:1079F0004440002048400020054B1A68054B196898
:107A00008A4201D3501A02E002F58063581A704787
:107A10005C4000206040002070B58AB00446002021
:107A200009900026182103A8FEF734FD00200190DC
:107A30000290002504F0010008B90AB070BD12F0F0
:107A400061FC022800D0F8E709A808F039FE00B967
:107A5000F3E701A80FF04AFC0646B6F1FF3F08D055
:107A6000BDF8040030B9BDF8060018B9BDF808002B
:107A700000B9E2E70998411E03AA00200BF0F4F8D0
:107A8000B0F1FF3F0ED001A903A814F045F8054658
:107A9000002D07DB0448007810B901200249087066
:107AA00002490D7100BFC8E706400020785300204E
:107AB00018E0411E88B20D4909680D4A12689142CA
:107AC00000D1704709490968491C0A4A914204D308
:107AD000A2F58061054A116004E004490968491C67
:107AE000024A11600028E4D100BFEAE748400020C4
:107AF000444000201059002018E0411E88B20D4972
:107B000009680D4A1268914200D170470949096815
:107B1000491C0A4A914204D3A2F58061054A1160CA
:107B200004E004490968491C024A11600028E4D1B4
:107B300000BFEAE7604000205C400020305F00208A
:107B40000122014B1A707047004100200849095C6E
:107B500001290CD1002206490A54891F898C31B1B0
:107B60000349891F898C491E014A921F91847047DD
:107B700002500020004870472450002070B52DEDC1
:107B8000068B0646164890F8540028BB1448C66475
:107B90001448046800F03AFE0546AC4201D204F1F4
:107BA0008074601BFEF73CFE41EC1A0B9FED0E0B40
:107BB00053EC102BFEF7B4FD41EC190B9FED0C0BB1
:107BC00053EC102BFEF737FD41EC180BFEF754FE7B
:107BD0000349086208464462BDEC068B70BD000094
:107BE000A0FF002004B50040FCA9F1D24D62404046
:107BF000000000000070A740034991F8541009B933
:107C00000149086570470000A0FF002001460348B5
:107C1000405C012800D170470020FCE702500020A2
:107C200010B50021064802F05FFE012005490870EA
:107C30003220488001208880092001F075FC10BDA9
:107C4000497E0200FC4F002010B51A4840880028E9
:107C50002ED00121184802F047FE1648808868B9E6
:107C60001448007818B901201249087002E0002079
:107C70001049087001200F49888014E00D480078F1
:107C800018B90E49092001F02FFC0A480078012894
:107C900004D14FF07F41092001F026FC054880887F
:107CA000401E0449888003484088401E014948809E
:107CB00010BD0000FC4F0020497E020000103FFF75
:107CC00070B50446241F4FF40070B0EB145F00D071
:107CD00070BD08340120094981F854000846806CC1
:107CE00040F002008864202221460448FEF7B9FBD8
:107CF0002546A869C01EA86100BFE9E7A0FF0020D3
:107D00000649095C012908D0012204490A54891F47
:107D1000898C491C014A921F9184704702500020AF
:107D2000F0B5BFB006460F46002400253846FEF7E2
:107D3000BCFB85B2F82D02D9601E3FB0F0BD07F044
:107D40002FFB30B100222046611CCCB20DF8002080
:107D500005E001222046611CCCB20DF8002020462F
:107D6000611CCCB20DF800600DEB04002A463946C8
:107D7000FEF777FB6019C4B222466946AD20FFF7D3
:107D800061FADAE70120064981F854000846806C60
:107D900040F001008864034801680148816270472F
:107DA000A0FF002004B5004010B51648806D0128E2
:107DB00009D05C211348FEF76DFB0120114988654D
:107DC000002081F8540026210F48FEF763FB0120B4
:107DD0000D49087032204880012088800B4A0CA190
:107DE000C82002F0A7FD0E4A0EA1642002F0A2FDF9
:107DF0001249AD20FFF7D0FB242211491148FEF7AC
:107E000030FB10BDA0FF0020FC4F0020497E020087
:107E1000457863657074696F6E5F4C65640000003F
:107E2000B57E0200457863657074696F6E5F556E4C
:107E30006B6F776E52657365740000003B42030000
:107E4000E45300202450002000B589B000200AF03F
:107E500015FF012811DB01AA002108460AF004FFE2
:107E6000BDF80400ADF81C00BDF80600ADF81E001A
:107E7000BDF80800ADF8200001E009B000BDBDF973
:107E8000200040F2DC51884206DB0848808C002844
:107E900002DDFFF7D9FE06E0BDF920000449884263
:107EA00001DCFFF7BDFE00BFE7E70000FC4F00204C
:107EB00024FAFFFF10B52DED048BCAB0FC210BA8EE
:107EC000FEF7E8FAFC210BA8FEF7E4FA554890F813
:107ED0005400012839D15348806C00F0010000287B
:107EE00034D05048846A406AA04201D904F18074B9
:107EF0004C49496A601AFEF793FC41EC190B9FED5F
:107F00004A0B53EC102BFEF70BFC41EC180B8DEDDC
:107F1000028B4448006A00904248036DC26C44A141
:107F20000BA804F079FD0BA91120FFF7F9FE00283A
:107F300073D13C48806C20F001003A4988640846BF
:107F4000806C002869D181F8540066E03548806C67
:107F500000F00200A8B31E223B4B3248C169806981
:107F6000C01ECDE90832CDE906012E4840692D49F1
:107F700009692C4AD2682B4B9B68CDE90232CDE9C6
:107F800004102848406827490968CDE900102548B1
:107F9000036DC26C2D490BA804F03EFD0BA9112006
:107FA000FFF7BEFE002838D11E48806C20F002008A
:107FB0001C4988640846806C20BB002081F854006E
:107FC0002BE0FFE71748806C00F00400D8B115489B
:107FD0002C3000902C38036DC26C1DA10BA804F04E
:107FE0001BFD0BA91120FFF79BFE58B90D48806CB3
:107FF00020F004000B4988640846806C10B900200A
:1080000081F8540009E05C210648FEF743FA01209C
:1080100004498865002081F854004AB0BDEC048B07
:1080200010BD0000A0FF0020FCA9F1D24D6240402D
:1080300069643A307825782C307825782C25642CA2
:1080400025660D0A0000000001040100D86D04003F
:1080500069643A307825782C307825782C2573009F
:10806000704770B50025002600240CE04FF4E62090
:1080700000EB043630461BF0F9FE05460DB1032037
:1080800070BD601CC4B2012CF0DB0020F8E770B5B5
:108090000025002600240CE04FF4E82000EB043615
:1080A00030461BF0E3FE05460DB1032070BD601C99
:1080B000C4B2022CF0DB0020F8E770B500250026E2
:1080C00000240CE04FF4EC2000EB043630461BF0AB
:1080D000CDFE05460DB1032070BD601CC4B2022C5C
:1080E000F0DB0020F8E710B504461C2221464FF4CF
:1080F000E62010F07DF810BD7CB500240020019032
:10810000DA48FFF7F0FF0546D8480068D8498842AA
:108110001FD1D648007E05280FDBFFF7B8FFFFF719
:10812000CCFF0020D149087600F0C0F918B1D1A1E8
:108130000820FFF7F5FD04F0CFFCCC48007E401C82
:10814000CA49087600F0B2F918B1CAA10820FFF7B1
:10815000E7FDCD4815F093F9002436E004EB440127
:10816000CA4A52F82100FEF7A0F9064604EB440083
:10817000C64A52F8201001AB3246C3481AF08DFAB5
:1081800008BB04EB4400C14901EB8000007A9DF874
:108190000410884217D104EB4401BC4A52F8210074
:1081A000FEF783F9064601A8009004EB4400B74AA5
:1081B00002EB8000436804EB440052F82010324682
:1081C000B1481AF02CFA601C84B21A2CC6DBB048F5
:1081D0000068A749884276D0FFF759FFFFF76DFF87
:1081E0009021AB48FEF756F9A148A9490860002044
:1081F00008719E4800689E49884231D100240DE0F4
:108200009A48001D015DA248801D015597480A301B
:10821000015D9F4832300155601C84B2062CEFDBB3
:10822000002401E0601C84B2062CFBDB002401E08A
:10823000601C84B2062CFBDB8C4801699448C16247
:108240008A48818A924801868848807D904981F8D1
:1082500028008648C07D08718448807E48710AE005
:108260001C218248FEF716F900F020F918B181A10F
:108270000820FFF755FD00241EE004EB4401834A6B
:1082800052F82100FEF711F9064604EB44007F493D
:1082900001EB8000007A009004EB44000A4602EBF8
:1082A0008000436804EB440052F8201032467648C0
:1082B0001AF04AF9601C84B21A2CDEDB00207449E3
:1082C0000860002437E044E004EB44016F4A52F8B0
:1082D0002100FEF7EAF8064604EB44006B4A52F828
:1082E000201001AB324668481AF0D7F908BB04EBFE
:1082F0004400664901EB8000007A9DF80410884232
:1083000017D104EB4401614A52F82100FEF7CDF881
:10831000064601A8009004EB44005C4A02EB800092
:10832000436804EB440052F82010324656481AF0D5
:1083300076F9601C84B21A2CC6DB554800684C499B
:10834000884204D053A10820FFF7EAFC7CBD04F06A
:10835000C3FB002485E004EB44014C4A52F82100A1
:10836000FEF7A3F8064604EB4400484A52F82010F2
:1083700001AB324644481AF090F9E0BB04EB4400EC
:10838000424901EB8000007A9DF80410884218D120
:1083900004EB44013D4A52F82100FEF786F80646F8
:1083A00001A8009004EB4400384A02EB80004368C7
:1083B00004EB440052F82010324633481AF02FF9EB
:1083C0004DE004EB4401314A52F82100FEF76DF80C
:1083D000064604EB44002D4A52F8201032462A4843
:1083E0001AF0F7F804EB4401284A52F82100FEF78E
:1083F0005CF8064600E015E004EB4400234901EB7D
:108400008000007A009004EB44000A4602EB8000F2
:10841000436804EB440052F8201032461A481AF020
:1084200093F81CE004EB4401184A52F82100FEF7CF
:108430003CF8064604EB4400144901EB8000007A46
:10844000009004EB44000A4602EB8000436804EB12
:10845000440052F8201032460B481AF075F8601CA0
:1084600084B21A2CFFF677AF00BF6FE708540020E4
:10847000AA5555AA73617665206261636B75702099
:108480006661696C00000000CC3F00204866040073
:1084900078530020466C6173682077726974652098
:1084A00068656164206661696C00000070B5002534
:1084B000002610481049086000240CE04FF4E62024
:1084C00000EB043630461BF0D1FC05460DB103200D
:1084D00070BD601CC4B2012CF0DB072206494FF4CA
:1084E000E6201BF009FD05460DB10220F0E7002053
:1084F000EEE70000AA5555AA08540020F8B500255B
:10850000002422E004EB4401124A52F82100FDF756
:10851000CCFF064604EB44000E4901EB8000007AD4
:10852000009004EB44000A4602EB8000436804EB31
:10853000440052F82010324607481AF0DCF805468D
:108540000DB10220F8BD601CC4B21A2CDADB002089
:10855000F8E7000048660400CC3F0020F8B5064666
:108560000F46144633212248FDF794FF012020498D
:10857000383981F83800012E0CD06FF48050304427
:1085800078B1B0F5405F1CD06FF44051084400282A
:1085900022D10DE0322217A11548401CFDF761FFE2
:1085A00021E0322219A11248401CFDF75AFF1AE0BF
:1085B00025461DA10E48401CD5E9003204F02CFAD6
:1085C00011E02546286800901EA10948401CD5E905
:1085D000013204F021FA06E03A461FA10448401C8B
:1085E00004F01AFA00BF00BFFFF788FFF8BD0000D3
:1085F000B053002053443A20415353455254494FFD
:108600004E204641494C45440D0A000053443A204F
:10861000494E56414C4944204D454D4F52592041F9
:1086200043434553530D0A00415353455254494F58
:108630004E204641494C45442025733A25750D0A84
:10864000000000006572726F723A25752C25733A2E
:1086500025750D0A00000000554E4B4E4F574E2019
:108660004641554C54203078253038580A000000D7
:10867000FEB54948406AB0F5006F7CD208F026FD8F
:10868000074608F029FD3D184FF07F4000EA0560DD
:108690004FF47F0101EA052108434FF47F4101EACD
:1086A0001521084340EA156002903C4800780128F3
:1086B0000ED1FFF702FD28B139A10B20FFF730FBE7
:1086C0000220FEBD00213448416200203349087079
:1086D0003149496A4FF4EC2202EB8100012202A9E0
:1086E0001BF00AFC06460EB10220EAE72A48406A5F
:1086F000401C2949486208464169C161816901629B
:10870000FFF7FCFE18B12AA10820FFF709FB04249B
:108710000020019038E004EB44012B4A52F821007C
:10872000FDF7C3FE074604EB4400274A52F8201029
:1087300001AB3A46254819F0B0FF18BB04EB4400E2
:10874000214901EB8000007A9DF80410884219D17C
:1087500004EB44011C4A52F82100FDF7A6FE07462F
:1087600001A8009004EB4400174A02EB8000436824
:1087700004EB440000E00AE052F820103A461348A7
:1087800019F04DFF601CC4B2052CC4DB01E00220CF
:1087900097E7002095E7000078530020E83F00208D
:1087A000636C6561722073746570206661696C002A
:1087B0007361766520696E666F726D6174696F6E44
:1087C000206661696C00000048660400CC3F002010
:1087D00000200D49096891ED070ABCEEC00A10EEB1
:1087E000101AC8B20A2806DD0A2190FBF1F000EB4E
:1087F00080014906080E642801DD642002E000289B
:1088000000DC0020704700009C4000200148006808
:108810007047000024410020094989790170084906
:10882000497941700649097981700549C978C17053
:108830000349897801710249497841717047000004
:108840001242002000BFEFF30880804600BFEFF324
:10885000098000BF4046FFF733FA0A2404B90DE04F
:1088600000BF4FF47A7505B904E0054EAF013846F4
:10887000B04700BF601E041EF3D100BF04F00CF926
:10888000C165040010B50021132016F098FE0120E8
:1088900017F02AFC0021142016F091FE012017F099
:1088A00023FC0121132016F08AFE012017F01CFC86
:1088B0000021132016F083FE10BD1CB5002000908F
:1088C0000346012211460190132016F07EFC13206E
:1088D00016F056FD132016F0D2FD0020009003463E
:1088E000012211460190142016F06FFC142016F09E
:1088F00047FD142016F0C3FD1CBD10B50021132048
:1089000016F05DFE0121142016F059FE012017F02B
:10891000EBFB0121132016F052FE012017F0E4FBBF
:108920000021132016F04BFE10BD2DE9F041074643
:108930000E4615469846002400F084F8384600F0AC
:1089400057F800F0AFF810B90020BDE8F0813046CC
:1089500000F04EF800F0A6F808B90020F5E700F0A6
:1089600071F8791CC8B200F043F800F09BF808B920
:108970000020EAE7002406E000F012F82855FFF78F
:1089800081FF601CC4B2A8F10100A042F4DC00F039
:1089900007F82855FFF7B1FF00F06CF80120D4E785
:1089A00070B500250121142016F009FE00BF17E064
:1089B0006006040E0021132016F001FE052017F0BA
:1089C00093FB0121132016F0FAFD052017F08CFB14
:1089D000142016F030FD08B144F00104681CC5B243
:1089E000082DE5DB0021132016F0E9FD204670BDBF
:1089F00070B50446002500BF1DE00021132016F0CD
:108A0000DEFD052017F070FB04F0800020B101218D
:108A1000142016F0D4FD03E00021142016F0CFFD41
:108A20006006040E0121132016F0C9FD052017F081
:108A30005BFB681CC5B2082DDFDB0021132016F09C
:108A4000BEFD70BD10B50121142016F0B8FD012146
:108A5000132016F0B4FD052017F046FB002114206A
:108A600016F0ADFD052017F03FFB0021132016F096
:108A7000A6FD10BD10B50021132016F0A0FD0021A9
:108A8000142016F09CFD052017F02EFB0121132069
:108A900016F095FD0121142016F091FD052017F028
:108AA00023FB10BD10B500240121142016F087FD12
:108AB000012017F019FB0121132016F080FD0BE0B7
:108AC000601CC0B20446322803DBFFF7D3FF00204E
:108AD00010BD012017F008FB142016F0ACFC002894
:108AE000EED10021132016F06AFD0120F0E72DE9F8
:108AF000F04180460D4616461F460024FFF7A2FFB0
:108B00004046FFF775FFFFF7CDFF10B90020BDE825
:108B1000F0812846FFF76CFFFFF7C4FF08B900207B
:108B2000F5E7002409E0305DFFF762FFFFF7BAFFC9
:108B300008B90020EBE7601CC4B2BC42F3DBFFF7CE
:108B400099FF0120E3E710B500210E2016F09BFDF0
:108B5000012017F0E1FA00210C2016F094FD01200D
:108B600017F0DAFA01210E2016F08DFD012017F022
:108B7000D3FA00210E2016F086FD10BD1CB5002092
:108B8000009003460122114601900E2016F06DFB65
:108B90000E2016F013FC0E2016F087FC002000902B
:108BA00003460122114601900C2016F05EFB0C20BA
:108BB00016F004FC0C2016F078FC1CBD10B500214A
:108BC0000E2016F060FD01210C2016F05CFD012046
:108BD00017F0A2FA01210E2016F055FD012017F022
:108BE0009BFA00210E2016F04EFD10BD2DE9F0413C
:108BF00007460E4615469846002400F084F838468D
:108C000000F057F800F0AFF810B90020BDE8F0818F
:108C1000304600F04EF800F0A6F808B90020F5E75D
:108C200000F071F8791CC8B200F043F800F09BF82E
:108C300008B90020EAE7002406E000F012F8285501
:108C4000FFF781FF601CC4B2A8F10100A042F4DC70
:108C500000F007F82855FFF7B1FF00F06CF801208D
:108C6000D4E770B5002501210C2016F00CFD00BFE3
:108C700017E06006040E00210E2016F004FD05200A
:108C800017F04AFA01210E2016F0FDFC052017F01E
:108C900043FA0C2016F0E7FB08B144F00104681C0D
:108CA000C5B2082DE5DB00210E2016F0ECFC2046B5
:108CB00070BD70B50446002500BF1DE000210E20E8
:108CC00016F0E1FC052017F027FA04F0800020B12F
:108CD00001210C2016F0D7FC03E000210C2016F037
:108CE000D2FC6006040E01210E2016F0CCFC0520FB
:108CF00017F012FA681CC5B2082DDFDB00210E2028
:108D000016F0C1FC70BD10B501210C2016F0BBFCA3
:108D100001210E2016F0B7FC052017F0FDF9002107
:108D20000C2016F0B0FC052017F0F6F900210E20FB
:108D300016F0A9FC10BD10B500210E2016F0A3FC02
:108D400000210C2016F09FFC052017F0E5F9012109
:108D50000E2016F098FC01210C2016F094FC052042
:108D600017F0DAF910BD10B5002401210C2016F01F
:108D70008AFC012017F0D0F901210E2016F083FCA7
:108D80000BE0601CC0B20446322803DBFFF7D3FFC0
:108D9000002010BD012017F0BFF90C2016F063FB76
:108DA0000028EED100210E2016F06DFC0120F0E726
:108DB0002DE9F04180460D4616461F460024FFF778
:108DC000A2FF4046FFF775FFFFF7CDFF10B9002067
:108DD000BDE8F0812846FFF76CFFFFF7C4FF08B934
:108DE0000020F5E7002409E0305DFFF762FFFFF7A0
:108DF000BAFF08B90020EBE7601CC4B2BC42F3DB49
:108E0000FFF799FF0120E3E710B50548007828B186
:108E1000044B054A0549064800F0DAF810BD000089
:108E20005848002075AB03006C4800205C480020C7
:108E3000EA8300200120014908707047584800204B
:108E40000020014908707047584800202DE9FC5F58
:108E500005460E4617469846DDE90CB9DDF838A000
:108E60004248007868B15B46424639463046CDE913
:108E7000009A1AF03FF83E49A1F1500010F034FF7B
:108E80000CE05B46424639463046CDE9009A0CF08C
:108E9000DBF83749A1F150000CF088F8304615F0A6
:108EA0008BF90446002C5ED0CDB33048007828B151
:108EB0002F4950392F481AF0B1F954E02E4890F854
:108EC00050302B48503890F850102B4A0CF096F840
:108ED0002A49A1F150000CF07DF828485038B0F82C
:108EE0005200401C25495039A1F85200084690F81C
:108EF000521090F85000401C204A503A115410462D
:108F0000B0F852000012114691F85010505410461B
:108F100090F85030042100201CF040F923E0FFE7D6
:108F200013485038B0F85200401C11495039A1F88C
:108F30005200084690F8521090F85000401C0C4A1D
:108F4000503A11541046B0F852000012114691F8F0
:108F500050105054104690F85000801CC3B20421A9
:108F600000201CF01BF9BDE8FC9F000058480020C1
:108F7000928300205C480020EE820020E6830020DF
:108F800070B504460D46E07804281AD16278211D98
:108F90000C48FDF766FA6078C01F0A4981F8500056
:108FA0006078801E215C6078C01E205C41EA002051
:108FB0000449A1F852000448007810B103481AF09F
:108FC0002DF970BDEE820020584800206C4800202A
:108FD0002DE9F04104460E4615461F4665480078C7
:108FE00010B101280CD10CE06889002808DD0120AF
:108FF0006049087028461AF0C7F930461AF0C4F9DB
:10900000B5E008E004F1540128461AF027F9B4F855
:10901000A60059490880688971898842F2DC68890C
:10902000002867DD04F1540128461AF017F9524868
:109030000088401C50490880B4F8A600098888427E
:1090400059D000BF4D480088401C4C4908804A4810
:109050000088401C48490880214630461AF0FEF836
:10906000B4F852004449098888423BD12146304631
:109070001AF0F4F894F8A43094F8501004F1540263
:109080002046B8473E49A1F1500010F03FFE3C4851
:109090005038B0F85200401C39495039A1F85200FC
:1090A000084690F8521090F85000401C344A503A4C
:1090B00011541046B0F852000012114691F85010A9
:1090C00050541146B1F8520000EBD0714910A0EB9A
:1090D000410131B9104690F85030042100201CF0B5
:1090E0005DF807E07089002803DC00202149087042
:1090F00000E0A7E73AE0214630461AF0AFF894F8CE
:10910000A43094F8501004F154022046B8471C498A
:10911000A1F1500010F0FAFD19485038B0F8520093
:10912000401C17495039A1F85200084690F85210D7
:1091300090F85000401C124A503A11541046B0F8B2
:1091400052000012114691F8501050541146B1F8D7
:10915000520000EBD0714910A0EB410131B910462B
:1091600090F85030042100201CF018F800BF00BF18
:10917000BDE8F0817C4800207E480020C83F0020E8
:10918000E683002070B505460C460020264908609D
:1091900026480021016041608160254801604160EE
:1091A00081604FF4A2712348FDF774F92248002131
:1091B0000160416081602148016041608160204818
:1091C00001604160816024211E48FDF763F924217C
:1091D0001D48FDF75FF96C211C48FDF75BF94FF462
:1091E000A2711B48FDF756F924211A48FDF752F9E0
:1091F00024211948FDF74EF924211248FDF74AF9B8
:1092000024211148FDF746F9144890ED000A214643
:10921000114811F0C9FB24220F491148FDF721F92B
:1092200000201049086070BDE44900201C8E002019
:10923000288E0020508A0020948B0020048E00206D
:10924000108E0020A08B0020C48B0020E88B002013
:10925000548C0020988D0020BC8D0020DC4900201B
:10926000E08D0020084A00202DE9F0432DED048B0D
:1092700087B081460D4600270026182101A8FDF77A
:1092800009F9B0460024288810FB00F06A8812FB18
:109290000200AA8812FB020000EE100AB8EEC00A13
:1092A00010EE101A0846FDF700FB41EC190BB0EE6A
:1092B000490AF0EE690A04F0F7FAB0EE408AF0EEDF
:1092C000608A51EC180BFDF7B8FA06462A48007878
:1092D00001280CD100202849087000BF04E027486D
:1092E00040F82460601CC4B2062CF8DB0DE00024BA
:1092F00007E02249601C51F8200041F82400601C5E
:10930000C4B2052CF5DB1D48466118221B4901A893
:10931000FDF7A7F800211FE0002017E001AA52F88E
:1093200020309446421C5CF8222093420CDD01ABB5
:10933000421C53F8228001AA52F82030421C4CF8FB
:10934000223001AA42F82080421CD0B2C1F10502AD
:109350008242E3DC481CC1B20529DDDB0199069895
:10936000401AB0F57A7F00DB0127384607B0BDEC24
:10937000048BBDE8F0830000B04000208471002021
:1093800010B50121102016F0E0F800200149087006
:1093900010BD0000C04000202DE9F041012002F086
:1093A000F5F8FF231A461946112002F0F5F80320BC
:1093B00002F002F901F0FEFB00231A466021164874
:1093C00001F0FCFB15490860102001210A4600232A
:1093D00006241D4600BF4FF0A0473E4641EA420723
:1093E00047EA830747EA042747EA054C06F5E067A2
:1093F00047F820C000BF002116F0A7F8084A09A1CD
:10940000052001F097FA084802F008F9074803F030
:10941000DBFABDE8F08100009C710020BC40002018
:10942000319402004C4544000347030015470300F4
:1094300010B500242048007810B1012835D126E06D
:109440001E48007810B300201C49087009240DE064
:109450001B4810F83400002806DD194901EBC4014F
:10946000486803F0A9F903E0601EC4B2002CEFDCE9
:1094700000BF24B90121102016F067F806E0002192
:10948000102016F062F801200B49087011E00B481B
:10949000007818B100200849087005E00122042175
:1094A0000848006802F08EF803E0002002490870C6
:1094B00000BF00BF10BD0000C1400020C040002020
:1094C0005C720020BC4000200A2800DB7047044A80
:1094D00002EBC00251600122024B1A7000BFF5E797
:1094E0005C720020C04000200A2800DB70470C4A54
:1094F00012F83020012A06D1094A02EBC002526854
:109500008A4200D1F2E70122054B03F830201A46C7
:1095100002EBC00251600122024B1A7000BFE5E766
:109520005C720020C04000200A2800DB7047074919
:1095300011F8301001B9F9E70021044A02F830109F
:109540000121034A117000BFF0E700005C720020A7
:10955000C040002010B50021052016F045F801207C
:1095600016F0CEFD0021042016F03EF8012016F082
:10957000C7FD0121052016F037F8012016F0C0FDC7
:109580000021052016F030F810BD1CB50020009019
:109590000346012211460190052015F02AFE052000
:1095A00015F0FDFE052015F075FF0020062103468D
:1095B0000122CDE900101146042015F01AFE042006
:1095C00015F0EDFE042015F065FF062015F099FE5C
:1095D0000121062016F008F8032015F092FE1CBDAC
:1095E00010B50021052015F0FFFF0121042015F022
:1095F000FBFF012016F084FD0121052015F0F4FF8A
:10960000012016F07DFD0021052015F0EDFF10BDB5
:109610002DE9F04107460E4615469846002400F015
:1096200084F8384600F057F800F0BDF810B9002073
:10963000BDE8F081304600F04EF800F0B4F808B90B
:109640000020F5E700F071F8791CC8B200F043F88B
:1096500000F0A9F808B90020EAE7002406E000F0CD
:1096600012F82855FFF776FF601CC4B2A8F101007C
:10967000A042F4DC00F007F82855FFF7B1FF00F036
:109680006CF80120D4E770B500250121042015F005
:10969000ABFF00BF17E06006040E0021052015F0A7
:1096A000A3FF052016F02CFD0121052015F09CFFDD
:1096B000052016F025FD042015F0C9FE08B144F080
:1096C0000104681CC5B2082DE5DB0021052015F05A
:1096D0008BFF204670BD70B50446002500BF1DE01D
:1096E0000021052015F080FF052016F009FD04F08B
:1096F000800020B10121042015F076FF03E0002155
:10970000042015F071FF6006040E0121052015F0FC
:109710006BFF052016F0F4FC681CC5B2082DDFDBDA
:109720000021052015F060FF70BD10B50121042057
:1097300015F05AFF0121052015F056FF052016F0FF
:10974000DFFC0021042015F04FFF052016F0D8FCA7
:109750000021052015F048FF10BD10B5002105209F
:1097600015F042FF0021042015F03EFF052016F001
:10977000C7FC0121052015F037FF0121042015F059
:1097800033FF052016F0BCFC10BD10B5052015F008
:10979000A0FD042015F09DFD062015F09AFD032084
:1097A00015F097FD10BD10B500240121042015F01F
:1097B0001BFF012016F0A4FC0121052015F014FF69
:1097C0000BE0601CC0B20446322803DBFFF7C5FF84
:1097D000002010BD012016F093FC042015F037FE88
:1097E0000028EED10021052015F0FEFE0120F0E753
:1097F0002DE9F04180460D4616461F460024FFF72E
:1098000094FF4046FFF767FFFFF7CDFF10B9002038
:10981000BDE8F0812846FFF75EFFFFF7C4FF08B9F7
:109820000020F5E7002409E0305DFFF754FFFFF763
:10983000BAFF08B90020EBE7601CC4B2BC42F3DBFE
:10984000FFF78BFF0120E3E77CB51448007900B9EE
:109850007CBD06F0C1FDF8B1002510F0F9FF4042D3
:10986000C6B20F48058800242A122146641C0DF850
:109870000120EAB22146641C0DF801202146641C37
:109880000DF8016023466A4603210020FDF786FD9E
:1098900000200349088000BF00BFD9E778530020AB
:1098A000C83F00202DE9F041022001210A46002492
:1098B0002346254600BF4FF0A0473E4641EA4207F7
:1098C00047EA840747EA032747EA054C06F5E067BD
:1098D00047F820C000BF00BF002115F019FEC820C6
:1098E00000F01AF8084802F051FE084A08A10020CA
:1098F00001F020F80121054800F0F6FF0549A420F9
:10990000FDF776FCBDE8F0813D990200E199020087
:109910004D5400002140030010B504464CB10548E9
:1099200004600121022015F0F3FD0121024800F03E
:10993000DBFF10BD78400020E199020010B504461D
:1099400023480068002842D02148006868B32048B6
:109950000068401E1E4908601E480068082809D09B
:109960000121022015F0D4FD1A480068401C194955
:1099700008600CE018480068022808D01648006803
:10998000401C154908600021022015F0C1FD114856
:109990000068082810D11048006802280CD1002067
:1099A0000D4908600B49086006E00020084908607E
:1099B00009490860074908600548006838B900216E
:1099C000022015F0A5FD0021044800F08DFF10BD18
:1099D00078400020804000207C400020E199020077
:1099E00070470000DFED150AC0ED000ADFED140A34
:1099F000C0ED010AF7EE000AC0ED020ADFED0F0A22
:109A0000C0ED030ADFED0D0AC0ED040ADFED0B0A1D
:109A1000C0ED050ADFED090AC0ED060ADFED070A11
:109A2000C0ED070ADFED050AC0ED080AF7EE000AEF
:109A300080EE801A80ED091A7047000000000000D7
:109A40000000C842014890ED0B0A7047785400208E
:109A5000014890ED0A0A704778540020014890EDC3
:109A60000C0A704778540020F0EE400AF6EE001A17
:109A700060EEA11AB0EE611AB0EE600A10EE100AA4
:109A80000C49A1EB600000EE100A21EE002AF7EE6F
:109A9000081A42EE401A61EE801AB0EE610A21EE19
:109AA000002AF7EE081A42EE401A61EE801AB0EE74
:109AB000610A7047DF59375F2DE9F041C0B00746B2
:109AC0008846164600240025AA200DF804002046EA
:109AD000641C1DF800002844C5B205200DF80400E0
:109AE0002046641C1DF800002844C5B2AF200DF8C4
:109AF00004002046641C1DF800002844C5B20DF87F
:109B000004702046641C1DF800002844C5B2F0B261
:109B10000DF804002046641C1DF800002844C5B25E
:109B200000200AE018F800100DF804102146641C0B
:109B30001DF801102944CDB2401CB042F2DB204692
:109B4000641C0DF80050A1B268461BF0E5FA40B065
:109B5000BDE8F08110B52DED108B98B00446F0EE05
:109B6000409AB0EE60AAF0EE41AAF0EE61CAB0EE03
:109B700042BAF0EE62BAB0EE43CAF0EE638AB0EEDB
:109B8000449A9FEDFE0A84ED110AC4ED12CA84EDD9
:109B900013BAC4ED14BAF5EEC0CAF1EE10FA09D149
:109BA000B5EEC0BAF1EE10FA04D1F5EEC0BAF1EE9E
:109BB00010FA7CD06CEEAC0A4BEE0B0A4BEEAB0A03
:109BC000B0EE600AFFF750FFB0EE408A2CEE880A34
:109BD000F0EE40CA2BEE080AB0EE40BA2BEE880A2F
:109BE000F0EE40BA6CEE0C0A48EEA80A49EE090AFB
:109BF000B0EE600AFFF738FFB0EE408A2CEE080A9C
:109C0000B0EE40CA28EE880AF0EE408A29EE080A33
:109C1000B0EE409A94ED020A20EE000A8DED170A8C
:109C200094ED020AD4ED030A20EE20EA94ED020A34
:109C3000D4ED040A20EE20DA94ED020AD4ED050AF0
:109C400020EE200A8DED160A94ED030A20EE000A9C
:109C50008DED150A94ED030AD4ED040A20EE200AD6
:109C60008DED140A94ED030AD4ED050A60EE20DAB6
:109C700094ED040A60EE00EA94ED040AD4ED050ABE
:109C800020EE20FA94ED050A60EE00FAB6EE000A26
:109C900030EE6E0A30EE6F0A20EE0C1A9DED140ABB
:109CA000DDED160A70EE600AB0EE410A00E045E113
:109CB00008EEA00A7DEE8D0A09EE200AF0EE000AF9
:109CC00060EE200ACDED130A9DED140ADDED160AB3
:109CD00030EE200A60EE0C0A9DED150AB6EE001A71
:109CE00031EE400A30EE6F1AB0EE600A08EE810ADB
:109CF0007FEE4E0A09EE200AF0EE000A60EE200A1E
:109D0000CDED120ADDED130A20EEA01ADDED120AE8
:109D100000EEA01AB0EE410A03F003FE8DED110A29
:109D20003DEECD0A20EE0C0A7FEE0E0A08EEA00AE8
:109D3000DDED150AB6EE001A71EE600A70EEEE0A5D
:109D400009EE200AF0EE000A20EE200A8DED100A3E
:109D50003DEECD0A8DED0F0A3EEE0F0A8DED0E0A97
:109D60009DED170AF6EE000A30EE600A30EE2F0A7B
:109D70008DED0D0AB6EE000A30EE6E0A70EE6F0A37
:109D80009DED110A20EE800A3DEECD1ADDED100AA0
:109D900000EE810A8DED0C0A9DED140ADDED160A28
:109DA00070EE600A9DED110A20EE800A3EEE0F1A59
:109DB000DDED100A00EE810A8DED0B0A7DEE2D0A15
:109DC0009DED110A20EE801A9DED150AF6EE000AAF
:109DD00030EEC00A70EE6E1ADDED100AB0EE410AE8
:109DE00000EEA10A8DED0A0A9DED0D0A6BEE000A48
:109DF0009DED0E0A4BEEC00A9DED0A0A28EE801A70
:109E00009DED0B0A09EE401A30EE810A8DED090A2C
:109E10009DED0F0A6BEE800A9DED0D0A4CEEC00A17
:109E20009DED0C0A29EE001A9DED0A0A0CEE401A6F
:109E300030EE810A8DED080A9DED0E0A6CEE800A67
:109E40009DED0F0A4BEE400A9DED0B0A2CEE001A19
:109E50009DED0C0A08EEC01A30EE810A8DED070A5E
:109E600094ED000AB5EEC00AF1EE10FA3CDD94ED77
:109E7000060A94ED001ADDED090A61EE200A94ED60
:109E8000091A00EE810A84ED060A94ED070A94EDA2
:109E9000001ADDED080A61EE200A94ED091A00EEC1
:109EA000810A84ED070A94ED080A94ED001ADDEDAD
:109EB000070A61EE200A94ED091A00EE810A84ED8A
:109EC000080A94ED060A30EE290AF0EE409A94ED65
:109ED000070A30EE0A0AB0EE40AA94ED080A30EE06
:109EE0002A0AF0EE40AA0BE09FED240A84ED060A50
:109EF0009FED220A84ED070A9FED200A84ED080AEF
:109F000094ED011A9DED090AF0EE690A41EE000A8E
:109F1000F0EE609A94ED011A9DED080AF0EE4A0AFF
:109F200041EE000AB0EE60AA94ED011A9DED070A19
:109F3000F0EE6A0A41EE000AF0EE60AA94ED090A1A
:109F4000F6EE000A20EE200A20EE290AF0EE409AF2
:109F500094ED090AF6EE000A20EE200A20EE0A0A25
:109F6000B0EE40AA94ED090AF6EE000A20EE200AAF
:109F700020EE2A0AF0EE40AA02E0000000000000F5
:109F800094ED020A8DED060A94ED030A8DED050AA3
:109F900094ED040A8DED040A9DED050AB1EE400A28
:109FA00060EE290A9DED040A40EE4A0A94ED050A86
:109FB00040EE6A0A94ED020A30EE800A84ED020A4D
:109FC0009DED060A20EE290ADDED040A00EEAA0A3C
:109FD000D4ED050A00EECA0AD4ED030A30EE200AD9
:109FE00084ED030A9DED060A60EE0A0A9DED050A5E
:109FF00040EE6A0A94ED050A40EE290A94ED040A3F
:10A0000030EE800A84ED040A9DED060A20EE2A0A4D
:10A01000DDED050A00EE8A0ADDED040A00EEE90A2C
:10A02000D4ED050A30EE200A84ED050AD4ED020ACB
:10A0300060EEA00A94ED031AD4ED031A41EE210A52
:10A0400094ED041AD4ED041A41EE210A94ED051A98
:10A05000D4ED051A41EE210AB0EE600AFFF704FDC7
:10A06000B0EE408A94ED020A20EE080A84ED020A5E
:10A0700094ED030A20EE080A84ED030A94ED040A25
:10A0800020EE080A84ED040A94ED050A20EE080A81
:10A0900084ED050AD4ED031A94ED032AB6EE001AF6
:10A0A00001EEC21AD4ED041A94ED042A01EEC21A8C
:10A0B000F0EE410A94ED021AD4ED031A21EE211AB2
:10A0C000D4ED041A94ED052A01EE821AB0EE410A8D
:10A0D00003F0EEF9DFED390A20EE200A84ED0A0ADA
:10A0E000D4ED030A94ED051A60EE810A94ED021A8C
:10A0F000D4ED041A41EE610AB8EE001A60EE810A4E
:10A10000B0EE600A02F0D8FEDFED2C0A20EE200A45
:10A1100084ED0B0AD4ED041A94ED042AB6EE001A6D
:10A1200001EEC21AD4ED051A94ED052A01EEC21A09
:10A13000F0EE410A94ED031AD4ED041A21EE211A2F
:10A14000D4ED021A94ED052A01EE821AB0EE410A0E
:10A1500003F0AEF9DFED190A20EE200A84ED0C0AB7
:10A1600094ED020A84ED0D0A94ED030A84ED0E0AC3
:10A1700094ED040A84ED0F0A94ED050A84ED100AAB
:10A1800004F1440204F13401684618F0DEFF04F1E2
:10A19000340018F0C7FF04F13402694604F14400AA
:10A1A00018F0D3FF94ED140AF7EE000A30EE600ABF
:10A1B00084ED140A18B0BDEC108B10BDE12E654281
:10A1C00010B54FF4807014F094FE80B14FF480709D
:10A1D00014F098FE012014F09FFE2048407930B919
:10A1E00001201E49487108460168002088474FF445
:10A1F000827014F07EFE50B14FF4827014F082FE33
:10A20000022014F089FE15480168012088474FF4A8
:10A21000887014F06EFE50B14FF4887014F072FE26
:10A22000102014F079FE0D480168022088474FF491
:10A23000867014F05EFE80B10020094908604FF47A
:10A24000867014F05FFE082014F066FE00200349BB
:10A250008871084601680320884710BDB04A002075
:10A26000340C004010B51CF035F800F013F8FFF77F
:10A2700093F8FFF717FBFDF73FFFFDF795FD10BDC6
:10A2800010B50249024811F0E3FB10BDC04A00209E
:10A2900000C0014010B5034A03A147F2305000F05E
:10A2A00049FB10BD45A30200505752002DE9F04173
:10A2B000FFF766F808F0B8FC0DF050F80220002116
:10A2C00061B900BF00BF4FF0A0421346012505FA57
:10A2D00000F2C3F80C2500BF00BF0CE000BF00BFB8
:10A2E0004FF0A0421346012505FA00F2C3F80825F5
:10A2F00000BF00BF00BF00BFC82014F01FFEFCF766
:10A30000B4FC04211C20FCF705FD1C2200200221C6
:10A3100000231D461E4600BF4FF0A04C674643EA8F
:10A32000450C4CEA800C4CEA062C4CEA014C07F533
:10A33000E06848F822C000BF00BF33DF0446BDE834
:10A34000F081000010B5FEF743FA002833D10FF07A
:10A3500019FF01282FD1FEF78BF918B116A10D2096
:10A36000FDF7DEFC242218491848FCF77AF8002093
:10A3700017494876FEF79AF818B116A10D20FDF797
:10A38000CFFCFEF7BBF818B118A10D20FDF7C8FCF3
:10A390004FF47A70FFF7C0FA0DF08CFE002406E04F
:10A3A00005F09EF8642014F0C9FD601CC4B20A2CAC
:10A3B000F6DBFFF77BFF10BD736176652073746574
:10A3C00070206661696C000024500020E453002076
:10A3D0000854002070777220736176652062616393
:10A3E0006B7570206661696C0000000070777220E8
:10A3F0007361766520696E666F726D6174696F6EE8
:10A40000206661696C00000010B5044694F91300E1
:10A4100010F1140F28DDA08B102825D113480078E7
:10A4200010BBA069007A46281ED1A069407A552841
:10A430001AD1A069807A4E2816D1A069C07A5F2807
:10A4400012D101200949087010210948FCF722F8AF
:10A450000749A06982680A60C0684860002000E07F
:10A46000401CA18B8142FBDC10BD00003F4000205E
:10A470000055002010B52DED048BF0EE408AB0EEB3
:10A48000608A9FEDD20AB0EE409AD148006890F8F9
:10A49000210020B1012870D002286CD1D7E0B3EEA2
:10A4A000040AB4EEC08AF1EE10FA1BDD0220C8499E
:10A4B000096881F82100B0EE680A0AF01DFBC44863
:10A4C000006880ED050AC2480068D0ED050AB0EECC
:10A4D000600AF0EE490A12F03DFCBD48006880EDCC
:10A4E000060A48E0B0EE680A02F0E8F8B8480068EA
:10A4F00080ED050A0120B649096881F82100B2EE15
:10A50000040AC8EE800AF0EE609AB0EE690A10F014
:10A51000B5FEAF480068D0ED050A30EE600AF2EEF5
:10A520000E0AB4EEE00AF1EE10FA16DCB2EE040AFE
:10A53000C8EE800AF0EE609AB0EE690A10F09EFE56
:10A54000A3480068D0ED050A30EE600AFAEE0E0A64
:10A55000B4EEE00AF1EE10FA0DD2B2EE040AC8EE43
:10A56000800AF0EE609AB0EE690A10F087FE984813
:10A57000006880ED050A20E1FFE7B3EE040AB4EEBF
:10A58000C08AF1EE10FA19DD02209149096881F8BC
:10A5900021009FED900A8E48006880ED030A8C48E8
:10A5A0000068D0ED050AB0EE600AF0EE490A12F03C
:10A5B000D1FB8748006880ED060A47E0B0EE680AE4
:10A5C00002F07CF88248006880ED040A8048006848
:10A5D00090ED040A7E480068D0ED050A30EE600A6E
:10A5E000F2EE0E0AB4EEE00AF1EE10FA10DC784852
:10A5F000006890ED040A76480068D0ED050A30EE58
:10A60000600AFAEE0E0AB4EEE00AF1EE10FA08D291
:10A610006F48006890ED040A6D48006880ED050AF7
:10A6200014E06B48006890ED050A69480068D0EDB9
:10A63000040AB4EEE00AF1EE10FA07DD644800689F
:10A6400090ED040A6248006880ED050AB5E0B3EEBB
:10A65000040AB4EEC08AF1EE10FA27D201205C4958
:10A66000096881F82100B2EE040AC8EE800A584851
:10A670000068C0ED000A5648006890ED050ADFED5D
:10A68000560AB4EEE00AF1EE10FA0EDD0AF094FA82
:10A6900000280AD01E2014F0C2FE002805D19FED2C
:10A6A0004F0A4B48006880ED050A85E0484800687D
:10A6B00090ED050ADFED4A0AB4EEE00AF1EE10FA79
:10A6C00000DD7AE0F7EE000A414800681830B0EE8D
:10A6D000480AFDF73BF93E480068D0ED060AB0EEA7
:10A6E000600AF0EE490A01F0DDFF3948006880EDAC
:10A6F000020AB0EE680A0AF0FFF93548006880EDFA
:10A70000040A9FED380AC8EE000A31480068C0ED1F
:10A71000030A2F48006890ED030AF7EE000AB4EE32
:10A72000E00AF1EE10FA05DDB7EE000A28480068ED
:10A7300080ED030A2648006890ED030AF7EE000A50
:10A7400030EEC00A22480068D0ED040A20EE200A4C
:10A750001F480068D0ED030A1D48006890ED021AFA
:10A7600000EE810A1A48006880ED040A1848006863
:10A7700090ED050A16480068D0ED040AB4EEE00A30
:10A78000F1EE10FA07D21248006890ED040A104862
:10A79000006880ED050A0E48006890ED050ADFEDBF
:10A7A0000F0AB4EEE00AF1EE10FA05DB9FED0C0A99
:10A7B0000748006880ED050A00BF00BF0448006834
:10A7C00090ED050ABDEC048B10BD00000000AF4306
:10A7D0009C400020000000003333C6420000C84205
:10A7E000CDCCC74200007A4410B54FF496610348BF
:10A7F000FBF750FE00200249087010BD4C4B0020B2
:10A80000D63D002070B50025002400BF50E004EBC9
:10A810008401324A02EB81018868FDF7AFF904EB4D
:10A8200084002E4901EB8000007B00B93EE004EB80
:10A8300084002A4901EB8000806870B328480668CC
:10A8400004EB840001EB8000408838B904EB8401FC
:10A85000224A02EB8101886880471DE001F03EFE3C
:10A8600004EB84011D4A02EB81014968401A04EBA4
:10A87000840102EB8101498888420DD301F02EFE4C
:10A8800004EB8401154A02EB8101486004EB84016A
:10A8900002EB81018868804700BF04EB84010F4A06
:10A8A00002EB81018868FDF7A7F900BF601CC4B204
:10A8B0000C4800788442AADB002408E004EB840002
:10A8C000064911F8200000B10125601CC4B20548FA
:10A8D00000788442F2DB284670BD00004C4B00201B
:10A8E00004B50040D63D002030B50246002017E0F8
:10A8F00000EB80030D4C04EB83039B6893420DD166
:10A9000000EB800314F823308B4206D001F00103E2
:10A9100000EB8004054D05F8243030BD431CD8B24F
:10A92000034B1B789842E3DB00BFF6E74C4B00205B
:10A93000D63D00202DE9F04105460F46164600247D
:10A9400021E004EB84002E4901EB80008068B042D6
:10A9500017D1012004EB8401294A02EB810108731D
:10A9600004EB8400114601EB8000458001F0B6FD48
:10A9700004EB8401224A02EB810148600120BDE81A
:10A98000F081601CC4B21F4800788442D9DB1D48A6
:10A9900000783C2802DB4FF0FF30F0E719480078E0
:10A9A00000EB8000164901EB80008660012015490C
:10A9B000097801EB8101124A02EB81010873114809
:10A9C000007800EB8000114601EB8000458001F02B
:10A9D00085FD0C49097801EB8101094A02EB8101EF
:10A9E00048600848007800EB8000114601EB8000C9
:10A9F000076104480078401C024908700020BEE747
:10AA00004C4B0020D63D002010B50146002015E03B
:10AA100000EB80020C4B03EB820292688A420BD15E
:10AA2000002200EB8003084C04EB83031A7300EB55
:10AA3000800304F8232010BD421CD0B2034A1278D0
:10AA40009042E5DB00BFF6E74C4B0020D63D0020EE
:10AA500010B5024600200FE000EB8003094C04EB28
:10AA600083039B68934205D100EB800304EB8303CF
:10AA7000598010BD431CD8B2034B1B789842EBDBC6
:10AA800000BFF6E74C4B0020D63D00202DE9F041F9
:10AA900005460320FCF780FF0746052D01DABDE8D7
:10AAA000F081002426E0174800EB04100078B8423B
:10AAB0001FD1144800EB0410C068D0B1002609E093
:10AAC000311D88B2FCF768FF0E4901EB041149689B
:10AAD0008855761C681FB042F2DC0A4901EB04116C
:10AAE0000872084A02EB041002EB0412D16888478E
:10AAF00004E0641C044800688442D4D300BF00BF53
:10AB0000CDE70000105900204C400020F0B5C1B046
:10AB100005460320FCF750FF0746052F12DA0024F4
:10AB200006E0211D88B2FCF747FF01A90855641C07
:10AB3000681FA042F5DCC3B201AA39460020FCF729
:10AB400009FE00BF052D01DA41B0F0BD002426E06A
:10AB5000164800EB04100078B8421FD1134800EBF0
:10AB60000410C068D0B1002609E0311D88B2FCF79E
:10AB700023FF0E4901EB041149688855761C681FB4
:10AB8000B042F2DC094901EB04110872074A02EBFA
:10AB9000041002EB0412D168884704E0641C0448E6
:10ABA00000688442D4D300BF00BFCDE7305F0020EF
:10ABB0006840002010B500F025F810BD2DE9F041E7
:10ABC00007460C4615461E460848807A30B10020DC
:10ABD00000F0ECFC00F00EF8FFF7ECFF0448076013
:10ABE00084808560C660BDE8F081000014410020CB
:10ABF0009C79002010B5024815F01EFC10BD000025
:10AC00000C41002070B50025084809490268094830
:10AC100015F046FB044604B16D1E681C20B9064AB7
:10AC200006A10020FFF786FE70BD00002041002035
:10AC3000144100200C4100206133030070776D5FE8
:10AC4000696E69740000000010B5034A1068034A79
:10AC50001168884710BD0000084B0020044B0020FD
:10AC600010B504220021024810F096FE10BD00002D
:10AC7000004002402DE9F0472DED068B86B00546D9
:10AC80000E4617464FF00008C146C246002005E0B8
:10AC900035F9101003AA42F82010401C0328F7DBF6
:10ACA0000598002801DB014600E04142884600206B
:10ACB00004E036F910104DF82010401C0328F8DB92
:10ACC0000298002801DB014600E041428946ED4838
:10ACD000007803280CDBEC484068EB490860084624
:10ACE000806848600220E74908700120E749086051
:10ACF000E44801780078401CE24A1070E24840F8CD
:10AD00002180E348007803280CDBE2484068E149F1
:10AD100008600846806848600220DD49087001200C
:10AD2000DA490860DA4801780078401CD84A107087
:10AD3000D84840F82190D848007803280CDBD74841
:10AD40004088D64908800846808848800220D24939
:10AD500008700120CD490860B888404201B2CE4851
:10AD600002780078401CCC4B1870CC4820F81210A8
:10AD7000C648006801287DD1C3488068C249496837
:10AD8000401A12D4C648008820B9BF488068C54917
:10AD9000086011E0BC488068C249096888420BDD40
:10ADA000B9488068BF49086006E0BD48008818B906
:10ADB000B5488068BC490860B6488068B5494968AC
:10ADC000401A12D4B948008820B9B2488068B849FE
:10ADD000086011E0AF488068B549096888420BDD1A
:10ADE000AC488068B249086006E0B048008818B9ED
:10ADF000A8488068AF490860A3488068AA490968E4
:10AE0000401A40F24C41884212DD0120A4490880DA
:10AE10009D488068A4490968401AA7490968884282
:10AE200006DD99488068A0490968401AA24908606F
:10AE3000984880689F490968401A40F24C4188420E
:10AE400012DD012099490880924880689949096873
:10AE5000401A9A490968884206DD8E4880689549FB
:10AE60000968401A95490860874880688E490968D2
:10AE7000401A00E0ECE040F2EE21884227DD8E48E7
:10AE80000068FBF7BCFC41EC1A0B9FED8D0B53ECFB
:10AE9000102BFBF7D3FB41EC180B7B498968814AE7
:10AEA0001268501AFBF7ABFC41EC190B53EC182B52
:10AEB000FBF726FD12D27448806873494968441A2A
:10AEC000002C01DB204600E06042642806DA002006
:10AED0007349088040F24C40774908606D488068AB
:10AEE00074490968401A40F2EE21884227DD734810
:10AEF0000068FBF784FC41EC1A0B9FED710B53ECDF
:10AF0000102BFBF79BFB41EC180B62498968684AE0
:10AF10001268501AFBF773FC41EC190B53EC182B19
:10AF2000FBF7EEFC12D25B4880685A494968441A24
:10AF3000002C01DB204600E06042642806DA002095
:10AF40005A49088040F24C405C4908605648006805
:10AF500010B90020524908805648006810B90020F6
:10AF6000524908805848008838BB5848B0F900005A
:10AF7000B0F5967F05DA55480088401C00B2534969
:10AF8000088000205249088045480088012803D0E5
:10AF90004648008801280AD14C48B0F9000008282A
:10AFA00005DB4FF0010A01204749088062E04FF0BD
:10AFB000000A0020444908805CE04FF0000A444841
:10AFC000B0F90000B0F5967F05DA41480088401CD2
:10AFD00000B23F49088000203C4908803C4BB3F94F
:10AFE0000030062B30DB2E4B1B886BBB2B4BB3F991
:10AFF0000030A3F5FA62002A01DB134600E0534259
:10B00000B3F5967F19DC254BB3F90230A3F5FA614D
:10B01000002901DB0B4600E04B42B3F5967F0CDCC8
:10B020001E4BB3F90430A3F5FA60002801DB034698
:10B0300000E04342B3F5967F06DD1C4B1B881BB92D
:10B0400000202149088015E001201F49088011E0F7
:10B050004FF0000A0C488068134908600A4880686D
:10B06000104908600B4880681249086009488068E8
:10B070000F4908600AF0FF0006B0BDEC068BBDE882
:10B08000F08700004C4A00205C920020584A0020C3
:10B090004D4A002068920020544A00205C4A00205B
:10B0A000364A0020404A00203C4A0020384A00200E
:10B0B000484A0020444A0020644A0020684A002090
:10B0C0009A9999999999D93F524A0020504A00205B
:10B0D0004E4A0020FEB54FF4827014F085FD002822
:10B0E00037D04FF4827014F089FD6C4890F82E0030
:10B0F00018B16A4890F82F0058B300208DF800006E
:10B1000066484068019065480189ADF80810C0683C
:10B1100018B900206149087412E06048008B5F494B
:10B1200048830846C06848600846008B08810020B4
:10B13000C860084690F82E0010B9002014F080FD79
:10B1400056480168684688470020544981F82F0016
:10B1500000BF524890F82E00002852D04FF4807063
:10B1600014F042FD00284CD04FF4807014F046FDDE
:10B170004A48408B494991F82D10884216DD4748CE
:10B18000408B464991F82D10401A444948830A469D
:10B1900012890B465B8BD21A0B465B6803EB4200AD
:10B1A0000A4692F82D1014F00BFD23E03B48408B2B
:10B1B0003A4991F82D1088420FD13848C06860B1E3
:10B1C0000120364981F82F00002048830A4692F872
:10B1D0002D10D06814F0F4FC0CE03048408B2F495F
:10B1E00091F82D10884205D101202C4981F82F00BB
:10B1F000002048834FF4827014F000FD042014F006
:10B200001FFD4FF4887014F0EFFC70B14FF488709C
:10B2100014F0F4FC00202149087402208DF800008D
:10B22000084601686846884700BF4FF48A7014F0EA
:10B23000DBFC38B14FF48A7014F0E0FC00201749B1
:10B2400008742AE01548456924E0B5FA85F64FF000
:10B250000040F0408543B00000F58C74204614F0A7
:10B26000C3FCB8B1204614F0C9FC01208DF80000E1
:10B27000A4F58C70C0F3C7008DF80400A4F58C70A1
:10B28000012121EA90018DF8051004480168684603
:10B29000884700BF002DD8D100BFFEBD7C930020A1
:10B2A0000246002106E00548405C904201D10020A2
:10B2B0007047491C0029F6D00220F9E768680400AD
:10B2C00070B505460C462846FFF7EAFF061E01D07A
:10B2D000304670BD012C04D10121284614F052F9EA
:10B2E00004E01CB90021284614F04CF90020F0E7D6
:10B2F00010B5002409E00D49085D0121FFF7E0FFCA
:10B300000A49085D13F0D9FF641C002CF3D00848EB
:10B3100013F005FF032013F0D0FF042013F0CDFF3E
:10B32000052013F0CAFF002010BD0000686804006B
:10B33000386804007FB50025174B0FCB8DE80F0050
:10B3400003208DF8020004208DF8010005208DF8FF
:10B35000000000208DF80C004FF000400290062005
:10B360008DF8040000230D4A69460D4813F07AFE5B
:10B37000064606B16D1E002404E00A49085D13F07C
:10B38000B4FF641C002CF8D0681C20B9064A07A141
:10B390000020FFF7CFFA7FBD6C680400D15D040088
:10B3A0003868040068680400F13303007370693082
:10B3B0005F696E6974000000F8B506460F461446D2
:10B3C0001D462346002239463046009500F04EF8CF
:10B3D000F8BDF8B506460F4614461D462346012221
:10B3E00039463046009500F041F8F8BD2DE9F84F98
:10B3F00005460E4617469846DDF8289042F2107A28
:10B400002846FFF74DFF041E02D02046BDE8F88F06
:10B4100000212846FFF754FF0020124908704346D8
:10B420003A4631461048CDF8009013F05FFE0446CE
:10B430000CB10120EAE70AE0BAF10000AAF1010A22
:10B4400005D101212846FFF73BFF0120DEE7054833
:10B4500000780028F0D001212846FFF731FF0020B6
:10B46000D4E700007E410020386804002DE9FC4745
:10B4700081460D4690461E460A9C4846FFF710FF3F
:10B48000071E02D03846BDE8FC87812C01D9032075
:10B49000F9E7B8F1000F16D145F080000190601C6B
:10B4A000C0B2144B012201A900904846FFF79EFF4D
:10B4B00007460FB13846E6E722460E49491C30469A
:10B4C000FAF7CFFF13E00B48057022463146401CC7
:10B4D000FAF7C7FF00200090601CC2B200230549A4
:10B4E0004846FFF783FF07460FB13846CBE70020F9
:10B4F000C9E70000147A002010B50249024810F094
:10B50000F9FA10BDC49300200030004010B5034983
:10B510004FF0402010F0EEFA10BD0000E89300203C
:10B5200010B50249024810F0E5FA10BD0C94002055
:10B530000030024070B50A4813F0B1FC044600BF69
:10B54000254635B100BF07A262212846FAF762FE00
:10B5500000BF00BF0CB1062070BD0020FCE700005A
:10B56000688000202E2E5C2E2E5C2E2E5C626C6578
:10B570005F6366675C686F73742E630010B513F0C9
:10B58000B6FC10BD10B514F07BFC10BD014948712C
:10B59000704700001441002030B5034D28706970D9
:10B5A000AA70EB7030BD0000144100200149887280
:10B5B00070470000144100200149088170470000D5
:10B5C0001441002070B504460D46164633462A46FF
:10B5D0002146024814F0EEFE70BD00000C41002030
:10B5E00001480078704700001142002010B5002487
:10B5F0000BE0084850F8240028B1064850F8241001
:10B600004FF47A708847601CC4B2034800788442C3
:10B61000EFDB10BD204B0020D43D0020024600216E
:10B6200017E00E4850F82100904202D14FF0FF3051
:10B6300070470A4850F8210048B909480078401C72
:10B64000074B1870054840F821200020F0E7481CFF
:10B65000C1B20529E5DB6FF00100E9E7204B0020CE
:10B66000D43D002002460020002100BF27E0411CFD
:10B6700022E000EBC0030B4402EB8303D3ED000A8E
:10B6800001EBC103034402EB830393ED001A70EE58
:10B69000810AB6EE001A20EE810A00EBC0030B44CB
:10B6A00002EB830383ED000A01EBC103034402EBC9
:10B6B000830383ED000A491C0929DADB401C0928B1
:10B6C000D5DB704790ED031AD0ED061A01EE801A13
:10B6D00080ED031A90ED041AD0ED071A01EE801ADE
:10B6E00080ED041A90ED051AD0ED081A01EE801ACB
:10B6F00080ED051A90ED0C1AD0ED0F1A01EE801AAC
:10B7000080ED0C1A90ED0D1AD0ED101A01EE801A92
:10B7100080ED0D1A90ED0E1AD0ED111A01EE801A7F
:10B7200080ED0E1A90ED151AD0ED181A01EE801A60
:10B7300080ED151A90ED161AD0ED191A01EE801A47
:10B7400080ED161A90ED171AD0ED1A1A01EE801A34
:10B7500080ED171A90ED1B1AD0ED361A01EE801A03
:10B7600080ED1B1A90ED1C1AD0ED371A01EE801AED
:10B7700080ED1C1A90ED1D1AD0ED381A01EE801ADA
:10B7800080ED1D1A90ED241AD0ED3F1A01EE801ABB
:10B7900080ED241A90ED251AD0ED401A01EE801AA2
:10B7A00080ED251A90ED261AD0ED411A01EE801A8F
:10B7B00080ED261A90ED2D1AD0ED481A01EE801A70
:10B7C00080ED2D1A90ED2E1AD0ED491A01EE801A57
:10B7D00080ED2E1A90ED2F1AD0ED4A1A01EE801A44
:10B7E00080ED2F1A90ED1E1AD0ED391A01EE801A55
:10B7F000D0ED211A90ED3C2A42EE001A00EE211AFB
:10B8000080ED1E1A90ED1F1AD0ED3A1A01EE801A43
:10B81000D0ED221A90ED3D2A42EE001A00EE211AD8
:10B8200080ED1F1A90ED201AD0ED3B1A01EE801A20
:10B83000D0ED231A90ED3E2A42EE001A00EE211AB6
:10B8400080ED201A90ED271AD0ED421A01EE801AF1
:10B85000D0ED2A1A90ED452A42EE001A00EE211A88
:10B8600080ED271A90ED281AD0ED431A01EE801AC8
:10B87000D0ED2B1A90ED462A42EE001A00EE211A66
:10B8800080ED281A90ED291AD0ED441A01EE801AA5
:10B89000D0ED2C1A90ED472A42EE001A00EE211A44
:10B8A00080ED291A90ED301AD0ED4B1A01EE801A76
:10B8B000D0ED331A90ED4E2A42EE001A00EE211A16
:10B8C00080ED301A90ED311AD0ED4C1A01EE801A4D
:10B8D000D0ED341A90ED4F2A42EE001A00EE211AF4
:10B8E00080ED311A90ED321AD0ED4D1A01EE801A2A
:10B8F000D0ED351A90ED502A42EE001A00EE211AD2
:10B9000080ED321A90ED211AD0ED3C1A01EE801A2A
:10B91000D1ED021A61EE801A90ED1C2A01EE821A16
:10B92000D1ED011A61EE801A90ED1D2A01EEC21AC6
:10B9300080ED211A90ED221AD0ED3D1A01EE801A09
:10B94000D1ED021A61EE801A90ED1B2A01EEC21AA7
:10B95000D1ED001A61EE801A90ED1D2A01EE821AD7
:10B9600080ED221A90ED231AD0ED3E1A01EE801AD6
:10B97000D1ED011A61EE801A90ED1B2A01EE821AB8
:10B98000D1ED001A61EE801A90ED1C2A01EEC21A68
:10B9900080ED231A90ED2A1AD0ED451A01EE801A97
:10B9A000D1ED021A61EE801A90ED252A01EE821A7D
:10B9B000D1ED011A61EE801A90ED262A01EEC21A2D
:10B9C00080ED2A1A90ED2B1AD0ED461A01EE801A5E
:10B9D000D1ED021A61EE801A90ED242A01EEC21A0E
:10B9E000D1ED001A61EE801A90ED262A01EE821A3E
:10B9F00080ED2B1A90ED2C1AD0ED471A01EE801A2B
:10BA0000D1ED011A61EE801A90ED242A01EE821A1E
:10BA1000D1ED001A61EE801A90ED252A01EEC21ACE
:10BA200080ED2C1A90ED331AD0ED4E1A01EE801AEB
:10BA3000D1ED021A61EE801A90ED2E2A01EE821AE3
:10BA4000D1ED011A61EE801A90ED2F2A01EEC21A93
:10BA500080ED331A90ED341AD0ED4F1A01EE801AB2
:10BA6000D1ED021A61EE801A90ED2D2A01EEC21A74
:10BA7000D1ED001A61EE801A90ED2F2A01EE821AA4
:10BA800080ED341A90ED351AD0ED501A01EE801A7F
:10BA9000D1ED011A61EE801A90ED2D2A01EE821A85
:10BAA000D1ED001A61EE801A90ED2E2A01EEC21A35
:10BAB00080ED351A90ED091AD1ED021A61EE211AC6
:10BAC00090ED361A01EE801AD0ED121A91ED012A8E
:10BAD00061EE821A01EEC01A80ED361A90ED0A1A54
:10BAE000D1ED021A61EE211A90ED371A01EE801A9B
:10BAF000D0ED131A91ED012A61EE821A01EEC01AFF
:10BB000080ED371A90ED0B1AD1ED021A61EE211A71
:10BB100090ED381A01EE801AD0ED141A91ED012A39
:10BB200061EE821A01EEC01A80ED381A90ED001A0B
:10BB3000D1ED021A61EE211A90ED3F1A01EEC01A02
:10BB4000D0ED121A91ED002A61EE821A01EE801AF0
:10BB500080ED3F1A90ED011AD1ED021A61EE211A23
:10BB600090ED401A01EEC01AD0ED131A91ED002AA3
:10BB700061EE821A01EE801A80ED401A90ED021AF1
:10BB8000D1ED021A61EE211A90ED411A01EEC01AB0
:10BB9000D0ED141A91ED002A61EE821A01EE801A9E
:10BBA00080ED411A90ED001AD1ED011A61EE211AD3
:10BBB00090ED481A01EE801AD0ED091A91ED002A95
:10BBC00061EE821A01EEC01A80ED481A90ED011A5A
:10BBD000D1ED011A61EE211A90ED491A01EE801A99
:10BBE000D0ED0A1A91ED002A61EE821A01EEC01A18
:10BBF00080ED491A90ED021AD1ED011A61EE211A79
:10BC000090ED4A1A01EE801AD0ED0B1A91ED002A40
:10BC100061EE821A01EEC01A80ED4A1A90ED391ACF
:10BC2000D0ED3C1A00EE211AD0ED0C1A91ED022A4B
:10BC300061EE821A01EE801AD0ED151A91ED012AFB
:10BC400061EE821A01EEC01A80ED391A90ED3A1AAF
:10BC5000D0ED3D1A00EE211AD0ED0D1A91ED022A19
:10BC600061EE821A01EE801AD0ED161A91ED012ACA
:10BC700061EE821A01EEC01A80ED3A1A90ED3B1A7D
:10BC8000D0ED3E1A00EE211AD0ED0E1A91ED022AE7
:10BC900061EE821A01EE801AD0ED171A91ED012A99
:10BCA00061EE821A01EEC01A80ED3B1A90ED421A45
:10BCB000D0ED451A00EE211AD0ED031A91ED022ABB
:10BCC00061EE821A01EEC01AD0ED151A91ED002A2C
:10BCD00061EE821A01EE801A80ED421A90ED431A4D
:10BCE000D0ED461A00EE211AD0ED041A91ED022A89
:10BCF00061EE821A01EEC01AD0ED161A91ED002AFB
:10BD000061EE821A01EE801A80ED431A90ED441A1A
:10BD1000D0ED471A00EE211AD0ED051A91ED022A56
:10BD200061EE821A01EEC01AD0ED171A91ED002AC9
:10BD300061EE821A01EE801A80ED441A90ED4B1AE2
:10BD4000D0ED4E1A00EE211AD0ED031A91ED012A22
:10BD500061EE821A01EE801AD0ED0C1A91ED002AE4
:10BD600061EE821A01EEC01A80ED4B1A90ED4C1A6A
:10BD7000D0ED4F1A00EE211AD0ED041A91ED012AF0
:10BD800061EE821A01EE801AD0ED0D1A91ED002AB3
:10BD900061EE821A01EEC01A80ED4C1A90ED4D1A38
:10BDA000D0ED501A00EE211AD0ED051A91ED012ABE
:10BDB00061EE821A01EE801AD0ED0E1A91ED002A82
:10BDC00061EE821A01EEC01A80ED4D1A90ED0F1A45
:10BDD000D1ED021A61EE211A90ED3C1A01EE801AA3
:10BDE000D0ED181A91ED012A61EE821A01EEC01A07
:10BDF000D1ED021A61EE801A90ED372A01EE821A17
:10BE0000D1ED011A61EE801A90ED382A01EEC21AC6
:10BE100080ED3C1A90ED101AD1ED021A61EE211A54
:10BE200090ED3D1A01EE801AD0ED191A91ED012A1C
:10BE300061EE821A01EEC01AD1ED021A61EE801A8B
:10BE400090ED362A01EEC21AD1ED001A61EE801A89
:10BE500090ED382A01EE821A80ED3D1A90ED111A0C
:10BE6000D1ED021A61EE211A90ED3E1A01EE801A10
:10BE7000D0ED1A1A91ED012A61EE821A01EEC01A74
:10BE8000D1ED011A61EE801A90ED362A01EE821A88
:10BE9000D1ED001A61EE801A90ED372A01EEC21A38
:10BEA00080ED3E1A90ED061AD1ED021A61EE211ACC
:10BEB00090ED451A01EEC01AD0ED181A91ED002A46
:10BEC00061EE821A01EE801AD1ED021A61EE801A3B
:10BED00090ED402A01EE821AD1ED011A61EE801A2E
:10BEE00090ED412A01EEC21A80ED451A90ED071A35
:10BEF000D1ED021A61EE211A90ED461A01EEC01A38
:10BF0000D0ED191A91ED002A61EE821A01EE801A25
:10BF1000D1ED021A61EE801A90ED3F2A01EEC21AAD
:10BF2000D1ED001A61EE801A90ED412A01EE821ADD
:10BF300080ED461A90ED081AD1ED021A61EE211A31
:10BF400090ED471A01EEC01AD0ED1A1A91ED002AB1
:10BF500061EE821A01EE801AD1ED011A61EE801AAB
:10BF600090ED3F2A01EE821AD1ED001A61EE801A9F
:10BF700090ED402A01EEC21A80ED471A90ED061AA4
:10BF8000D1ED011A61EE211A90ED4E1A01EE801AE0
:10BF9000D0ED0F1A91ED002A61EE821A01EEC01A5F
:10BFA000D1ED021A61EE801A90ED492A01EE821A53
:10BFB000D1ED011A61EE801A90ED4A2A01EEC21A03
:10BFC00080ED4E1A90ED071AD1ED011A61EE211A9B
:10BFD00090ED4F1A01EE801AD0ED101A91ED002A63
:10BFE00061EE821A01EEC01AD1ED021A61EE801ADA
:10BFF00090ED482A01EEC21AD1ED001A61EE801AC6
:10C0000090ED4A2A01EE821A80ED4F1A90ED081A3F
:10C01000D1ED011A61EE211A90ED501A01EE801A4D
:10C02000D0ED111A91ED002A61EE821A01EEC01ACC
:10C03000D1ED011A61EE801A90ED482A01EE821AC4
:10C04000D1ED001A61EE801A90ED492A01EEC21A74
:10C0500080ED501A90ED011AD1ED021A61EE211A0D
:10C0600090ED061A01EE801AD0ED021A91ED012A28
:10C0700061EE821A01EEC01A80ED061A90ED001AE8
:10C08000D1ED021A61EE211A90ED071A01EEC01AE5
:10C09000D0ED021A91ED002A61EE821A01EE801AAB
:10C0A00080ED071A90ED001AD1ED011A61EE211A08
:10C0B00090ED081A01EE801AD0ED011A91ED002AD8
:10C0C00061EE821A01EEC01A80ED081A90ED0A1A8C
:10C0D000D1ED021A61EE211A90ED0F1A01EE801ACD
:10C0E000D0ED0B1A91ED012A61EE821A01EEC01A11
:10C0F00080ED0F1A90ED091AD1ED021A61EE211AA6
:10C1000090ED101A01EEC01AD0ED0B1A91ED002A35
:10C1100061EE821A01EE801A80ED101A90ED091A74
:10C12000D1ED011A61EE211A90ED111A01EE801A7B
:10C13000D0ED0A1A91ED002A61EE821A01EEC01AC2
:10C1400080ED111A90ED131AD1ED021A61EE211A49
:10C1500090ED181A01EE801AD0ED141A91ED012A13
:10C1600061EE821A01EEC01A80ED181A90ED121AD3
:10C17000D1ED021A61EE211A90ED191A01EEC01AE2
:10C18000D0ED141A91ED002A61EE821A01EE801AA8
:10C1900080ED191A90ED121AD1ED011A61EE211AF3
:10C1A00090ED1A1A01EE801AD0ED131A91ED002AC3
:10C1B00061EE821A01EEC01A80ED1A1A9FED191A6B
:10C1C00020EE011A61EE000A002210E002EBC20329
:10C1D000134400EB830393ED001A31EE201A02EBB7
:10C1E000C203134400EB830383ED001A521C032A9D
:10C1F000ECDB062212E002EBC203134400EB8303E4
:10C2000093ED001ADFED081A00EEA11A02EBC2034B
:10C21000134400EB830383ED001A521C092AEADB66
:10C220007047000017B7D1380000C84201480249E2
:10C23000086070470090D003184B002010B512F032
:10C240000FF828B195480088C0F30420944908608D
:10C2500012F05EF810B193489349486712F094F8D1
:10C2600030B18E48E0380068C0F342308F49086032
:10C2700012F0B6F828B18E48006820F080708C4922
:10C28000086012F0CBF848B100208A4908604FF0EE
:10C290008041C1F810018549091F086012F0EAF8D1
:10C2A00018B1032081496431086012F001F968B1C6
:10C2B00005208149086001207F497831086000200D
:10C2C0007D49083108603F20091F086012F00EF90F
:10C2D000002855D07148E0300068784908606F4800
:10C2E000E4300068091D08606C48E8300068091DEA
:10C2F00008606A48EC300068091D08606748F03043
:10C300000068091D08606548F4300068091D086070
:10C310006248F83000686949203108605F48FC30A5
:10C320000068091D086066480068091D08606448C7
:10C33000001D0068091D0860614808300068091D7B
:10C3400008605F480C300068091D08605C481030C8
:10C3500000685A4940310860594814300068091D86
:10C360000860574818300068091D086054481C30A0
:10C370000068091D0860524820300068091D0860E7
:10C3800011F042FF30B14548CC38006800F04F0052
:10C390004C49086011F090FF40B14B48006800F034
:10C3A000010018B16FF001004749086011F0CEFF9D
:10C3B00028B14648006840F48060444908603C4821
:10C3C0007438006840F4700039497439086000BF5F
:10C3D00000BF00BFBFF34F8F00BF00BF00BF00BF53
:10C3E00000BF00BFBFF36F8F00BF00BF00BF384862
:10C3F000006800F00100F0B101203649086000BF7C
:10C40000354800680028FBD03148006820F0010062
:10C410004FF01021C1F80C0200BF2F48006800281F
:10C42000FBD000202B49086000BF2B480068002883
:10C43000FBD000F071FB26480C38006800F000408B
:10C4400028B923480838006800F0004018B30120DC
:10C450002049086000BF204800680028FBD0152054
:10C460001B490C39086000BF1B4800680028FBD03E
:10C47000152117480838016000BF174800680028D8
:10C48000FBD000201349086000BF13480068002853
:10C49000FBD000F041FBFFF7C9FE10BD24030010E4
:10C4A000403501400DF0ADBA00C007403C050040EA
:10C4B000FCED00E00C0100401056004020C500409B
:10C4C00024040010E40E0040000400403C1700402B
:10C4D0000C12001004E5014000E40140014800682E
:10C4E00070470000084100207CB500251B4903C9A6
:10C4F000CDE9000102208DF802000020ADF8000017
:10C50000174A6946174814F03FF8044604B16D1EF7
:10C51000012321220021134813F0C2FF044664B115
:10C520000123212200210F4813F0BAFF044624B151
:10C530000D4A0EA10020FEF7FDF90A4814F008F894
:10C54000084814F011F80C4800F03EFA681C20B9B5
:10C550000A4A0BA10020FEF7EDF97CBD106804002B
:10C56000593A040008680400913303007274635F51
:10C57000636F6E666967000031480300C1330300D2
:10C580007274635F696E69740000000002460021E6
:10C5900012E00C4850F82100904202D16FF00100E7
:10C5A0007047084850F8210020B9064840F821207B
:10C5B0000020F5E7481CC1B20A29EADB4FF0FF3042
:10C5C000EEE700006479002010B503460021002248
:10C5D00014E00D4850F8220098420DD1114607E0B2
:10C5E000094C481C54F8200044F82100481CC1B2F2
:10C5F0000929F5DB002010BD501CC2B20A2AE8DB75
:10C600004FF0FF30F7E700006479002010B5FFF726
:10C610006BFF0BF027FE06F0A9FA0DF081FDFAF78B
:10C620002FFDFAF7EBFE0DF05DFF0DF07FFE0DF034
:10C63000F3FD03F03BFD03F00BF804F099F804F070
:10C64000EBFA02F007FF04F04DFD03F0CBFE04F01F
:10C650004FF904F065F903F06BFC04F0BFFE03F042
:10C66000AFFC04F079FC02F0F1FB04F0B5F804F043
:10C67000F3FA19F033FF0BF01DFD10BD10B5FEF7F6
:10C68000C1F850B9FEF7B2FF0EF0CCF8044617F02F
:10C6900037F90349086000F07DF9FBF7E1FC10BDB4
:10C6A000D03D0020B0EE401A81EE200ADFED021AE4
:10C6B00020EE210A704700000000C84210B52DEDA1
:10C6C000048BB0EE408A9FED260AB0EE409A9FEDB3
:10C6D000240AF0EE408A2348006890F8230060B1F5
:10C6E000B2EE040AC8EE000A1E480068C0ED000A57
:10C6F00000201C49096881F82300B2EE040AC8EE44
:10C70000000AF0EE609A17480068DFED170AB0EEF5
:10C71000690A0BF0DFFCF0EE408A9FED140AF4EE9C
:10C72000C08AF1EE10FA04D29FED0D0AB0EE409AE5
:10C7300011E09FED0F0AF4EEC08AF1EE10FA04DD6D
:10C740009FED0C0AB0EE409A05E0B0EE680A0EF0DC
:10C7500095FDB0EE409AB0EE490ABDEC048B10BDD9
:10C76000000000009C4000200AD7233C0000A043AA
:10C770000000D2430000C84208B500BF4FF48070EB
:10C780000B49405808B1012000E0002078B1094869
:10C790000068804700BF00204FF48071044A885031
:10C7A000084611464058009000BF00BF00BF08BDBA
:10C7B00000000140CC4A00202DE9F0410246C2F3BE
:10C7C0000744C2F30726D5B2802300200021CCE025
:10C7D000880006EA0307D7B1664F3F88DFF898C1A3
:10C7E0002CF81070634FB7F802C0DFF88C81471C3B
:10C7F00028F817C05F4FB7F804C0871C28F817C087
:10C800005C4FB7F806C0C71C28F817C019E05B4F8B
:10C810003F88DFF864C12CF81070584FB7F802C099
:10C82000DFF85481471C28F817C0544FB7F804C0EC
:10C83000871C28F817C0514FB7F806C0C71C28F846
:10C8400017C0880004EA030717B34A4FB7F800C0BF
:10C85000494F403727F810C0464FB7F80280464F7F
:10C86000403700F1010C27F81C80424FB7F80480D4
:10C87000414F403700F1020C27F81C803D4FB7F8BC
:10C8800006803D4F403700F1030C27F81C8021E063
:10C890003A4FB7F800C0384F403727F810C0374F2D
:10C8A000B7F80280344F403700F1010C27F81C80A4
:10C8B000324FB7F80480304F403700F1020C27F8B0
:10C8C0001C802E4FB7F806802B4F403700F1030C29
:10C8D00027F81C80880005EA030717B3254FB7F82F
:10C8E00000C0254F803727F810C0224FB7F80280CC
:10C8F000214F803700F1010C27F81C801D4FB7F83D
:10C9000004801D4F803700F1020C27F81C80194F5E
:10C91000B7F80680184F803700F1030C27F81C8009
:10C9200021E0164FB7F800C0134F803727F810C02A
:10C93000124FB7F80280104F803700F1010C27F832
:10C940001C800E4FB7F804800B4F803700F1020CAB
:10C9500027F81C80094FB7F80680074F803700F191
:10C96000030C27F81C805B08491C0829FFF630AF30
:10C97000BDE8F081F86704009C71002000680400A5
:10C9800010B50122042102480068FEF71BFE10BD0D
:10C99000BC40002010B500240BE0084850F82400EB
:10C9A00028B1064850F82410054800688847601CE4
:10C9B000C4B2044800788442EFDB10BD344B002041
:10C9C000D03D0020D53D00200246002117E00E4852
:10C9D00050F82100904202D14FF0FF3070470A48D2
:10C9E00050F8210048B909480078401C074B1870DE
:10C9F000054840F821200020F0E7481CC1B2062974
:10CA0000E5DB6FF00100E9E7344B0020D53D002065
:10CA100010B50BF04FFB10BD0FB4084B10B504A9B7
:10CA200002AA039801F0C8FC044602A9002002F003
:10CA30005AF8204610BC5DF814FB0000E7EA02003B
:10CA400003B401984100009850EAC12018BF0420A7
:10CA50004A0D18BF40F0010040F2FF72B2EB515F87
:10CA600008BF40F00200012808BF052002B070474F
:10CA70004100080218BF04200A0E18BF40F0010050
:10CA80004FF07F4232EA010108BF40F00200012866
:10CA900008BF05207047000000BF00BF00BFBFF304
:10CAA0004F8F00BF00BF00BF0948006800F4E0607E
:10CAB00008490843001D0649086000BF00BF00BFC9
:10CAC000BFF34F8F00BF00BF00BF00BF00BFFDE737
:10CAD0000CED00E00000FA0500BF00BF00BFBFF38F
:10CAE0004F8F00BF00BF00BF0948006800F4E0603E
:10CAF00008490843001D0649086000BF00BF00BF89
:10CB0000BFF34F8F00BF00BF00BF00BF00BFFDE7F6
:10CB10000CED00E00000FA0500BF00BF00BFBFF34E
:10CB20004F8F00BF00BF00BF0948006800F4E060FD
:10CB300008490843001D0649086000BF00BF00BF48
:10CB4000BFF34F8F00BF00BF00BF00BF00BFFDE7B6
:10CB50000CED00E00000FA0570B5C1482DED020BA8
:10CB60002DED0E8B82B0119D25F000449FEDBEDBB4
:10CB70009FEDBFEB84423EDBA4F140511098A1F140
:10CB80007F6108430FD0BC48844202DC28D1109852
:10CB900030B39DED100B02B0BDEC0E8B02B0BDE8C2
:10CBA000704001F0C5BA9DED100B53EC1D2B51ECFC
:10CBB000100BF9F743FD9DED100B41EC180B53ECF6
:10CBC0001E2B51EC100BF9F739FD53EC182BF9F72C
:10CBD0008EFC41EC100B02B0BDEC0E8B02B070BDB0
:10CBE000012001F021FB02B0BDEC0E8B02B0BDE8CC
:10CBF000704001F0B1BAA1489FEDA18B844256DA92
:10CC00009DED100BB4F1795F0ADA51EC100BFFF7D0
:10CC100017FF042808BF01F0AFFA9DED100BDAE70B
:10CC200053EC102B51EC100BF9F708FD41EC190BEC
:10CC300095480621B0EE490AF0EE690A784401F001
:10CC400063F953EC192B51EC100BF9F7F7FC41EC9D
:10CC50001A0B8E48B0EE490AF0EE690A04217844B6
:10CC600001F052F953EC192B51EC100BF9F7E6FCDB
:10CC700053EC182BF9F73BFC41EC100B51EC1A0B61
:10CC800053EC102BF9F74CFDCDE900019DED000BA5
:10CC900053EC102B9DED100B51EC100BF9F7CEFC63
:10CCA0009DED101B53EC112BF9F721FCD2E09DED0B
:10CCB000100B51EC100B0BF06FF953EC182BF9F72C
:10CCC000BAFC9FED730BCDE9000153EC102B9DEDE9
:10CCD000000B51EC100BF9F7B1FC41EC190B6E484D
:10CCE0000621B0EE490AF0EE690A784401F00CF929
:10CCF00053EC192B51EC100BF9F7A0FC41EC1B0B7A
:10CD00006648B0EE490AF0EE690A0421784401F061
:10CD1000FBF853EC192B51EC100BF9F78FFC53EC8B
:10CD2000182BF9F7E4FB41EC1C0B51EC190B19F033
:10CD3000FDF841EC180B5A489FED5BABA04222DC9A
:10CD400053EC1C2B51EC1B0BF9F7EAFCCDE900016D
:10CD50009DED000B51EC180B53EC102BF9F76EFC0A
:10CD600053EC182BF9F7C3FB53EC1A2BF9F766FCBD
:10CD700053EC1D2BF9F75CFC53EC1E2BF9F75BFC15
:10CD800041EC100B5FE08DED008B002000909DEDDD
:10CD9000000B51EC180B53EC102BF9F7A8FB9DED91
:10CDA000000B41EC1E0B53EC102B51EC100BF9F760
:10CDB00045FC53EC192BF9F73EFC53EC1E2BF9F70D
:10CDC000AFFC41EC190B53EC1C2B51EC1B0BF9F78E
:10CDD000A7FC41EC1B0B53EC1A2B51EC190BF9F788
:10CDE0002DFC53EC1D2BF9F726FC41EC190B53ECF1
:10CDF0001A2B51EC180BF9F721FC53EC1B2BF9F70C
:10CE00001DFC53EC192BF9F713FC9DED000B41ECC5
:10CE1000180B53EC1A2B51EC100BF9F70FFC9FED8C
:10CE2000249B53EC192BF9F706FC41EC100B51EC49
:10CE3000180B53EC102BF9F7FBFB53EC192BF9F7FC
:10CE4000FAFB41EC100B002D3FF7C5AE51EC100B77
:10CE500081F0004141EC100BBDE600000000000035
:10CE60000000F03F00000000075C143326A6913C50
:10CE7000182D4454FB21F93F0000F07F0000E03FF3
:10CE8000000000000000F03F889F0100969F010015
:10CE9000000000000000E03FDA9E0100E89E010073
:10CEA0003333EF3F000000000000000000000040AE
:10CEB000182D4454FB21E93F10B54FF00E402DEDE5
:10CEC000028BB0EE408A18EE104A00EB4400B0F13D
:10CED000506F4AD84FF0FC40B0EB440F22D2B0EE76
:10CEE000C80AF7EE000A30EEC00AF6EE000A60EE5D
:10CEF000208A18EE900A19F050F801EE100A14F08A
:10CF0000004F1DBFDFED2D0A9FED2D0AB1EE411A36
:10CF1000DFED2C0A08BF9FED2C0AF8EE001A21EE77
:10CF2000218A05E0DFED290A68EE088AB0EE600A82
:10CF30009FED271ADFED271A30EE080A48EE811A16
:10CF40009FED251A08EEA11ADFED241A48EE811A8A
:10CF50009FED231A08EEA11A68EE281ABDEC028B89
:10CF600001EE810A30EE200A10BD4FF0E440B0EB34
:10CF7000440F0CD918EE100AFFF77AFD042808BFF9
:10CF800001F018F9B0EE480ABDEC028B10BD4FF06D
:10CF90007F40B0EB440F07D2B0EE480ABDEC028BE5
:10CFA000BDE8104001F0F8B8012001F03DF9BDECFA
:10CFB000028BBDE8104001F0F5B800000000C9BFC9
:10CFC00022AAFDB90000C93F22AAFD3900000000D5
:10CFD00024FE1C3DC78AD83C1E67383D1B93993DF3
:10CFE000AFAA2A3E0000000070B59B482DED020B51
:10CFF0002DED068B079D25F00044A04218DC9748D4
:10D00000844202DC0AD1069840B19DED060BBDECCE
:10D01000068B02B0BDE8704001F08AB8002DCCBF8D
:10D020009FED8F0B9FED900BBDEC068B02B070BD9A
:10D030008F48A04215DD8F48A042D8BF4FF0FF3483
:10D0400058DD9DED060B51EC100BFFF7F9FC0428A1
:10D0500008BF01F091F89DED060BBDEC068B02B008
:10D0600070BD9DED060B51EC100B0AF095FFCDE95C
:10D07000060181489FED828BA0423CDD8248A042A0
:10D080001FDD00249FED82AB9DED060B53EC1A2BA8
:10D0900051EC100BF9F72BFA9DED060B41EC190B37
:10D0A00053EC1A2B51EC100BF9F7C8FA53EC182B70
:10D0B000F9F7BEFA53EC192BF9F732FBCDE906016B
:10D0C00049E09DED060B012453EC182B51EC100B9D
:10D0D000F9F70DFA9DED060B41EC190B53EC182BEB
:10D0E00051EC100BF9F7A4FA53EC192BF9F718FBD4
:10D0F000CDE906012FE06848A0421FDD02249FED24
:10D10000689B9DED060B53EC192B51EC100BF9F7B6
:10D1100095FA53EC182BF9F7EAF99DED060B41EC63
:10D12000180B53EC192B51EC100BF9F781FA53EC57
:10D13000182BF9F7F5FACDE906010CE09DED060B89
:10D14000032453EC102B9FED580B51EC100BF9F707
:10D15000E7FACDE906019DED060B53EC102B51ECDF
:10D16000100BF9F76BFA41EC180B53EC182BF9F78D
:10D1700065FA41EC190B4E480621B0EE490AF0EE73
:10D18000690A784400F0C0FE53EC182B51EC100BE8
:10D19000F9F754FA41EC180B4648B0EE490AF0EEA4
:10D1A000690A0521784400F0AFFE53EC192B51ECCD
:10D1B000100BF9F743FA41EC100B51EC180B53EC40
:10D1C000102B002C0EDAF9F792F99DED061B53ECAB
:10D1D000112BF9F733FA9DED061B53EC112BF9F7E0
:10D1E0002AFA35E0F9F783F99DED061B53EC112B74
:10D1F000F9F724FA41EC100B2F48784400EBC400F7
:10D2000090ED001B51EC100B53EC112BF9F710FAB9
:10D210009DED061B53EC112BF9F70AFA41EC100BAC
:10D220002648784400EBC40090ED001B51EC100B35
:10D2300053EC112BF9F7FFF941EC100B002DA2BFB5
:10D24000BDEC068B02B070BD51EC100B81F00041BB
:10D2500041EC100B01E70000000010440000F07FDB
:10D26000182D4454FB21F93F182D4454FB21F9BFDC
:10D270000000DC3F0000203E0000F33F0000000003
:10D28000000000000000F03F0000E63F000000004A
:10D29000000000000000004000800340000000008B
:10D2A000000000000000F83F000000000000F0BF98
:10D2B000FA9A0100B09A01003A9A0100F29901002D
:10D2C00070B56B4E2DED040B2DED028B82B0DDF8A9
:10D2D0001CC0DDE905235C422CF000411C4341EAFF
:10D2E000D474049D22F00040B44205D86C422C4313
:10D2F00040EAD474B4420BD99DED061B9DED040B9E
:10D3000002B0BDEC028B04B0BDE8704000F01ABF63
:10D31000ACF14054A4F17F641C430BD0022404EA16
:10D32000AC7444EAD27405439FED538B9FED542BAC
:10D3300007D015E09DED040B51EC100B04F01DF926
:10D3400042E0002C11BF012C9DED040B02B0BDEC9E
:10D35000028B04BF04B070BD022C38D0032C3BD02C
:10D360000B439FED491B9FED4A0B0AD0B14218D1E8
:10D37000B04209D121F0804120F080400791059012
:10D380000FE0002A15DA10E0434B7B44002C08BF65
:10D3900093ED000B0DD0012C10D0022C17D0032CD4
:10D3A0001AD0B0421DD1002A03DAB0EE410AF0EEE5
:10D3B000610A02B0BDEC028B04B070BD93ED000BAE
:10D3C00051EC100B81F0004141EC100BF1E7B0EE95
:10D3D000480AF0EE680AECE7B0EE420AF0EE620AA4
:10D3E000E7E7401A00153C28C8BF8DED000B19DC9B
:10D3F000BCF1000FBEBF10F13C0F9FED290B8DED6E
:10D40000000B0FDB9DED060B53EC102B9DED040B79
:10D4100051EC100BF9F784F90AF0BEFD04F0ADF8F9
:10D42000CDE90001002C08BF9DED000BC1D0012CFF
:10D4300010D0022C9FED1C0B53EC102B9DED000B1C
:10D4400051EC100B0DD0F9F7F3F853EC182BF9F75A
:10D45000EFF8B9E7019880F0004001909DED000BD6
:10D46000A7E7F9F7E5F853EC182BF9F7E4F8ABE781
:10D470000000F07F00000000182D4454FB210940FB
:10D48000182D4454FB2109C0182D4454FB21F9BF29
:10D49000182D4454FB21F93F52990100000000006F
:10D4A0000000000000000000075C143326A6A13C29
:10D4B00010EE100A10B510EE901A4FF0684202EB11
:10D4C00040032DED028BB3F1654F3CBF02EB4102EF
:10D4D000B2F1654F7CD200BFC0F3C753C1F3C7524E
:10D4E0009A1A1B2A09DD10F0004F14BF9FED6E0A37
:10D4F0009FED6E0ABDEC028B10BD12F11A0F1BDA04
:10D5000011F0004F09D010F0004F0CBF9FED680ADA
:10D510009FED680ABDEC028B10BD80EE208A18EEEC
:10D52000100AFFF7A5FA042808BF00F043FEB0EE8A
:10D53000480ABDEC028B10BD4200B2EB410F37D957
:10D5400010F0004F19BFDFED5C1A9FED5C1ADFEDA4
:10D550005C1A9FED5C1AB0EE602A0A46F1EE400AB2
:10D5600080F00041B0EE420A10460A1A5200B2F1B1
:10D57000807F34D2484010F0004FDFED532A9FEDFA
:10D58000533A1DBFBEEE002A71EEE21A31EE431A85
:10D59000B6EE002A04BF71EEA21A31EE031AF0EEC5
:10D5A000402A42EE602A40EE020A82EEA02A18E0EB
:10D5B00011F0004F04BF9FED461AF0EE411AD4D08F
:10D5C00010F0004F1CBFDFED431A9FED431A00E03F
:10D5D00026E004BFDFED411A9FED411AC5E780EE5A
:10D5E000202A22EE020ADFED3F0ADFED3F2ABDECE2
:10D5F000028B40EE202ADFED3D0A40EE220ADFEDED
:10D600003C2A40EE202ADFED3B0A40EE220A22EEC1
:10D61000000A00EE201A31EE020A30EE210A10BD97
:10D620004FF07F42B2EB400F28BFB2EB410F05D263
:10D63000BDEC028BBDE8104000F0B1BD40EA010333
:10D640005B0008BF41F0FF410BD0B2EB400F08BFB9
:10D65000B2EB410F08D120F0804000EE100A21F01B
:10D66000804100EE901A37E7B2EB400F12BF5FEA3D
:10D67000410240F0FF4001F000413FF42DAF4A006D
:10D6800092EA40033FF528AF002AACBF9FED1A1A7B
:10D690009FED1A1A20EE010A60EE810A10EE100AC0
:10D6A00010EE901A18E70000DB0FC9BFDB0FC93F6F
:10D6B000DB0F4940DB0F49C00000C9BF22AAFDB9FA
:10D6C0000000C93F22AAFD390060ED3EC30ACE37F3
:10D6D00000000000000049C022AA7DBA00004940B5
:10D6E00022AA7D3A2DAD65BD8FB8D53D0FB511BECF
:10D6F00061C84C3EA8AAAABE0000804F0000802F3F
:10D7000010B52F499FED2C1B2DED020B84B0059811
:10D7100020F000408842D8BF9DED040B2DDD294943
:10D72000884209D1049840B94FF0010000F07CFD17
:10D7300000F012FD06B010BD05DB9DED040B00F0FE
:10D74000F7FC06B010BD68469DED040B00F008F92B
:10D7500010F0030004BF9DED021B9DED000B0CD0EB
:10D7600001280ED09DED021B9DED000B022817D065
:10D77000012000F045FC06B010BD00F00DFB06B026
:10D7800010BD9DED021B9DED000B012000F038FC4B
:10D7900051EC100B81F0004106B041EC100B10BDB4
:10D7A00000F0FAFA51EC100B81F0004106B041ECA8
:10D7B000100B10BD00000000000000000000000081
:10D7C000FB21E93F0000F07F2DED020B019820F0D6
:10D7D000004001909DED000B02B07047000000007A
:10D7E00010B52F499FED2C1B2DED020B84B0059831
:10D7F00020F000408842DCBF00209DED040B32DDAC
:10D800002849884209D1049840B94FF0010000F03E
:10D810000BFD00F0A1FC06B010BD05DB9DED040B77
:10D8200000F086FC06B010BD68469DED040B00F0CC
:10D8300097F810F0030011D0012818D09DED021BBD
:10D840009DED000B02281AD000F0A6FA51EC100B47
:10D8500081F0004106B041EC100B10BD9DED021BA4
:10D860009DED000B012000F0CBFB06B010BD9DED3F
:10D87000021B9DED000B00F08FFA06B010BD0120D9
:10D8800000F0BEFB51EC100B81F0004106B041EC02
:10D89000100B10BD000000000000000000000000A0
:10D8A000FB21E93F0000F07F00B52DED048BB0EEC9
:10D8B000409AF0EE609A83B051EC190BF9F72FF90A
:10D8C00041EC180B18EE100A18EE901A8DED008B33
:10D8D000002818BF0120084320F00040C0F17F60FD
:10D8E00000F1E040C00F14D019EE101A19EE900AA2
:10D8F0008DED009B002918BF0121084320F0004056
:10D90000C0F17F6000F1E040C00F04BF012000F0D3
:10D910008BFCB0EE480A03B0F0EE680ABDEC048B55
:10D9200000BD10B52DED028BB1EEC08A18EE100AC5
:10D9300020F00040C0F1FF40C00F0AD010EE100AE6
:10D9400020F00040C0F1FF40C00F04BF012000F0F4
:10D950006BFCB0EE480ABDEC028B10BD000000006D
:10D960002DE9F14F04462DED020B2DED088B8AB009
:10D970009FEDE70B80ED020B139EE74826F0004574
:10D9800085420ADC9DED120B002084ED000B0AB0ED
:10D99000BDEC088B03B0BDE8F08FE0489FEDE0AB35
:10D9A0009FEDE1BBA84247DDE14F9FEDE39B9FED7B
:10D9B000E48B9DED120B53EC1A2B51EC100B002E47
:10D9C0001CDDF8F735FE41EC100BBD4208D053ECDE
:10D9D0001B2B51EC100BF8F72BFEC4E900010BE0F8
:10D9E00053EC192B51EC100BF8F722FE53EC182BCB
:10D9F000F8F71EFEC4E900010120C8E7F8F777FD3B
:10DA000041EC100BBD4208D053EC1B2B51EC100B1A
:10DA1000F8F76DFDC4E900010BE053EC192B51EC54
:10DA2000100BF8F764FD53EC182BF8F760FDC4E910
:10DA300000014FF0FF30AAE7C348A84279DB9DED13
:10DA4000120B51EC100B0AF0A7FA41EC180B9FEDEA
:10DA5000C00B53EC102BF8F7F1FD9FEDBF1B53ECFF
:10DA6000112BF8F744FDF8F7E8FE0746F8F7C7FE74
:10DA700041EC190B53EC1A2BF8F7E0FD53EC182B83
:10DA8000F8F7D9FD41EC180B53EC1B2B51EC190B9B
:10DA9000F8F7D4FDDFF8C8A241EC100B4FEA155897
:10DAA0000125FA4453EC102B51EC180BF8F7C0FD8C
:10DAB000032DC4E900013DD0C1F30A5005EB451127
:10DAC000A8EB00001139814234DA0AEB051BB0EEF5
:10DAD00048AA9BED000BF0EE68AA53EC102B51EC1A
:10DAE000190BF8F7ABFD41EC1B0B51EC1A0B53EC87
:10DAF0001B2BF8F79DFD41EC180B51EC1A0B53EC66
:10DB0000182BF8F795FD53EC1B2BF8F791FD9BEDC7
:10DB1000020B41EC1A0B53EC102B51EC190BF8F7DC
:10DB20008DFD53EC1A2BF8F783FD41EC100B6D1CA7
:10DB3000B8E70EE0002EA8BF3846BFF628AF94ED38
:10DB4000000B51EC100B81F00041C4E90001784258
:10DB50001DE7C6F3130040F4801EC6F30A50A0F27E
:10DB6000F530471100F01F05C5F12000DDF848B081
:10DB700008900020069007900520EC467949002D7A
:10DB800007EB0002794408BF51F8221009D051F880
:10DB9000223001EB8201AB404A68089922FA01F178
:10DBA0001943A1FB0E26A1FB0B131A449A4234BF62
:10DBB0000123002303EB06080CEB8003D3E901A645
:10DBC0000E448E4234BF0121002192448A4411B197
:10DBD000924502D903E0924501D2012100E00021E3
:10DBE000C3E901A641444CF82010011EA0F1010038
:10DBF000C4DC029800F10050850F0298DDE903674C
:10DC00008000DDF81480F8F7FAFD41EC1A0B30467D
:10DC1000F8F706FE9FED541B53EC112BF8F70EFDA1
:10DC200041EC1B0B3846F8F7FBFD9FED511B53EC05
:10DC3000112BF8F703FD41EC180B4046F8F7F0FD07
:10DC40009FED4D1B53EC112BF8F7F8FC41EC190B31
:10DC500051EC180B53EC192BF8F749FC53EC1B2B28
:10DC6000F8F745FC53EC1A2BF8F741FCCDE9080115
:10DC7000002008909DED080B53EC1A2B51EC100B73
:10DC8000F8F7D6FC53EC1B2BF8F7D2FC53EC182B0F
:10DC9000F8F7CEFC53EC192BF8F7CDFC9FED381BB1
:10DCA00053EC112BF8F7CAFC9FED370B41EC180B26
:10DCB00053EC102B9DED080B51EC100BF8F7BEFC4C
:10DCC00053EC182BF8F713FC9FED310B41EC180BBC
:10DCD00053EC102B9DED080B51EC100BF8F7AEFC3C
:10DCE00053EC182BF8F703FC41EC100B139810F0D1
:10DCF000004F06D06D4251EC100B81F0004141EC19
:10DD0000100B284684ED000B41E6000000000000E7
:10DD10000000000000000000FB21E93F7CD9024028
:10DD200000004054FB21F93F3163621A61B4D03DD9
:10DD3000FB21F93F000000000000601A61B4D03DF3
:10DD40007370032E8A19A33BFB21394100000000A8
:10DD500083C8C96D305FE43F000000000000E03F71
:10DD60004292010090910100000000000000103E6E
:10DD7000000000000000103C000000000000103A0D
:10DD8000182D4454FB21F93D3326A611460B113CB6
:10DD900000000054FB21F93D10B52DED040B2DEDD5
:10DDA000088B82B0B0EE419AF0EE619A0B9820F0A9
:10DDB00000449FED4BABB4F1795F11DA9DED0A0B96
:10DDC00051EC100BF8F739FD002801BFB0EE4A0AFC
:10DDD000F0EE6A0A02B0BDEC088B04BF04B010BDBF
:10DDE0009DED0A0B53EC102B51EC100BF8F726FCB1
:10DDF00041EC180B3C480621B0EE480AF0EE680AE8
:10DE0000784400F081F853EC182B51EC100BF8F724
:10DE100015FC9DED0A0B41EC1B0B53EC192B51EC3F
:10DE2000100BF8F70BFC41EC190B53EC1B2B51ECCE
:10DE3000180BF8F703FC53EC192BF8F7F9FB9FEDDF
:10DE40002C0B41EC190B53EC102B51EC180BF8F781
:10DE5000F5FB41EC100B2848844210DA53EC192BE7
:10DE600051EC100BF8F7E4FB53EC1A2BF8F7E3FB3B
:10DE700041EC100B02B0BDEC088B04B010BD1F4884
:10DE8000A042BCBF9FED1E1B8DED001B06DBA4F561
:10DE900000100190002000909DED001B51EC100B34
:10DEA00053EC112BF8F7C4FB9DED000B41EC180B64
:10DEB00053EC102B51EC1A0BF8F7BAFB41EC1A0B90
:10DEC00053EC192B51EC180BF8F7B2FB53EC1A2B4F
:10DED000F8F7B1FB41EC100BCCE7000000000000AC
:10DEE000000000000000F03FAC8E010000000000C8
:10DEF000000000000000E03F3333D33F0000E93F63
:10DF0000000000000000D23F70B504462DED028BEA
:10DF10004D1E00EBC500B0EE408AF0EE608A90ED39
:10DF2000000B35F0060017D053EC182B51EC100BFA
:10DF3000F8F784FB41EC100B6D1E04EBC50090ED6F
:10DF4000001B51EC100B53EC112BF8F7D0FA41ECFD
:10DF5000100B35F00600E7D1022D36D0042D1CD071
:10DF6000062D1CBFBDEC028B70BD53EC182B51EC81
:10DF7000100BF8F763FB94ED0A1B53EC112BF8F729
:10DF8000B6FA53EC182BF8F759FB94ED081B53EC39
:10DF9000112BF8F7ACFA41EC100B53EC182B51ECA9
:10DFA000100BF8F74BFB94ED061B53EC112BF8F715
:10DFB0009EFA53EC182BF8F741FB94ED040B53EC4D
:10DFC000102BF8F794FA41EC100B53EC182B51EC92
:10DFD000100BF8F733FB94ED021B53EC112BF8F701
:10DFE00086FA53EC182BF8F729FB94ED001B53EC41
:10DFF000112BF8F77CFABDEC028B41EC100B70BDD5
:10E0000031B504462DED040B2DED0A8BB0EE41BA6F
:10E01000F0EE61BA0B989DED0A0B20F00040B0F1D4
:10E02000795F0DDA51EC100BFEF70AFD042808BFEA
:10E0300000F0A2F89DED0A0BBDEC0A8B05B030BDD7
:10E0400053EC102B51EC100BF8F7F8FA41EC180BCD
:10E050009DED0A0B53EC182B51EC100BF8F7EEFA70
:10E0600041EC190B2C48B0EE480AF0EE680A052185
:10E070007844FFF749FF9FED2ACBB0EE40AAF0EEBF
:10E0800060AA9CB353EC1C2B51EC190BF8F7D6FA91
:10E0900041EC1C0B53EC1A2B51EC190BF8F7CEFA90
:10E0A0009FED210B41EC190B53EC102B51EC1B0B8A
:10E0B000F8F7C4FA53EC192BF8F7BAFA53EC182B0B
:10E0C000F8F7BCFA53EC1B2BF8F7B2FA53EC1C2B05
:10E0D000F8F7AEFA9DED0A1B53EC112BF8F7ABFAEB
:10E0E000BDEC0A8B05B041EC100B30BDFFE753ECE3
:10E0F0001A2B51EC180BF8F7A1FA53EC1C2BF8F77C
:10E10000F6F953EC192BF8F799FA9DED0A1B53EC2D
:10E11000112BF8F7ECF9E3E73C8D0100000000005B
:10E12000495555555555C5BF000000000000E03F5A
:10E1300010B553EC102B51EC100BF8F7D8F941EC5B
:10E14000100B10BD10B553EC112B51EC100BF8F760
:10E15000CEF941EC100B10BD9FED050B10B553EC43
:10E16000102B51EC100BF8F7DBFA41EC100B10BD43
:10E1700000000000000000009FED050B10B553ECFF
:10E18000102B51EC100BF8F759FA41EC100B10BDA5
:10E19000000000000000001030EE000A704730EE72
:10E1A000200A7047DFED020A80EEA00A70470000E7
:10E1B000000000009FED020A20EE000A70470000F8
:10E1C0000000001002E008C8121F08C1002AFAD19E
:10E1D00070477047002001E001C1121F002AFBD1E7
:10E1E000704700000146202908DA012088400A4AC9
:10E1F000104008B1012070470020FCE7402909DAEF
:10E20000A1F12000012202FA00F008B10120F2E79A
:10E210000020F0E70120EEE7FC06FFBD00BFEFF3B2
:10E220001081084672B670470149086070470000C7
:10E230001C4B00202DE9FF5F82B00021DDE9043096
:10E24000020DDDF840B0034318D044F61050A2F29E
:10E25000FF3242431514119801281FD0A5EB0B0083
:10E26000401C5FEA000A4FF000064E4FDFF838917D
:10E27000B046504615D5CAF1000413E011980124A8
:10E280004AA3012801D16FEA0B010298119AC0E953
:10E290000031C0E9024206B0BDE8F09FCBF10000BA
:10E2A000DFE704460021404A491842EB0450CDE91B
:10E2B000001012E0E00707D032463B464046494690
:10E2C000F8F7BCF98046894632463B461046194667
:10E2D000F8F7B4F906460F466410002CEAD1DDE9E0
:10E2E0000401DDE90023BAF1000F06DAF8F7A6F918
:10E2F00042464B46F8F7A2F905E0F8F711FA424614
:10E300004B46F8F70DFA04460E460022284BF8F764
:10E31000F7FA03D84FF0FF30014607E00022254B03
:10E3200020463146F8F7E3F8F8F74AFC102409E0F4
:10E33000002C0ADB0A220023F8F762F8039B303234
:10E340001A55641E50EA0102F2D1641C039AC4F10A
:10E3500011031444119A012A03D0012208430DD15C
:10E360000AE0084304D000204FF0110B119072E72F
:10E37000A3EB0B056D1E0DE05B4504DD4FF00002C5
:10E3800005F1010504E003DA4FF00002A5F10105F3
:10E39000002AECD002981199C0E90231C0E9004589
:10E3A00079E70000000014400000F03F300000005A
:10E3B0000000F0430000E03F2DE9FF4F95B09B4681
:10E3C0008946064600250FE2252877D100242746F6
:10E3D000F84A0121059400E0044316F8013F203B70
:10E3E00001FA03F01042F7D130782A2811D06FF0EB
:10E3F0002F033078A0F13002092A16D8059A44F08C
:10E40000020402EB820203EB42021044761C0590E8
:10E41000EFE759F8042B0592002A03DA504244F43E
:10E420000054059044F00204761C30782E2816D152
:10E4300016F8010F44F004042A280DD06FF02F02C3
:10E440003078A0F13003092B09D807EB870302EBE2
:10E450004303C718761CF3E759F8047B761C307821
:10E460006C280FD006DC4C2817D068280DD06A28FD
:10E4700014D104E0742810D07A280FD10DE044F4B0
:10E4800000140AE044F4801401E044F4401472786B
:10E49000824202D104F58014761C761C30786628FE
:10E4A0000BD013DC582877D009DC002875D045281C
:10E4B000F6D04628F4D047281AD19DE118E0632809
:10E4C00035D0642879D0652812D195E1702873D0B1
:10E4D00008DC6728F1D069286FD06E280DD06F282E
:10E4E00006D1B5E073282CD0752875D0782874D063
:10E4F0005A46179990476D1C75E1C4F302500228E3
:10E5000009D003280DD0D9F8001004280DD00D60D3
:10E5100009F1040967E1D9F80010EA17C1E90052CE
:10E52000F6E7D9F800100D80F2E70D70F0E719F862
:10E53000041B8DF8001000208DF80100EA46012030
:10E5400003E059F804AB4FF0FF3061074FF00001D2
:10E5500002D40DE008F101018846B9420FDA804586
:10E56000F8DB1AF808100029F4D108E008F10101DD
:10E5700088468142FADB1AF808100029F6D105987E
:10E580005B46A0EB080721463846179A00F094FA3C
:10E59000284400EB080507E04DE029E10DE01AF8FA
:10E5A000010B5A4617999047B8F10108F7D25B461C
:10E5B00021463846179A13E142E00A220092C4F33A
:10E5C00002524FF0000A022A08D059F804CB032A5D
:10E5D0004FEAEC710AD00DE029E02AE009F10701C9
:10E5E00021F00702F2E802C1914609E00FFA8CFC23
:10E5F0004FEAEC71042A03D14FFA8CFC4FEAEC711C
:10E60000002907DA0A460021DCF1000C61EB020167
:10E610002D2202E0220504D52B228DF804200122B0
:10E6200003E0E20701D02022F7E7904659E00A21F3
:10E6300002E010220DE010214FF0000A00910BE0E3
:10E6400010224FF0000A44F004040827009203E06F
:10E6500008224FF0000A0092C4F30252022A05D0A9
:10E6600059F804CB0021032A08D009E009F1070179
:10E6700021F00702F2E802C1914605E01FFA8CFC86
:10E68000042A01D10CF0FF0C4FF00008220728D516
:10E69000702806D0009B83F0100353EA0A0305D0CC
:10E6A0000EE040228DF80420012208E05CEA01021D
:10E6B00006D030228DF804208DF805000222904605
:10E6C000009B83F0080353EA0A030AD15CEA0102C3
:10E6D00001D1620705D530228DF804204FF00108E2
:10E6E0007F1E582804D034A003900EA802900DE09D
:10E6F00036A0F9E753466046009AF7F781FE844654
:10E700000398825C0298401E029002705CEA01004D
:10E71000F0D1029806A9081A00F1200A600702D574
:10E7200024F4803400E00127574502DDA7EB0A00FE
:10E7300000E0002000EB0A01009005984144401AD7
:10E740000590E00306D45B462146179A059800F031
:10E75000B3F90544002706E001A85A46C05D1799A1
:10E7600090476D1C7F1C4745F6DBE0030CD55B46EC
:10E770002146179A059800F09FF9054404E03020DF
:10E780005A46179990476D1C0099481E0090002921
:10E79000F5DC08E0029802995A460078491C02917B
:10E7A000179990476D1CBAF10001AAF1010AF1DC3A
:10E7B00065E1000009280100303132333435363745
:10E7C00038396162636465660000000030313233BD
:10E7D000343536373839414243444546000000005D
:10E7E00000F058F90544761C307800287FF4ECAD31
:10E7F00019B02846BDE8F08F620700D4062709F15A
:10E80000070222F0070CFCE80223E14603F000486F
:10E810005FEA080C02D00FF2702C0DE05FEA045C96
:10E8200002D50FF2682C07E05FEAC47C02D00FF239
:10E83000602C01E0AFF2700C4FF0FF3823F0004382
:10E84000CDF850C065280CD006DC452809D04628F4
:10E850001DD047283DD13DE0662818D067287ED1DD
:10E8600038E00021112F01DB112000E0781CCDE9F8
:10E87000000106A90EA8FFF7DDFCDDE90F010E9AE5
:10E8800003910021009207F1010A04914DE04FF03D
:10E8900000400097CDE9011006A90EA8FFF7CAFCB9
:10E8A000DDE90F0203920E9B11990022DDF80CA006
:10E8B0000093049211B9791C00EB010AB7EB0A002E
:10E8C00004D4C0F1FF3007F1010A0490AAEB07005D
:10E8D000019044E0012F00DA01270021112F01DD12
:10E8E000112000E03846CDE9000106A90EA8FFF787
:10E8F000A1FCDDE90F010E9A039100210491009221
:10E90000BA4621070CD40399514500DA8A46BAF178
:10E91000010F05DD009AAAF10101515C302908D0F0
:10E92000B84202DA10F1040F06DA0121CDE9011034
:10E9300015E0AAF10101E9E7002805DC049901448A
:10E940000491AAEB000102E0411C514500DD8A461A
:10E950000499401A401C01904FF00040029020079B
:10E9600004D40198504501DBCDF8048000208DF8D7
:10E970004F0002980DF14F07B0F1004F25D02B202A
:10E980000E9002984FF0020800280CDA40420290E4
:10E990002D200E9007E00A210298F7F7E5FF3031AD
:10E9A000029007F8011DB8F10001A8F10108F2DC9E
:10E9B00002980028EFD1791E0E980870307800F088
:10E9C000200040F0450007F8020D12A8C01B00F11E
:10E9D00007081498007800B1012000EB0A010198A3
:10E9E00001EBE07105984144401A401E0590E00398
:10E9F00006D45B462146179A059800F05DF8054459
:10EA00001498007818B15A46179990476D1CE00386
:10EA100024D55B462146179A059800F04DF8054429
:10EA20001CE00498002807DBDDE90301884203DDD0
:10EA30000098405C179901E0179930205A4690479A
:10EA4000049805F10105401C04900198401E0190B6
:10EA500004D12E205A46179990476D1CBAF1000137
:10EA6000AAF1010ADDDC05E017F8010B5A461799F7
:10EA700090476D1CB8F10001A8F10108F4DC5B4679
:10EA80002146179A0598ABE62D0000002B000000E8
:10EA9000200000002DE9F041044600251E461746DF
:10EAA000880404D405E039462020B0476D1C641E5C
:10EAB000F9D52846BDE8F0812DE9F041044600254E
:10EAC0001E469046C80301D5302700E02027880461
:10EAD00004D505E041463846B0476D1C641EF9D5A3
:10EAE0002846BDE8F0810A68531C0B60107070471F
:10EAF0002DE9FC4105461CA103C9CDE90001002711
:10EB0000287800282DD11A4A128891B2686811F02D
:10EB1000A3FD06462EBB00240BE004EBC400154900
:10EB20000844C07920B1E0B20DF80700781CC7B2E4
:10EB3000641C082CF1DB002408E00F4830F81400B6
:10EB40001DF804100D4A22F81100641C08480068E2
:10EB50008442F2D30A48006818B108480849096895
:10EB60008847BDE8FC810000FFFFFFFFFFFFFFFFBC
:10EB70006C410020AC790020F4790020047A002058
:10EB80007041002070470246002104E0505C08B14B
:10EB900001207047491C0629F8D30020F9E770B519
:10EBA00004460D4604F22740FFF7EDFF0646012D0F
:10EBB00006D0022D0DD0032D11D0042D19D113E054
:10EBC000A07928B194F8240010B90EB1012070BDCD
:10EBD00000BFE07910B10EB10220F8E700BF207A43
:10EBE00008B10320F3E700BF607A08B10420EEE724
:10EBF00000BF0020EBE70146481C052290FBF2F322
:10EC000002FB1300C0B270472DE9F04704460D46E1
:10EC10002F4695F82080B4F81C9000260BE007EBF7
:10EC200046124946A06902F0FCFE10B10120BDE881
:10EC3000F087701CC6B24645F1DB0020F7E70146BD
:10EC400091F82420012A01D1EE2000E01F20704716
:10EC5000014671B1002009E0064A52F820201AB995
:10EC6000044A42F8201003E0421CD0B20228F3DB31
:10EC700000BF70474C480020014600200BE0084AC6
:10EC800052F820208A4204D10022054B43F820206C
:10EC900003E0421CD0B20228F1DB00BF7047000045
:10ECA0004C48002030B5B1B004200590AC2106A836
:10ECB000F7F7F0FB02208DF8180000208DF81A00FD
:10ECC00004908DF8100001208DF8110004208DF8BB
:10ECD000120001208DF813001E20ADF8040004A9D5
:10ECE00003910420ADF8080001A91E9105208DF8BC
:10ECF0001B0005A807900121ADF8641011491A9175
:10ED000001218DF894104FF4A071289144F25061C4
:10ED100029910D482F9006A90C4802F0EEFE0446FA
:10ED200000BF254635B100BF09A28C212846F7F760
:10ED300071FA00BF00BF0121044802F0DBFE31B0D0
:10ED400030BD0000CC410020E50F0400647B0020B2
:10ED50002E2E5C2E2E5C2E2E5C626C655F636667C9
:10ED60005C736C6176652E630000000070B5032152
:10ED7000084802F064FF0446082C0AD000BF25466C
:10ED800035B100BF04A2AD212846F7F743FA00BF12
:10ED900000BF70BD647B00202E2E5C2E2E5C2E2EBC
:10EDA0005C626C655F6366675C736C6176652E633D
:10EDB0000000000070B5094991F8540074DF044662
:10EDC000082C0AD000BF254635B100BF04A2B621E9
:10EDD0002846F7F71FFA00BF00BF70BD647B002014
:10EDE0002E2E5C2E2E5C2E2E5C626C655F63666739
:10EDF0005C736C6176652E63000000001CB5FAF749
:10EE0000C4FCFCF797FA00210F480DF090FD01A912
:10EE10000D480DF07BFD9DF8040010B14FF0FF3060
:10EE20001CBD002108480DF0B9FD02200090694684
:10EE300005480DF095FD9DF8000010B14FF0FF3032
:10EE4000EEE70020ECE70000987A002010B5054AB4
:10EE500005A16420FBF76EFD0649B020F8F7C8F95C
:10EE600010BD000079EE02006170705F417574683A
:10EE70006F6E00001D3E030010B51C480079C8B13C
:10EE80000BF022FD78B11A4800781E2812DA1848D3
:10EE90000078401C164908700123164AB021002052
:10EEA000F8F758FC06E012480078002802DD002040
:10EEB0000F49087016F09AFC80B10F4800780028BE
:10EEC00013DD0D480078401CC0B20B49087096282D
:10EED0000BDD9620087016F051FC06E0064800781D
:10EEE000012802D001200449087010BD7853002089
:10EEF0003D4000203E4000203C40002010B50E4820
:10EF00000079B8B101F068FAA0B10C480179007934
:10EF1000401C0A4A107105290CDB00201146C870FC
:10EF2000074803F063FE0123044AD21CA2210020FB
:10EF3000F8F710FC10BD0000785300203C3F002083
:10EF40003066040010B51448007850B10020124912
:10EF5000087012490820FAF7C7FA01211048FBF798
:10EF6000C3FC1C2000BF4FF0A042114600BFD1F8E7
:10EF70001025C24002F0010400BF54B909480068DE
:10EF8000A04206D00820FAF7CFFA00210448FBF788
:10EF9000ABFC0448046010BDF83F00209F009FFFB9
:10EFA00045EF02000040002030B587B0182101A8CD
:10EFB000F7F770FA0BF036FC08B907B030BD002443
:10EFC000002003F05BFE04B2002C7DDD611E01AA6F
:10EFD000002003F049FEBDF9082065480388654913
:10EFE000654816F00DFD62480088052826DDBDF94C
:10EFF00008006049B1F90010401AFF281BDC5E4888
:10F00000B0F90000BDF90810401AFF2813DC5A4877
:10F01000B0F900005749B1F90010401AFF280ADC86
:10F02000BDF9040010F5167F05DA54480088401C2D
:10F030005249088002E00020504908804C4800886E
:10F04000401C4B490880BDF8040010FB00F0BDF8DF
:10F05000061011FB0100BDF8081011FB0105A5F514
:10F060008000002801DB014600E04142444A914211
:10F070000ADABDF90810B1F5C06F05DD4148008816
:10F08000401C4049088002E000203E4908803D487D
:10F090000088052803DA39480088042802DD0620A4
:10F0A0003949087038480078002804DD364800786F
:10F0B000401E3549087034480078002839DD33484F
:10F0C000007800BB642000E04FE030490870F9F799
:10F0D0007FFB142804DD2E490420FAF705FA03E02B
:10F0E0002C490420FAF700FA0121AFF24310FBF794
:10F0F000FBFB2948007990B10123284AB021284818
:10F10000F8F74CF90BE021480078022807D10420D9
:10F11000FAF70AFA0021AFF26F10FBF7E5FB1B4884
:10F120000078012820DD19480078401E1749087032
:10F130001AE01648007850B10020144908700420E5
:10F14000FAF7F2F90021AFF29F10FBF7CDFB15485B
:10F15000007848B90120134908700420FAF7E4F94F
:10F1600000211148FBF7C0FB00BF00BF25E70000EE
:10F17000643E0020843E00206C3E0020663E00205D
:10F18000A0860500683E00206A3E00206B3E0020FD
:10F19000009F00FF00103FFF78530020393E002001
:10F1A0003C3E0020383E0020ADF1020030B587B073
:10F1B000182101A8F7F76EF90BF034FB08B107B07E
:10F1C00030BD0025002003F059FD05B2002D7DDD86
:10F1D000691E01AA002003F047FDBDF8040010FBE2
:10F1E00000F0BDF8061011FB0100BDF8081011FB7E
:10F1F0000104A4F58000002801DB014600E0414243
:10F200005D4A914208DABDF90810B1F5C06F03DD1F
:10F2100003205A49087008E058480078002804DDA7
:10F2200056480078401E55490870A4F58000002813
:10F2300001DB014600E041424F4A914208DABDF944
:10F24000041011F5617F03DA03204D49087008E0CE
:10F250004B480078002804DD49480078401E4849A2
:10F260000870A4F58000002801DB014600E041425F
:10F27000414A914207DABDF9081011F5806F02DAB0
:10F2800000203E490870A4F58001002901DB0A46F0
:10F2900000E04A42384B9A420CDABDF904000028DB
:10F2A00001DB024600E04242B2F5C87F02DA0020EC
:10F2B0003349087031480078002803DC3048007872
:10F2C000002839DD2F48007800BB00E052E00A201A
:10F2D0002C490870F9F77CFA142804DD2A49042027
:10F2E000FAF702F903E029490420FAF7FDF80121B1
:10F2F000AFF24710FBF7F8FA2548007990B10123E7
:10F30000244AB0212448F8F749F80BE01D4800785A
:10F31000022807D10420FAF707F90021AFF2731091
:10F32000FBF7E2FA17480078012822DD154800783B
:10F33000401E144908701CE01248007850B10020AB
:10F34000104908700420FAF7EFF80021AFF2A3107B
:10F35000FBF7CAFA1148007801280AD100200F49AA
:10F3600008700420FAF7E0F80021AFF2BF10FBF7B5
:10F37000BBFA00BF00BF22E7A0860500603E002068
:10F38000613E0020623E0020009F00FF00103FFF12
:10F3900078530020393E00203C3E0020383E0020BB
:10F3A00001480079704700007853002010B58AB0FA
:10F3B00000246846F9F730FA00980290BDF804007E
:10F3C000ADF80C00A41D00222146641C02A8425482
:10F3D00001222146641C425404222146641C4254EA
:10F3E00001222146641C425400222046611CCCB2FA
:10F3F00002A90A541E222046611CCCB202A90A545A
:10F400000AF0C0FE022803D00AF0BCFE032806D191
:10F4100001222046611CCCB202A90A5405E0002258
:10F420002046611CCCB202A90A540948007930B1C7
:10F43000234602AAB1210020F7F7B0FF05E02346DA
:10F4400002AAB1210020F8F785F90AB010BD00002A
:10F450007853002010B5034A03A16420FBF76AFA31
:10F4600010BD000075F402006170705F6368617226
:10F470006765000010B50AF085FE04461448007860
:10F48000844224D0012C04D0022C0AD0032C1AD19F
:10F4900010E00520FAF748F800210E48FBF724FA9F
:10F4A00012E001210B48FBF71FFA0B490520FAF780
:10F4B0001BF809E001210748FBF716FA0749052068
:10F4C000FAF712F800E000BF00BF0148047010BD59
:10F4D0000440002075F4020000103FFF009F00FF71
:10F4E00030B589B00024202101A8F6F7D3FF684683
:10F4F0004CDF00988010009001222146641C01A876
:10F500004254F9F765F901462246641C01A881546A
:10F510000098C2B22146641C01A84254241D3B48F5
:10F520004069020E2146641C01A8425437484069D4
:10F53000C0F307422146641C01A842543348808A24
:10F54000C0F307222146641C01A842542F48027DC3
:10F550002146601CC4B201A8425401F003F92146BF
:10F56000621CD4B201AA505401F0F0F82146621C8A
:10F57000D4B201AA5054201DC4B224488069020E9E
:10F580002046611CCCB201A90A5420488069C0F30E
:10F5900007422046611CCCB201A90A541B48008BCB
:10F5A000C0F307222046611CCCB201A90A541748B7
:10F5B000027E2046611CCCB201A90A540AF01EFC4E
:10F5C0000546C5F307222046611CCCB201A90A54A6
:10F5D0002046611CCCB201A90D5401F0BDF8C0F366
:10F5E00007222046611CCCB201A90A5401F0B4F8EC
:10F5F000C2B22046611CCCB201A90A54234601AA1A
:10F60000A1210020F7F7CAFE09B030BD78530020D1
:10F6100070B50546002400BF06E0601C6968095CFF
:10F620000A480155601CC4B2082CF6DB6968487AA8
:10F6300001F06EF905480C38406A28B100210348F2
:10F640000C38416208F0ECFD70BD000084530020CE
:10F6500010B50649A120F7F7CBFD00F037FA044AB0
:10F6600004A14FF4FA60FBF765F910BD4D410300AA
:10F6700081F602006170705F636C69656E740000F2
:10F6800010B50E48007900B110BD16F0AFF890B17A
:10F6900000F0A2FE68B10A4801780078401C084AD0
:10F6A0001070042907DB002011460870FFF718FFCF
:10F6B00001E0FFF715FF00BFE6E7000078530020E8
:10F6C000863F002070B5044660688078616849789C
:10F6D00040EA01251648406AA0B11548406A401E1C
:10F6E0002821B0FBF1F0401C124908801048406A04
:10F6F000401E2821B0FBF1F201FB1200401C0E4914
:10F70000088004E000200B4908800B49088055B9A7
:10F7100001200A490870002009490880084600882D
:10F7200000F010F802E0284600F0D8F870BD0000A4
:10F7300078530020A03E0020A23E00209D3E0020E5
:10F740009E3E00202DE9F0410546002408F065FDAD
:10F75000691EA02202FB010702222146641C5648B2
:10F760004254002007E055490B5C2146621CD4B28C
:10F77000514A5354401C0828F5DB514800880212B6
:10F780002046611CCCB24C490A544D4802782046B0
:10F79000611CCCB248490A542A122046611CCCB2E2
:10F7A00045490A542046611CCCB243490D54002DF2
:10F7B00034D101F08BFC804601F08EFC08EB000692
:10F7C000320E2046611CCCB23B490A54C6F30742B4
:10F7D0002046611CCCB238490A54C6F307222046A1
:10F7E000611CCCB234490A542046611CCCB2324967
:10F7F0000E54E01E085CFF280FD1A01E085CFF28F5
:10F800000BD1601E085CFF2807D10846005DFF2869
:10F8100003D12CA10B20F8F783FA44E02848008894
:10F82000854222D12B48008882002348011938469E
:10F8300008F0DEFC2748007804EB8000C4B2201FEB
:10F840001D49085CFF282ED1E01E085CFF282AD144
:10F85000A01E085CFF2826D1601E085CFF2822D16C
:10F8600018A10B20F8F75CFA1DE013480119A0223B
:10F87000384608F0BDFC04F1A000C4B2201F0E49B8
:10F88000085CFF280FD1E01E085CFF280BD1A01EEA
:10F89000085CFF2807D1601E085CFF2803D109A17E
:10F8A0000B20F8F73DFA2346034AA1210A48F7F74F
:10F8B00075FDBDE8F08100006451002084530020F4
:10F8C000A03E002073746570206F766572666C6F61
:10F8D00077000000A23E0020A43E002070B5C0B01A
:10F8E0000546002408F099FC691EA02202FB0106CF
:10F8F00002222146641C01A84254002007E023494B
:10F900000B5C2146621CD4B201AA5354401C082847
:10F91000F5DB1F48008802122046611CCCB201A909
:10F920000A541B4802782046611CCCB201A90A5433
:10F930002A122046611CCCB201A90A542046611C3F
:10F94000CCB201A90D541248008885420DD111484E
:10F950000088820001A80119304608F049FC0D48D2
:10F96000007804EB8000C4B208E001A80119A022CD
:10F97000304608F03DFC04F1A000C4B2234601AAC1
:10F98000A1210020F7F70AFD40B070BD845300208C
:10F99000A03E0020A23E002030B5A1B041240025A9
:10F9A000802101A8F6F776FD00208DF8040000BF45
:10F9B00005E03FA0415D01AA681C11546D1C0B2D90
:10F9C000F7D301A90819F8F727FFA01DC4B2002238
:10F9D0002046611CCCB201A90A5401222046611CB8
:10F9E000CCB201A90A5404222046611CCCB201A960
:10F9F0000A5401222046611CCCB201A90A540022FB
:10FA00002046611CCCB201A90A541E222046611C6A
:10FA1000CCB201A90A54002507E02848425D2046DF
:10FA2000611CCCB201A90A546D1C062DF5DB2348DC
:10FA30003238C06A020E2046611CCCB201A90A54B9
:10FA40001E483238C06AC0F307422046611CCCB25F
:10FA500001A90A5419483238808DC0F30722204684
:10FA6000611CCCB201A90A541448323890F82C20F9
:10FA70002046611CCCB201A90A5410483238008ECD
:10FA800002122046611CCCB201A90A540B4832383C
:10FA900090F830202046611CCCB201A90A542346BC
:10FAA00001AAA1210020F7F779FC21B030BD0000A8
:10FAB000534D4152542053484F450000AA53002053
:10FAC00001480078704700009C3E002010B5074AAE
:10FAD00007A14FF47A70FAF72DFF09484169C06910
:10FAE000814202D206484169C16110BD05FB020096
:10FAF0006170705F636C69656E745F7374657000CC
:10FB00007853002010B51C48007820B101280DD092
:10FB1000022829D11BE019480078012805D116498F
:10FB20000870FCF7DBFC1649086023E0FCF7D6FC04
:10FB300013490968401A42F21071884203D3022027
:10FB40000D49087002E0012000F0DAFD12E0F8F73C
:10FB50008FFD18B10BA10B20F8F7E2F80020074940
:10FB600008700549087005E0002003490870034942
:10FB7000087000BF00BF10BDC83E00209C3E0020A2
:10FB8000CC3E0020736176652073746570206661D9
:10FB9000696C000001200149087070479C3E0020FC
:10FBA00010B53248007810B1012853D109E015F0A2
:10FBB0001DFE28B101202D49087000202C49087035
:10FBC00051E00AF081FE80B129480078B8B90120DF
:10FBD0002749087000F0E2F92649087001230A4617
:10FBE000A3212548F7F7B6FD09E021480078002851
:10FBF00005DD00201E4908701F48F7F753FD1F4818
:10FC0000008898B1FCF76AFC1D490968401A1B4935
:10FC1000098888420AD30020184908800420F9F78F
:10FC200083FC0021AFF28700FAF75EFE15F0DEFDDF
:10FC300078B900200D490870104908800021AFF202
:10FC40009F00FAF751FE0420F9F76EFC0A48F7F717
:10FC500029FD08E0002005490870084908800420B3
:10FC6000F9F762FC00BF00BF10BD0000B53F0020E7
:10FC7000B43F0020B63F0020883F0020AC3F00206A
:10FC8000B03F002010B583480079A0B982480078C1
:10FC900001280FD1002080490870804908708049F0
:10FCA000086080490880804908700021AFF22B006D
:10FCB000FAF71AFE10BD78480078012802D001201A
:10FCC000754908707548007820B101282BD00228AA
:10FCD00073D173E0FFF7F4FE30B915F087FD18B962
:10FCE0000AF050FA012812D000F090FF78B901F024
:10FCF000C5F860B90121AFF27300FAF7F5FD13F012
:10FD0000C1FF00206649086001206449087061480D
:10FD1000007938B115F06AFD20B90AF0D5FD08B1B7
:10FD20000AF08AFDB3E0FFF7CBFEA8B915F05EFD3F
:10FD300090B90AF027FA01280ED15CA10E20F7F73E
:10FD4000EFFF0FF0D4F80021AFF2C700FAF7CCFDB7
:10FD500000205249087012E00AF0B6FD78B1002187
:10FD6000AFF2DF00FAF7C0FD4A48007920B1002069
:10FD70004C4908804C49087002204849087048489E
:10FD80000068401C46490860642815D3FFF798FEB8
:10FD900040B9404890F82800432803D14AA10F20D9
:10FDA000F7F7BEFF0FF0A3F80021AFF22710FAF724
:10FDB0009BFD00203949087069E064E000F00CFB0D
:10FDC00018B339480078022842D0364800883C28C9
:10FDD0003EDCF1EE0E0AB1EE0E0AF7F733FD30B954
:10FDE00002203149087000202E49088030E02D485B
:10FDF00000883C2803D13BA10F20F7F791FF294849
:10FE00000088401C2749088022E027480078012804
:10FE10001ED0244800883C281ADCDFED3B0A9FED09
:10FE20003A0AF7F70FFD30B901201F49087000208A
:10FE30001C4908800CE01B4800883C2803D133A1F2
:10FE40000F20F7F76DFF17480088401C1549088000
:10FE5000FFF736FE58B915F0C9FC40B90AF092F91F
:10FE6000012804D10AF030FD08B10AF0E5FC0AF0DF
:10FE70002BFD38B90021AFF2F310FAF735FD002061
:10FE80000649087003E000200449087000BF00BF65
:10FE900000BF0FE778530020BF3F0020B73F00208E
:10FEA000B83F0020BC3F0020BE3F002061647620A8
:10FEB000646973636F6E6E746564206F766572201B
:10FEC00074696D65000000007363616E207269677C
:10FED00068742073686F6573206F7665722074692B
:10FEE0006D65000075706461746520426C65206307
:10FEF0006F6E6E20696E74657276616C20372E3578
:10FF00006D73206661696C000000C84275706461A1
:10FF1000746520426C6520636F6E6E20696E746537
:10FF20007276616C203130306D73206661696C00CF
:10FF300010B50E4A0EA16420FAF7FCFC0E48F7F744
:10FF40005DFC0E48F7F736FC0D4A0EA16420FAF767
:10FF5000F1FC0F49A320F7F74BF90E49A320F7F75F
:10FF60001BFB0D49AC20F7F743F910BD85FC0200DF
:10FF7000636F6E6E656374002147030001470300E1
:10FF8000A1FB0200636F6E6E6563745F6C65640055
:10FF90002544030089450300BD3D030010B500243E
:10FFA000064890F82800432801D0022403E00AF014
:10FFB0008BFC00B10124204610BD000078530020C6
:10FFC00010B5054A05A10020FAF7B4FC0748F7F779
:10FFD0000DFB002010BD0000F1FF020064617461A0
:10FFE0005F7472616E7366657200000091000300B9
:10FFF00010B500F0F1F918B901F0E6F9002832D097
:020000040003F7
:100000001E48007830B901201C49087001211C48A5
:10001000FAF76AFCFCF762FA1A490968401AB0F567
:10002000FA7F12D3FCF75AFA1649086015F0DEFB86
:1000300018B9FEF7BFFEFEF799FE1348007920B10C
:100040000AF042FC08B913F01DFEFCF747FA0F490D
:100050000968401A032810D3FCF740FA0B490860DE
:10006000F8F7D2FE09E00548007830B100200349D6
:10007000087000210248FAF737FC10BDF43F002059
:10008000F1FF0200EC3F002078530020F03F0020F9
:1000900070B504460D46E078042803D12946204671
:1000A000F8F76EFF00F0F8FA70BD000010B588B0E8
:1000B000002004900590069007904A4890F8280088
:1000C000432868D10AF000FC08B10AF0B5FB15F02E
:1000D0008DFB08B115F052FBFEF76CFEFBF74EFAF4
:1000E000FFF75EF9002830D03E4890F8371090F8BE
:1000F000362090F835003B4B1B7ACDE90030CDE936
:1001000002213848C379827937A104A8FCF784FC1E
:1001100004A8F6F7CAF90446214604A80AF0DAFB57
:10012000002004900590069007902E488379C279AC
:1001300034A104A8FCF770FC04A8F6F7B6F904464D
:10014000214604A815F058FB21E0264890F8371006
:1001500090F8362090F83500224B1B7ACDE900301C
:10016000CDE902211F48C37982791FA104A8FCF7B9
:1001700053FC04A8F6F799F90446214604A815F0A3
:100180003BFB162123A00AF0A5FBFBF7F7F915F0BE
:10019000EDFAFEF7EBFD1348407966281DD09FED80
:1001A000210A2148F9F71EFC9FED1E0A1F48F9F7A6
:1001B00019FC02200AF03EF91D4802F0EFFC1D4A2E
:1001C0001DA16420FAF7B6FB1F49012002F0FAFFD7
:1001D00001211848FAF788FB02E001201B4908704A
:1001E00008B010BD785300202530325825303258E1
:1001F0002530325825303258253032582530325883
:100200000000000046554E5F2530325825303258E8
:10021000000000002A2A2A2A2A2A2A2A2A2A2A2AE6
:100220002A2A00000000D0422454002078540020E4
:10023000B0670400510203006170705F646574650B
:1002400063745F4C52000000197A020006400020DF
:1002500070B50949002002F0C9FE04460649012094
:1002600002F0C4FE0546012C01D1012D02D0024846
:1002700002F094FC70BD0000B067040010B50548A2
:1002800002F0B4FC0448FAF7BFFB00200AF0D2F8F1
:1002900010BD0000B067040051020300B4B0064670
:1002A0000F461446224639463046F8F757F90120E2
:1002B0002D4981F854000846806C40F004008864A1
:1002C0001C2129482C30F6F7E5F8012E0CD06FF4EC
:1002D0008050304478B1B0F5405F23D06FF4405186
:1002E0000844002830D10DE01C2220A11E482C30EB
:1002F000F6F7B7F834E01C2222A11B482C30F6F7A1
:10030000B0F82DE02546D5E9003000F10D0224A11A
:1003100002A8FCF781FB1C2202A913482C30F6F737
:10032000A0F81DE0254628680090686800F10D03DC
:100330001EA102A8AA68FCF76FFB1C2202A90A48AA
:100340002C30F6F78EF80BE03A461DA102A8FCF718
:1003500063FB1C2202A904482C30F6F782F800BF88
:1003600000BFFCF799FB0000A0FF002053443A2097
:10037000415353455254494F4E204641494C454400
:100380000D0A000053443A20494E56414C4944203E
:100390004D454D4F5259204143434553530D0A009B
:1003A000663A25732C6C3A25750D0A00653A257559
:1003B0002C663A25732C6C3A25750D0A0000000056
:1003C000554E4B4E4F574E204641554C5420307899
:1003D000253038580A000000014840797047000075
:1003E0003C3F002010B50A4A0AA16420FAF7A2FA9D
:1003F0000B49A220F6F7FCFE0A4A0BA14EF660203C
:10040000FAF798FA0B49012002F0DCFE10BD00005B
:10041000390403006170705F67616D650000000062
:10042000713F0300FDEE02004175746F4F757467F4
:10043000616D65007198030070B5002400256B485C
:100440000078002804DD69480078401E674908707C
:100450006748007810B101287CD144E06348C07837
:10046000002835D06349002002F0C0FD04466149F0
:10047000012002F0BBFD054634B92DB901205C49CD
:1004800008705A4948711DE0012C01D1012D19D085
:10049000584802F083FB58480078401CC0B25649C7
:1004A0000870C8280EDB002008705049C8705148F9
:1004B00002F09CFB51A10920F7F732FC00215648BD
:1004C000FAF712FA4948007910B10020474908713B
:1004D00046480078002805DD5048007910B100201A
:1004E00000F0E4F880E04D48007920B30AF0ECF920
:1004F00010B33E48007888B9012000F0D7F83E4894
:100500000078401CC0B23C49087064280DDB002014
:10051000087043A10920F7F703FC06E0364800788D
:10052000002802DD0020344908703048407810B1BE
:1005300000202E49487004E02C484078401C2B498C
:10054000487015F053F930B928488078401C274985
:10055000887006E03DE02548807810B100202349EE
:1005600088702248C07838B120488078322803DC6F
:100570001E48407864282BDD1C488078322803DD33
:100580002DA10920F7F7CCFB18484078642803DD3B
:1005900034A10920F7F7C4FB00201749087014495B
:1005A00008701249C870887048704871114802F08C
:1005B0001DFB1A48007910B1002000F077F80020E8
:1005C0003449087015F010F800211348FAF78CF937
:1005D0000AE00020064908700449C87088700021AC
:1005E0000D48FAF781F900BF00BF70BD3C3F002005
:1005F000553F002030660400543F002073686F654B
:100600007320696E746F2067616D65206D6F64651E
:10061000206661696C0000003904030078530020F3
:100620006E6F206765742072696768742073686FE5
:100630006573206461746100496E2067616D652097
:100640006D6F64652C636C69656E74206469736397
:100650006F6E6E746564206C6F6E672074696D6573
:1006600000000000496E2067616D65206D6F646554
:100670002C72696768742073686F6573206469738E
:10068000636F6E6E746564206C6F6E672074696D45
:1006900065000000493F0020034800781E2802D072
:1006A0001E200149087070473C3F002038B50446C1
:1006B000009401236A46A2210020F7F74BF838BDC9
:1006C00070B50446002500260C49002002F08EFC7F
:1006D00005460A49012002F089FC06465DB956B973
:1006E000002002F0CBFA20602068012801DB012005
:1006F00070BD0020FCE70020FAE70000B0670400AE
:1007000010B504460123094AA1210020F7F722F879
:100710000748007840B9022C06DB05480470012325
:10072000024AA121F7F716F810BD00001D3F002076
:10073000F83E002010B50123024AA1210248F7F734
:1007400009F810BD1C3F0020D43E0020014800786D
:1007500070470000D13E00200148B0F9000070470A
:10076000D23E00200148007870470000D03E0020B3
:1007700010B50249A120F6F70FFF10BDA1420300FA
:1007800010B513480078002820DD1149087800EBE7
:10079000D0714910A0EB410121B10E490720F8F7B3
:1007A00093FE04E04FF07F410720F8F78DFE0848E4
:1007B0000078142805DB0020054908700720F8F7A9
:1007C000B3FE03480078401C0149087010BD0000CA
:1007D00041400020AF0000FF10B5034A03A14FF4D1
:1007E0007A70FAF7A7F810BD499802004C6F73733E
:1007F0005061636B0000000030B58BB000251821FC
:1008000001A8F5F747FE0AF00DF800283BD01F4875
:100810000078012837D0FFF7DFFD78BB002002F019
:100820002DFA05B200242BE001AA2146002002F097
:100830001BFABDF81000ADF81C00BDF81200ADF8B1
:100840001E00BDF81400ADF82000BDF80400ADF89E
:100850002400BDF80600ADF82600BDF80800ADF88C
:100860002800BDF9281007A804F010FF012806D1C0
:1008700007484069401C0649486103E003E0641CE6
:10088000AC42D1DB00BF0BB030BD0000203F0020E8
:100890007853002070B5002512480468124800689B
:1008A000844201D204F180740F480068201A0F4975
:1008B000096808440D49086008460068C50BB4F192
:1008C000807F04D9A4F180700749086001E00648E0
:1008D0000460B5F5616F04D3002004490860FFF798
:1008E00059F970BD04B50040C43F0020C03F00204E
:1008F00010B5034A03A14FF47A70FAF71BF810BD44
:10090000950803006D6174685F486F7572000000A0
:10091000C0EB00114904014A11607047C03F00203C
:1009200010B50A4A0AA10020FAF704F80949A620DE
:10093000F6F75EFC0849A620F6F72EFE074A08A146
:100940004FF4FA70F9F7F6FF10BD00006D090300CF
:100950006F746100093F03001D420300590B03003F
:100960006F74615F666C61736800000010B58CB0D5
:10097000002007906348007820B1012861D0022848
:1009800077D17AE060480079002815DD5F4800786B
:10099000012855D15B49087009F04EFF0EF0A7FA07
:1009A00042F210715A48FAF753F8012307AAA62118
:1009B0000020F6F7F3FC43E05648006801283FD1D9
:1009C0005548007801283BD100205249086052491F
:1009D000087014F00BFF10B114F0D0FE01E0FEF728
:1009E000E9F905A8F7F718FF0020089009900A9088
:1009F0000B909DF819009DF818109DF817209DF890
:100A00001630CDE90032CDE902109DF815309DF881
:100A1000142042A108A8FBF7FFFF08A8F5F745FD41
:100A20000446214608A814F0E7FE14F09FFE0120BA
:100A3000344908704FF4FA613548FAF709F800BFF5
:100A40005CE031480079002805DD00202F4908705E
:100A50002C49087010E014F0C9FE58B9FEF786F969
:100A600042F210712A48F9F7F3FF02202549087075
:100A700002E03BE014F082FE40E014F0B7FE10B15B
:100A800000202049087000212148F9F7E1FFFEF716
:100A900091F90020089009900A900B901A4890F85C
:100AA000371090F8362090F83500174B1B7ACDE9B7
:100AB0000030CDE902211448C379827918A108A831
:100AC000FBF7AAFF08A8F5F7F0FC0446214608A8A2
:100AD00014F092FE19A10E20F7F722F914F046FE49
:100AE000FEF744F900200749087007E00020054997
:100AF000087000210648F9F7ABFF00BF00BF0CB03B
:100B000010BD0000843F0020785300205C3F00208F
:100B10006D090300583F00205E3F002046554E5FA0
:100B20002530325825303258253032582530325849
:100B3000253032582530325800000000616476209C
:100B4000646973636F6E6E746564206F766572207E
:100B500074696D650000000010B517480078012821
:100B600022D1F8F70DFCF7F783FD18B113A10E2081
:100B7000F7F7D6F8242216491648F5F772FC00203C
:100B800015494876F7F7BAFC18B114A10E20F7F70B
:100B9000C7F8F7F78BFC18B117A10E20F7F7C0F8CC
:100BA00002200549087006E003480078022802D1B7
:100BB00004200EF09BFE10BD5D3F00206F7461208D
:100BC000736176652073746570206661696C0000DE
:100BD00024500020E4530020085400206F7461204A
:100BE0007361766520696E666F726D6174696F6E90
:100BF000206661696C0000006F7461207361766526
:100C0000206261636B206661696C000001480078B6
:100C1000704700005C3F002010B5064A06A1642022
:100C2000F9F788FE074A08A14FF47A70F9F782FEB7
:100C300010BD0000A9EF0200426174446973706145
:100C40006C790000ADF10200426174446973706117
:100C50006C795F4E0000000010B50C4A0CA16420B6
:100C6000F9F768FE104A11A16420F9F763FE134AF0
:100C700013A14FF4FA70F9F75DFE1449B120F6F7AD
:100C8000B7FA1349B120F6F787FC10BD990D0300A0
:100C90006170705F706169725F52696768745F50FC
:100CA000726F636573730000D50C03006170705F31
:100CB000706169725F4C6566740000008107030013
:100CC000426C696E6B5F666C616700009144030063
:100CD000A145030030B589B008F08CFF08B909B010
:100CE00030BD2348007900B9F9E709F04BFA044612
:100CF0002048007800282DDD09F0E6FD10B109F04C
:100D00009BFD27E000F0C0F80020059006900790BA
:100D10000890174890F8371090F8362090F8350072
:100D2000134B1B7ACDE90030CDE902211048C3797D
:100D3000827911A105A8FBF76FFE05A8F5F7B5FBB1
:100D40000546294605A809F0C5FD10B90020094946
:100D5000087000BF0F480078002807DD012C05D17E
:100D600000200C4908700720F8F7DEFB00BFB6E74B
:100D7000785300204040002025303258253032582A
:100D800025303258253032582530325825303258E7
:100D9000000000004140002070B508F02BFF00B9B2
:100DA00070BD2E48007900B1FAE709F0EBF904466E
:100DB0002B48007810B101284CD115E0022C01D04D
:100DC000032C10D12748FDF743FFFAF7D7FB0C217E
:100DD00025A009F07FFDFAF7ADFB0120204908703E
:100DE00000202449087035E0022C0ED0032C0CD0D2
:100DF000FAF7C4FB00201A4908700720F8F794FBA3
:100E000009F062FD08B109F017FD1A4800780028C2
:100E10001ADD002017490870012011490870114897
:100E2000FDF72AFF09F050FD08B109F005FD8BDF41
:100E300005461148F5F739FB064631460E4809F0DC
:100E400049FDFAF777FB00BF09F03EFD08B1FEF758
:100E5000ADFA00BF00BF00BFA2E70000785300203A
:100E60004240002009A402002A2A2A2A2A2A2A2AE1
:100E70002A2A2A003F40002000550020014800781F
:100E8000704700004040002010B543201D4981F804
:100E900028000846C06A1C4908611A48008E8882EA
:100EA000184890F82800887500200DE01549891D24
:100EB0000A5C1549091D0A54124932310A5C12496B
:100EC0000A310A54411CC8B20628EFDBF7F7EEFAE4
:100ED00018B10EA10C20F6F723FFF7F7EEF818B1C2
:100EE00010A10C20F6F71CFF1C2106480C30F5F76A
:100EF000D1FAF7F703FB18B110A10C20F6F710FF99
:100F000010BD000078530020085400207061697201
:100F10002073617665206261636B7570206661691C
:100F20006C0000007061697220636C6561722073EF
:100F3000746570206661696C00000000466C617326
:100F4000685F53617665496E666F6D6174696F6E37
:100F5000206661696C00000010B50C48407E401CA2
:100F60000A4948760A4A0BA14FF47A70F9F7E2FC75
:100F70000B49AE20F6F73CF90A49B220F6F738F9EA
:100F8000094A0AA16420F9F7D5FC10BD08540020D5
:100F9000C50F03006170705F73616665000000003B
:100FA000914303008543030045EF02006170705FC9
:100FB000424C455F4C45444F4E5F505552504C4556
:100FC0000000000000B58BB01E48007E002812DD36
:100FD0001D480078401C1C490870084600783C28D1
:100FE00009DB002017490876F7F760FA18B117A156
:100FF0000D20F6F795FE1348407E012820DD2821BC
:1010000001A8F5F747FA282101A8F5F743FA154892
:10101000007930B10B48427E13A101A8FBF7FCFC1C
:1010200005E00848427E16A101A8FBF7F5FC01A9DE
:101030000D20F6F775FE10B900200249487600BF72
:101040000BB000BD08540020F93F002073617665A5
:10105000204572725374617274436E7420666169C4
:101060006C000000785300206C6566742073686F14
:10107000657320726573746172743A2564000000B0
:1010800072696768742073686F6573207265737422
:101090006172743A25640000014602290FD10A48A2
:1010A000007810B1012807D104E00120064A107031
:1010B000002070470020FCE700BF00BF01E00120D6
:1010C000F7E700BF0120F4E75D3F002001484069D9
:1010D0007047000078530020014880697047000085
:1010E0007853002010B50E4A0EA16420F9F722FCB7
:1010F0001049A520F6F77CF80F4A10A16420F9F7F3
:1011000019FC1349A520F6F747FA1249012002F00D
:1011100059F8114A11A16420F9F70CFC10BD000028
:10112000B1130300737465705F5265616C53656E33
:1011300064000000DD3F03006D11030073746570EF
:101140005F5265616C436F6E6E65637400000000F2
:1011500051420300A5340400F90703006D6174686F
:101160005F4461696C7953746570000038B5002084
:101170000090002400255048007820B101281CD0A0
:1011800002287DD150E04D480078012808D14A4915
:10119000087000204A4908704A4801F0FFFC0BE043
:1011A00049480078002807DD0020474908700123DE
:1011B000424AA521F6F7CEFA7CE04249002001F030
:1011C00015FF04463F49012001F010FF054684B990
:1011D0007DB90220384908703C4840693C490860A4
:1011E00000203C4908603C49088001203B490870C8
:1011F00019E0012C01D1012D15D0324801F0CEFCAF
:101200002F480078401C2E490870084600781428A2
:1012100009DB2C4801F0EAFC002027490870274927
:1012200008702E49087045E02B480088401C2A4968
:10123000088008460088B0F5167F10DB0020088083
:10124000009001236A46A521F6F784FA1D4801F0B3
:10125000CDFC0020214908701749087015E01A4894
:101260000078002804DD18480078401E16490870F0
:101270001548007848B90120009001236A4600E033
:1012800010E0A5210020F6F765FA0C48007840B977
:101290000020124908700B4801F0A8FC0020064904
:1012A000087007E00020054908700C4908700249E1
:1012B000087000BF00BF38BD383F0020303F00201D
:1012C000393F0020106604002C3F00207853002096
:1012D000243F0020283F00202E3F0020203F0020F8
:1012E0001CB52F480078012858D1002000900190AB
:1012F000002401222146641C0DF801202948406980
:1013000029490968401A020E2146641C0DF8012083
:101310002448406924490968401AC0F3074221461D
:10132000641C0DF801201F48808A1F490988401A53
:10133000C0F307222146641C0DF801201948007DE6
:1013400019490978401AC2B22146641C0DF80120DF
:1013500016480068020E2146641C0DF8012013484F
:101360000068C0F307422146641C0DF801200F48B5
:101370000088C0F307222046611CCCB20DF8002083
:101380000A4802782046611CCCB20DF800202346A2
:101390006A46A5210020F6F701F800BF1CBD000039
:1013A000203F002078530020243F0020283F0020C9
:1013B00010B50448007900B110BDFFF791FF00BFE0
:1013C000FAE700007853002003480078012800D194
:1013D00070470020FCE70000203F002010B50249C4
:1013E000AB20F5F705FF10BD8D40030010B5024896
:1013F00006F0AAFA10BD0000E04A002010B503462E
:101400000C460AB9072010BD19684A61012C01D1A8
:10141000012000E0002008610020F4E738B51348FF
:1014200000680090082358221149124800680DF006
:1014300089F804460CB1204638BD0F4A69460F486A
:1014400006F088FA04460CB12046F5E701210B4866
:1014500006F0F2FA01230A4A1946084806F046FA4D
:101460000120084908702046E6E70000F86A0400F9
:1014700048940020E86A040047380400E04A00204D
:10148000FFFF7F00EC4A00202DE9F04106460D46A3
:1014900017463446207F10B10020BDE8F081A761D7
:1014A00008F066FC401941F10001C4E9020120691D
:1014B00000B125612146002014F064FEEDE770B50F
:1014C00004462546002028772946012014F05AFEBC
:1014D00070BD10B50446204612F04CFC10BD000053
:1014E00070B5044625460E488068B0B1ADB9FCF72A
:1014F00095FE06460A4800680A49086008484068A0
:101500004FF0E021C1F804010020054988601EB9B0
:1015100000BF62B600BF00BF00BF00BF70BD0000CB
:101520003094002000E100E0F8B505460C4617466F
:101530002088001DB84201D90C20F8BD684679DF2B
:10154000064600BF304600B1F7E700BF0320218800
:1015500068542088401C20801920218868542088E5
:10156000401C208020884119BDF8000014F04BFE7B
:101570002188084420800020DFE710B541EC100BE3
:10158000FBF732FD51EC100B10BD2DE9F0412DEDB4
:10159000028B04460E4617461D46B0EE408AB0EE5A
:1015A000000A86ED000A95ED020A20EE080A86ED93
:1015B000010A95ED010AF1EE480A20EE200A86EDB7
:1015C000020A95ED020AF1EE480A20EE200A86EDA5
:1015D000030AB0EE000A86ED040A95ED000A20EE3B
:1015E000080A86ED050A95ED010A20EE080A86ED47
:1015F000060A95ED000AF1EE480A20EE200A86ED73
:10160000070AB0EE000A86ED080A394630460AF0AD
:10161000EBF824213046F4F73DFF94ED010A20EE6B
:10162000080AD5ED020A20EE200AD4ED000AB0EE39
:10163000001A01EE200AD4ED020A60EE880A95ED48
:10164000011A00EEC10A86ED000A94ED010AF0EEDF
:10165000000A20EE200AD4ED000A60EE880A95ED1B
:10166000021A00EEC10AD4ED020A60EE880A95ED76
:10167000001A00EE810A86ED010A94ED000A20EEC0
:10168000080AD5ED010A20EE200AD4ED020AB0EED8
:10169000001A01EE200AD4ED010A60EE880A95EDE9
:1016A000001A00EEC10A86ED020A94ED040A20EE4B
:1016B000080AD5ED020A20EE200AD4ED030AB0EEA6
:1016C000001A01EE200AD4ED050A60EE880A95EDB5
:1016D000011A00EEC10A86ED030A94ED040AF0EE49
:1016E000000A20EE200AD4ED030A60EE880A95ED88
:1016F000021A00EEC10AD4ED050A60EE880A95EDE3
:10170000001A00EE810A86ED040A94ED030A20EE29
:10171000080AD5ED010A20EE200AD4ED050AB0EE44
:10172000001A01EE200AD4ED040A60EE880A95ED55
:10173000001A00EEC10A86ED050A94ED070A20EEB4
:10174000080AD5ED020A20EE200AD4ED060AB0EE12
:10175000001A01EE200AD4ED080A60EE880A95ED21
:10176000011A00EEC10A86ED060A94ED070AF0EEB2
:10177000000A20EE200AD4ED060A60EE880A95EDF4
:10178000021A00EEC10AD4ED080A60EE880A95ED4F
:10179000001A00EE810A86ED070A94ED060A20EE93
:1017A000080AD5ED010A20EE200AD4ED080AB0EEB1
:1017B000001A01EE200AD4ED070A60EE880A95EDC2
:1017C000001A00EEC10A86ED080A22463946304664
:1017D0000CF0D9FBBDEC028BBDE8F0812DE9F041A6
:1017E0000446501E34F9105034F9106031F910706D
:1017F00031F910C0132018E034F91080A84501DD3C
:1018000034F9105034F91080B04501DA34F9106021
:1018100031F91080B84501DD31F9107031F91080CF
:10182000E04501DA31F910C0401EC2F114088045CC
:10183000E2DDF018A84203DB0CEB0300B84202DA49
:101840000120BDE8F0810020FBE72DE9F0410446CE
:101850000F46154615B90E20BDE8F081002028601E
:1018600000BF0CB90E20F7E700BF00BF206808B921
:101870000E20F1E700BF00BFE088C11700EB9171B7
:101880008910A0EB810109B10720E5E700BF3846C8
:1018900000F0DEFAC6B2142E01D10520DCE7207973
:1018A000B04201DC0420D7E7E188206806FB010094
:1018B00028600020D0E72DE9FC4105468846164601
:1018C000002437880020308095F82D0058B13A4622
:1018D0003146404600F08AFB044600BF204608B16E
:1018E000BDE8FC8100BFA87850B13A463146404679
:1018F000FFF71AFE044600BF204600B1F0E700BF24
:10190000E87860B1E97848B23B463246414606F095
:101910003EFC044600BF204600B1E1E700BF686816
:1019200068B1696891F900003B463246414614F0BF
:1019300049FC044600BF204600B1D1E700BF28891A
:1019400000280EDD43460622022105F10800CDE9FC
:10195000006714F0CBFC044600BF204600B1BFE78F
:1019600000BF288A00280EDD43460722032105F127
:101970001000CDE9006714F0B9FC044600BF204612
:1019800000B1ADE700BF288B00280EDD43461522CD
:10199000142105F11800CDE9006714F0A7FC0446F6
:1019A00000BF204600B19BE700BF286A58B13B4604
:1019B00032464146286A03F044FA044600BF2046F6
:1019C00000B18DE700BF686A58B13B4632464146D8
:1019D000686A0BF0D7F9044600BF204600B17FE7E4
:1019E00000BF95F82C0000280BDD3B4632464146EF
:1019F000284613F0F3FB044600BF204600B16FE712
:101A000000BF287858B13B463246414628460CF084
:101A10006FFB044600BF204600B161E700BF2046CF
:101A20005EE72DE9F84306468846154600200090FB
:101A30000DB9BDE8F88309236A464146304600F0F7
:101A40002BF80446BDF800003718BDF8000068B157
:101A500064B12846F4F729FDA04207D12246394651
:101A60002846F4F737FD08B90120E2E70020E0E757
:101A7000F8B504460E461546002000902B466A46EF
:101A80003146204600F008F807460FB90020F8BD9F
:101A9000BDF800002044FAE7F0B504460D461E46A6
:101AA00004B10AB90020F0BD002103E0605C401CD5
:101AB000084481B2481CA84206DA10888842F5DC46
:101AC000481C205CB042F1D1A94201DB0020EAE7CA
:101AD000881C87B2605C10B1605C401E00E0002092
:101AE00083B213B1F818A84201DD0020DBE71780AC
:101AF0001846D8E780F83010704770B504460D4698
:101B000005B10CB90E2070BD05F1780003F0B1F8F5
:101B100008B90720F7E70020A0702C2205F1780112
:101B2000201DF4F79EFC002084F83000D5F8A400B6
:101B30006063D5F8A800A0634FF6FF70A4F82404F2
:101B400004F58260C4F82004002140F22C40C4F85F
:101B50002614A4F82A140155207810B9FF2084F81F
:101B6000540004F15500C4F810042046FDF767F84E
:101B700040F21441085304F2144204F1550128467E
:101B8000FFF799FE064600BF304600B1BBE700BF35
:101B900004F231204FF4836108512046FDF74FF8DD
:101BA000A4F81C044FF48360015904F21C4205F1AF
:101BB0003C00FFF780FE064600BF304600B1A2E7BA
:101BC00000BF012151200155208B81B248200153D3
:101BD000012084F83C0000212164502001556169F6
:101BE000616404F13C02002104F1540072DF0646F6
:101BF00000BF304600B186E700BF012020703046AC
:101C000081E770B504460D462E462088102804D082
:101C1000112807D026280FD109E0214630460FF0C1
:101C200083FD0AE0214630460FF0F9FE05E021462B
:101C3000304610F0D7F800E000BF00BF70BD70B5AF
:101C400004460E46207808B9082070BDA670002111
:101C500040F22C40C4F82614A4F82A140155A079A7
:101C600010B1A078012809D0E07910B1A07801283E
:101C700004D0E07970B1A07802280BD1606B30B14C
:101C8000012084F82D040820616B884702E00020C1
:101C900084F82D0431462046FCF781FFA070606B6C
:101CA000A0B1A078032802D0A07804280ED16079D2
:101CB00060B194F82E0448B9002084F83004012063
:101CC00084F82F040720616B884702E0002084F825
:101CD0002F04182104F13C00F4F7DCFB012084F808
:101CE0003C0004F12C0010F08FFB20B194F82C1074
:101CF0005120015502E001215120015594F82400A2
:101D000060B104F1280010F07FFB20B194F8281096
:101D10005220015502E0012152200155002150209E
:101D20000155A078052824D2DFE800F01F030A112E
:101D3000180004F13C01204613F04EFB054619E063
:101D400004F13C01204613F02FFB054612E004F19C
:101D50003C01204613F052FB05460BE004F13C0128
:101D6000204613F079FB054604E0002084F831009A
:101D700000E000BF00BFA07898B104F13C0204F17C
:101D80005400D4F8201472DF05460DB128465CE7F4
:101D900094F8301094F8540073DF05460DB12846CE
:101DA00053E7606B18B194F83100616B88470020ED
:101DB0004BE700002DE9F041044600BF14B90E20A6
:101DC000BDE8F08100BF1C2221461C48F4F749FB06
:101DD0001B481A490860206860B120687ADF054610
:101DE0000DB12846ECE7164821680A680260496888
:101DF000416005E012487BDF05460DB12846DFE76C
:101E0000002617E006EB86000E4901EB800700BFB5
:101E10004FF6FF70388000BF0B4800EB461078602B
:101E20000A4A0021381DFFF7E9FA05460DB10320E3
:101E3000C6E7761C002EE5D00020C1E74C930020B9
:101E4000A64A002038930020189300201562040051
:101E500010B50446204600F01BF808B1204610BD1E
:101E60001420FCE770B504460025204600F010F869
:101E700050B1214605480CF0C0FB06460EB10220C9
:101E800000E00120054600BF284670BDA492002056
:101E900010B50446142C01DB002010BD2146024879
:101EA0000CF0ABFBF9E700009C92002010B5044653
:101EB00000BF0CB90E2010BD00BF00BF064800785F
:101EC000012801D00820F6E700BF04480168204639
:101ED00011F0D2FBEFE70000A44A0020984A00204E
:101EE0000146002200BF09B90E20704700BF00BFA5
:101EF000086808B90E20F8E700BF00BF486808B9B5
:101F00000E20F2E700BF0020064B18600120064BB0
:101F10001870064B08681860054B48681860104632
:101F2000E3E70000A04A0020A44A0020984A0020CD
:101F30009C4A002070B504460D4600BF04B970BD30
:101F400000BF00BF05B9FAE700BF00BF1448007822
:101F5000012800D0F3E700BF2E462088112815D0B5
:101F6000302804D0322807D0332814D109E0211DAD
:101F700030460FF043FE0FE0211D30460FF078FA97
:101F80000AE0211D30460FF089FC05E0211D304696
:101F90000FF038FD00E000BF00BF00BFCFE700003A
:101FA000A44A002070B504460D4600BF0CB90E20AF
:101FB00070BD00BF00BF0B480078012801D0082089
:101FC000F6E700BF0848006808B90820F0E794F871
:101FD000C80208B11120EBE72946204603F030FF84
:101FE000E6E70000A44A0020A04A00202DE9FC41B9
:101FF00005460C46174620880930B84202D90C2005
:10200000BDE8FC8168466DDF064600BF304600B182
:10201000F6E700BF0820218868542088401C2080F3
:102020001B20218868542088401C20802088284458
:10203000DDF801100160BDF8051081802088801D49
:1020400020809DF80000400818B9002021886854BD
:1020500002E00120218868542088401C2080002054
:10206000CEE7000070B50CF099FF044600BF204693
:1020700000B170BD00BF00BF084D28464FF0030CF3
:1020800000DF00BF044600BF204600B1F1E700BFFB
:102090000CF09EFF04462046EBE70000CC940020A5
:1020A000014600BF09B90E20704700BF014801601A
:1020B0000020F9E7144B002010B54FF0FF3100204D
:1020C0003DDF044600BF204600B110BD00BFB12176
:1020D00000203CDF044600BF204600B1F5E700BF0A
:1020E000044841690120884702200DF0FFFB0020D1
:1020F000EBE70000B094002010B505480068416986
:1021000000208847FFF7D8FF0446204610BD000096
:10211000144B002010B588B0044620216846F4F71F
:10212000B9F90320ADF8000020788DF802009DF881
:102130000D0020F0200020308DF80D009DF80D00DE
:1021400020F0080008308DF80D0001208DF81000F7
:102150008DF80C001720ADF8040001208DF8130055
:102160008DF812008DF811006088A21D694602F0FA
:1021700097FB08B010BD000030B585B00546244B74
:102180000FCB8DE80F0000BF15B90E2005B030BD94
:1021900000BF4FF6FF701F49888028684861002003
:1021A00008760846406908B91B4848611948FFF796
:1021B00077FF044600BF204600B1E7E700BF00BF3D
:1021C00001208DF812004FF65960ADF8100000BFE5
:1021D000104A921C04A90120A8DF044600BF204633
:1021E00000B1D3E700BF0B49684662DF044600BF79
:1021F000204600B1CAE700BF0648FFF78BFF044640
:1022000000BF204600B1C1E700BF0020BEE70000CC
:10221000B46B0400B0940020A17D030070B50446A7
:102220000D4600BF04B970BD00BF2088102806D03D
:10223000112808D051280AD0532810D10BE020468D
:102240000FF068FA0CE020460FF0CEFB08E02046C5
:102250000FF016FD04E020460FF06CFC00E000BF1C
:1022600000BF00BFDFE7000070B504460426207BF6
:10227000012802D0022822D109E005F093FD05468D
:102280000DB9012602E0112D00D1062619E0607B70
:10229000142801DC607B08B905260FE0627B04F19D
:1022A0000E011248F4F7DDF8607B1049091F8861C0
:1022B000084613F0FFF8054605B9012601E002269D
:1022C00000BF00BF012E0FD0207B314600F058F830
:1022D000054625B10648006841690320884704483F
:1022E000006841690220884770BD0000DC9400202E
:1022F000144B002070B505460E4600BF1E4800680E
:1023000020B11D48406808B1012000E0002000B95C
:1023100070BD00BF184800F1080142682846904788
:10232000044600BF082C24D07CB90020134909685A
:1023300048760121022000F023F80446CCB10F4872
:10234000006841690320884713E000200B490968B1
:1023500048760621022000F013F8044624B107480D
:1023600000684169032088470448006841690220E9
:10237000884700BFCCE70000CC940020144B00201D
:10238000F0B587B004460D46032700200190029067
:10239000039004900320069020208DF814008DF8FF
:1023A00015408DF816500E48C088ADF80400022084
:1023B0008DF806000020ADF8080006A8039005A8D7
:1023C00004900749888801A9AEDF064626B9BDF802
:1023D0001800032800D00C26304607B0F0BD0000DE
:1023E000B094002030B1012805D0022804D0032881
:1023F00007D102E006E005E004E000BF002100BFD5
:1024000000E000BF00BF70472DE9F04104460F46D1
:10241000A6883046FFF726FD0546012D03D020464D
:1024200000F0ACF818B120460EF0FAFE08E0022DDC
:1024300002D020881D2803D1002120460EF0FCFD8B
:10244000BDE8F0812DE9F04104460F46A6882088BA
:10245000102806D0112819D019283FD01A284AD19F
:1024600018E011F0BBF8304611F094F830B900BF15
:1024700022A2F0210420F3F7CDFE06E0E07B022843
:1024800003D131462C480CF0C7F834E0304611F047
:10249000C9F830E0207A0509042D01DB012000E0B5
:1024A00000200246314624480C3005F061FE032D21
:1024B00001DB012000E00020024631461E480830C2
:1024C00005F056FE022D01DB012000E0002002464F
:1024D00031461948001D05F04BFE0CE0207A48B942
:1024E000607AC0F3C0052A46314613480C3005F027
:1024F0003FFE00BF00BF00BFBDE8F0812E2E5C2E66
:102500002E5C2E2E5C2E2E5C2E2E5C2E2E5C636F8F
:102510006D706F6E656E74735C626C655C636F6D1D
:102520006D6F6E5C626C655F636F6E6E5F7374611E
:1025300074652E6300000000A492002070B504466C
:102540000D462088102806D0112808D012280ED059
:10255000502810D107E020460FF06AF80CE0204622
:102560000FF029FA08E020460FF06EFC04E0204648
:102570000FF046F800E000BF00BF70BD01460888BC
:10258000262801D1012070470020FCE710B5002467
:1025900008E0074850F8240018B1054951F8240014
:1025A0008047641C034800788442F2DB10BD0000C1
:1025B000488200204848002010B5002408E0074861
:1025C00050F8240018B1054951F824008047641CD4
:1025D000034800788442F2DB10BD000054820020E2
:1025E000494800202DE9F04107460C46207820B1EB
:1025F000012824D0022829D127E0618804F10E02A5
:10260000384600F035F8054600BF2E4636B100BF0B
:1026100010A275213046F3F7FDFD00BF00BF38461C
:1026200000F02EF9054600BF2E4636B100BF09A2C4
:1026300078213046F3F7EEFD00BF00BF06E0A18928
:102640000A4AA0681268904700E000BF00BFBDE8DA
:10265000F08100002E2E5C2E2E5C2E2E5C626C65AE
:102660005F6366675C686F73742E63003C42002092
:1026700070B504460E46154600BF0CB90E2070BD5D
:1026800000BF26812DB16988A18128886081A98831
:10269000E1813146A0690CF0EBF8F0E770B586B047
:1026A00004460D461A4B0FCB01AE0FC600BF14B93E
:1026B0000E2006B070BD00BF00BF0DB90E20F8E7B8
:1026C00000BF00BFA86808B90E20F2E700BFE11DF7
:1026D00001A862DF064600BF304600B1E9E700BF4F
:1026E000E0798DF816000120ADF814004FF6FF7068
:1026F0002081286820616868606100206081002175
:10270000E181A868A06105A8FFF7D0FBD1E7000030
:10271000A869040070B586B005460E46344604B17B
:102720000DB906B070BD20894FF6FF71884203D005
:102730002089A988884200D0F3E72888112806D08C
:10274000392816D1294620460FF00AFA12E0A88847
:10275000218988420CD1206950B102208DF80400F3
:102760004FF6FF70208101A920462269904700BFE3
:1027700000E000BF00BF00BFD3E770B586B00546DC
:102780000C46142101A8F3F785FE04F10E0620780B
:1027900000283AD1A088012837D1A079E979884268
:1027A00033D1002022E000EBC00136F811100229DD
:1027B00002D0032917D107E000EBC00106EB41016D
:1027C0000A89ADF816200FE000EBC00106EB4101CD
:1027D0000989ADF8121000EBC00106EB41014A89EE
:1027E000ADF8142000E000BF00BF401C217A8142F8
:1027F000D9D8286948B16088ADF8060000208DF866
:10280000040001A928462A69904706B070BD00005F
:1028100070B588B004460E46154600BF14B90E20A8
:1028200008B070BD00BF20216846F3F733FEB62D17
:1028300001DD0720F4E720894FF6FF71884201D1BE
:102840000820EDE701208DF800000C480290039469
:10285000E189ADF81210ADF816500021ADF8141052
:10286000069602208DF8100001218DF811102289A2
:102870006946A0690CF026F8D2E70000B99A030077
:1028800010B5044600BF0CB90E2010BD00BF208952
:102890004FF6FF71884201D0A08908B90820F4E7FB
:1028A0000121204601F0CCFFEFE72DE9F04186B091
:1028B0000446884617461D4600BF1CB90E2006B0C8
:1028C000BDE8F08100BF01AA29466069FEF7BDFF9F
:1028D000064600BF304600B1F1E700BF4FF6FF707B
:1028E000854201D0019808B90520E8E701980078F1
:1028F00008B90820E3E73888B62801DD0720DEE7BD
:1029000000200290039004900590A088ADF8080084
:10291000CDF81480049701208DF80A0002A92846FA
:10292000AEDFCCE770B58EB004460E463E4B0FCB03
:1029300009AD0FC500BF14B90E200EB070BD00BFA9
:1029400000BF0EB90E20F8E700BF3068A061214635
:1029500009A862DF054600BF284600B1EDE700BFC9
:1029600020788DF836000120ADF83400A21C0DA9A6
:10297000A8DF054600BF284600B1DEE700BF2021E2
:1029800001A8F3F787FD0220ADF8040020788DF848
:102990000600B620ADF808000120ADF80A008DF859
:1029A00010009DF8110020F0080008308DF811008B
:1029B0009DF8110020F00400001D8DF81100012089
:1029C0008DF815008DF81600608804F10C0201A93D
:1029D00001F066FF05460DB12846AEE7202101A8AB
:1029E000F3F758FD0320ADF8040020788DF80600B9
:1029F000B620ADF808000120ADF80A008DF81000EF
:102A00009DF8110020F0100010308DF81100012009
:102A10008DF815008DF816008DF817006088221DBE
:102A200001A901F03DFF88E7B869040070B50446CC
:102A30000D4605B104B970BD2E462088102804D07B
:102A4000502807D057280FD109E0214630460EF014
:102A500027FE0AE0214630460FF022FA05E0214623
:102A600030460FF099F800E000BF00BF00BFE2E77A
:102A700010B5002408E0074850F8240018B10549B3
:102A800051F824008047641C034800788442F2DB3C
:102A900010BD0000B07F00200E42002010B50024C1
:102AA00008E0074850F8240018B1054951F82400FF
:102AB0008047641C034800788442F2DB10BD0000AC
:102AC000F07F00200F42002070B50446204613F02E
:102AD00094FB0546C5F3400070BD70B50446204622
:102AE00013F08BFB054605F0010070BD38B50DF005
:102AF00085F9044600BF25463DB100BF15A240F24E
:102B0000BB112846F3F786FB00BF00BF00200090F2
:102B1000694601200DF0A6F8044600BF25463DB1E8
:102B200000BF0CA240F2C1112846F3F773FB00BFAF
:102B300000BF68460DF0F4F8044600BF25463DB1DD
:102B400000BF04A240F2C5112846F3F763FB00BFA3
:102B500000BF38BD2E2E5C2E2E5C2E2E5C626C6566
:102B60005F6366675C686F73742E630010B5002442
:102B700005F044FC401C00B9641E70210648F3F7C0
:102B800089FC0020044981F86E00601C10B94FF0E8
:102B9000FF3010BD0020FCE7AC72002070B5044689
:102BA0000CB9002070BD002509E00F4850F8250041
:102BB000A04203D100F056FB2046F3E76D1C0C2D1C
:102BC000F3DB00250BE0084850F8250030B9064833
:102BD00040F8254000F046FB2046E3E76D1C0C2D35
:102BE000F1DB0020DEE70000AC72002070B5054686
:102BF00015B94FF0FF3070BD00240DE0094850F8C2
:102C00002400A84207D10020064941F8240000F022
:102C100029FB0020EFE7641C0C2CEFDB6FF00100B8
:102C2000E9E70000AC72002010B5002005F0C6FCFA
:102C30000446601C10B94FF0FF3010BD012005F0B4
:102C4000BDFC0446601C10B94FF0FF30F5E7702161
:102C50000448F3F71FFC0020024981F86E0000BF12
:102C6000EBE70000AC72002070B504460D46164636
:102C700032462946204605F00FFD70BD10B50446CA
:102C8000204605F027FD10BD10B5024602B111B96E
:102C90004FF0FF3010BD002067E100EB400303EB75
:102CA000C00313441B7A00EB400404EBC0040C4443
:102CB000247AA34206DD00EB400303EBC003134478
:102CC0001B7A05E000EB400303EBC0030B441B7AC7
:102CD00000EB400404EBC0041444237200EB4003F7
:102CE00003EBC00313445B7900EB400404EBC00426
:102CF0000C446479A34206DD00EB400303EBC00300
:102D000013445B7905E000EB400303EBC0030B4485
:102D10005B7900EB400404EBC0041444637100EBE6
:102D2000400303EBC003D35C00EB400404EBC0049E
:102D30000C5DA34205DD00EB400303EBC003D35C55
:102D400004E000EB400303EBC003CB5C00EB40046A
:102D500004EBC004135500EB400303EBC003134422
:102D60009B7800EB400404EBC0040C44A478A3421D
:102D700006DD00EB400303EBC00313449B7805E042
:102D800000EB400303EBC0030B449B7800EB4004D3
:102D900004EBC0041444A37000EB400303EBC00336
:102DA00013445B7A00EB400404EBC0040C44647AE7
:102DB000A34206DD00EB400303EBC00313445B7A40
:102DC00005E000EB400303EBC0030B445B7A00EB30
:102DD000400404EBC0041444637200EB400303EBB3
:102DE000C00313449B7900EB400404EBC0040C4483
:102DF000A479A34206DD00EB400303EBC0031344B8
:102E00009B7905E000EB400303EBC0030B449B7987
:102E100000EB400404EBC0041444A37100EB400336
:102E200003EBC00313445B7800EB400404EBC004E5
:102E30000C446478A34206DD00EB400303EBC003BF
:102E400013445B7805E000EB400303EBC0030B4445
:102E50005B7800EB400404EBC0041444637000EBA7
:102E6000400303EBC00313449B7A00EB400404EBE4
:102E7000C0040C44A47AA34206DD00EB400303EB3C
:102E8000C00313449B7A05E000EB400303EBC0034F
:102E90000B449B7A00EB400404EBC0041444A3727F
:102EA00000EB400303EBC0031344DB7900EB400469
:102EB00004EBC0040C44E479A34206DD00EB4003BC
:102EC00003EBC0031344DB7905E000EB400303EBA5
:102ED000C0030B44DB7900EB400404EBC004144452
:102EE000E37100EB400303EBC0031344DB7800EB1A
:102EF000400404EBC0040C44E478A34206DD00EB7C
:102F0000400303EBC0031344DB7805E000EB400310
:102F100003EBC0030B44DB7800EB400404EBC0047C
:102F20001444E37000EB400303EBC00313441B792C
:102F300000EB400404EBC0040C442479A34206DDFA
:102F400000EB400303EBC00313441B7905E000EBE7
:102F5000400303EBC0030B441B7900EB400404EB7C
:102F6000C00414442371431CD8B20228FFF695AE66
:102F700000208FE610B502460020137A0C7AA34297
:102F800000D0401C53794C79A34200D0401C1378E8
:102F90000C78A34200D0401C93788C78A34200D0D8
:102FA000401C537A4C7AA34200D0401C93798C7910
:102FB000A34200D0401C53784C78A34200D0401C60
:102FC000937A8C7AA34200D0401CD379CC79A34267
:102FD00000D0401CD378CC78A34200D0401C137999
:102FE0000C79A34200D0401C10BD0000F0B506468D
:102FF0000D460DB1022E01DB0220F0BD29686A6882
:10300000554B03F10B0416B1012E71D14DE00F7A2F
:1030100093F808C0674501DD0220EEE74F7993F889
:1030200005C0674501DD0220E7E70F7893F800C08F
:10303000674501DD0220E0E78F7893F802C067451D
:1030400001DD0220D9E74F7A93F809C0674501DD19
:103050000220D2E78F7993F806C0674501DD022090
:10306000CBE74F7893F801C0674501DD0220C4E744
:103070008F7A93F80AC0674501DD0220BDE7CF795A
:1030800093F807C0674501DD0220B6E7CF7893F8D3
:1030900003C0674501DD0220AFE70F7993F804C054
:1030A000674501DD0220A8E74FE0177A94F808C0D1
:1030B000674501DD0220A0E7577994F805C0674510
:1030C00001DD022099E7177894F800C0674501DD1B
:1030D000022092E7977894F802C0674501DD02204C
:1030E0008BE7577A94F809C0674502DD022084E730
:1030F0002AE0977994F806C0674501DD02207CE755
:10310000577894F801C0674501DD022075E7977A8A
:1031100094F80AC0674501DD02206EE7D77994F87C
:1031200007C0674501DD022067E7D77894F803C040
:10313000674501DD022060E7177994F804C0674510
:1031400001DD022059E700E000BF00BF024F583FF9
:1031500097F86E0000BF50E704730020411C21B9AE
:103160000021174A82F86E1028E0042804D10521B6
:10317000134A82F86E1021E0052804D10321104A79
:1031800082F86E101AE0062804D104210C4A82F855
:103190006E1013E0102804D10721094A82F86E103E
:1031A0000CE01A2806D3411C21B10821044A82F8F8
:1031B0006E1003E00621024A82F86E10704700008C
:1031C000AC72002002460B460BB1022A02DB4FF024
:1031D000FF30704700210BE0114800EBC100406850
:1031E000984204D10E4800F831200020F1E7491C34
:1031F0000529F1DB00210EE0094800EBC100406821
:1032000040B9074800EBC1004360054800F8312091
:103210000020DEE7491C0529EEDB4FF0FF30D8E740
:10322000DC72002070B50646012515E0002410E090
:103230000B4810F83400A8420AD1094800EBC4003A
:10324000406828B1064800EBC40041683046884712
:10325000641C052CECDB6D1E002DE7DA70BD000050
:10326000DC720020FEB5FF25002400BF0CE004EB5B
:10327000440000EBC401374808440021016041606C
:1032800001818172601CC4B2022CF0DB002414E0C6
:103290003048583850F8240068B12E48583850F853
:1032A000240001682B48FFF7EFFC0546681C10B9A5
:1032B0004FF0FF30FEBD601CC4B20C2CE8DB694649
:1032C000002005F0CFF923496846FFF753FE074673
:1032D0006946012005F0C6F91E490B316846FFF723
:1032E00049FE06461FB916B94FF0FF30E2E719490B
:1032F000002005F09DF90546681C10B94FF0FF301D
:10330000D8E714490B31012005F092F90546681CF5
:1033100010B94FF0FF30CDE70F4805F0FFFE05462E
:10332000681C10B94FF0FF30C4E70C4805F002FFED
:103330000546681C10B94FF0FF30BBE705F006FFEB
:10334000054625B901200349583981F86E0000204F
:10335000B0E70000047300205D3103002532030054
:1033600010B504A11720F4F7DBFC10B90748F7F7F4
:103370004BFB10BD6273705F70776D5F696E69742F
:103380005F6572726F720D0A000000006133030006
:1033900010B504A11920F4F7C3FC10B90748F7F7DA
:1033A00033FB10BD6273705F7274635F636F6E6630
:1033B00069675F6572726F720D0A000091330300D6
:1033C00010B504A11920F4F7ABFC10B90748F7F7C2
:1033D0001BFB10BD6273705F7274635F696E69740A
:1033E0005F6572726F720D0A00000000C133030046
:1033F00010B504A11320F4F793FC10B90748F7F7B0
:1034000003FB10BD6273705F737069305F696E6932
:10341000745F6572726F720D0A000000F133030071
:1034200010B504A11820F4F77BFC10B90748F7F792
:10343000EBFA10BD6273705F7764745F696E6974D4
:103440005F6572726F720D0A000000002134030084
:1034500030B503460C4600201FE09FED110A02EB39
:10346000800181ED000A002114E002EB800595ED5A
:10347000000A01EB800503EB8505D5ED000A04EB9E
:10348000810595ED001A00EE810A02EB800585EDBD
:10349000000A491C0429E8DB401C0928DDDB30BD9B
:1034A0000000000030B5A1B005460C4694ED140AAA
:1034B0008DED010A94ED180A8DED020A94ED190ABA
:1034C0008DED030A94ED1A0A8DED040A94ED380A85
:1034D0008DED050A94ED3C0A8DED060A94ED3D0A4A
:1034E0008DED070A94ED3E0A8DED080A94ED410A30
:1034F0008DED090A94ED450A8DED0A0A94ED460A10
:103500008DED0B0A94ED470A8DED0C0A94ED4A0AF5
:103510008DED0D0A94ED4E0A8DED0E0A94ED4F0AD5
:103520008DED0F0A94ED500A8DED100A002012E087
:1035300001A901EB001101EB800191ED000ADFED23
:10354000FE0A30EE200A01A901EB001101EB800117
:1035500081ED000A401C0428EADB11A901A809F04A
:103560004DFC94ED020ADDED110A20EE200AD4EDA7
:10357000060A9DED151A00EE810AD4ED070A9DEDAD
:10358000191A00EE810AD4ED080A9DED1D1A00EE0D
:10359000810A85ED000A94ED020ADDED120A20EEA3
:1035A000200AD4ED060A9DED161A00EE810AD4ED2C
:1035B000070A9DED1A1A00EE810AD4ED080A9DED66
:1035C0001E1A00EE810A85ED010A94ED020ADDED76
:1035D000130A20EE200AD4ED060A9DED171A00EE1C
:1035E000810AD4ED070A9DED1B1A00EE810AD4ED85
:1035F000080A9DED1F1A00EE810A85ED020A94ED7E
:10360000020ADDED140A20EE200AD4ED060A9DED33
:10361000181A00EE810AD4ED070A9DED1C1A00EE7F
:10362000810AD4ED080A9DED201A00EE810A85ED8D
:10363000030A94ED0B0ADDED110A20EE200AD4ED09
:103640000F0A9DED151A00EE810AD4ED100A9DEDCA
:10365000191A00EE810AD4ED110A9DED1D1A00EE33
:10366000810A85ED040A94ED0B0ADDED120A20EEC5
:10367000200AD4ED0F0A9DED161A00EE810AD4ED52
:10368000100A9DED1A1A00EE810AD4ED110A9DED83
:103690001E1A00EE810A85ED050A94ED0B0ADDED98
:1036A000130A20EE200AD4ED0F0A9DED171A00EE42
:1036B000810AD4ED100A9DED1B1A00EE810AD4EDAB
:1036C000110A9DED1F1A00EE810A85ED060A94EDA0
:1036D0000B0ADDED140A20EE200AD4ED0F0A9DED51
:1036E000181A00EE810AD4ED100A9DED1C1A00EEA6
:1036F000810AD4ED110A9DED201A00EE810A85EDB4
:10370000070A94ED140ADDED110A20EE200AD4ED2B
:10371000180A9DED151A00EE810AD4ED190A9DEDE7
:10372000191A00EE810AD4ED1A0A9DED1D1A00EE59
:10373000810A85ED080A94ED140ADDED120A20EEE7
:10374000200AD4ED180A9DED161A00EE810AD4ED78
:10375000190A9DED1A1A00EE810AD4ED1A0A9DEDA0
:103760001E1A00EE810A85ED090A94ED140ADDEDBA
:10377000130A20EE200AD4ED180A9DED171A00EE68
:10378000810AD4ED190A9DED1B1A00EE810AD4EDD1
:103790001A0A9DED1F1A00EE810A85ED0A0A94EDC2
:1037A000140ADDED140A20EE200AD4ED180A9DED6E
:1037B000181A00EE810AD4ED190A9DED1C1A00EECC
:1037C000810AD4ED1A0A9DED201A00EE810A85EDDA
:1037D0000B0A94ED1D0ADDED110A20EE200AD4ED4E
:1037E000210A9DED151A00EE810AD4ED220A9DED05
:1037F000191A00EE810AD4ED230A9DED1D1A00EE80
:10380000810A85ED0C0A94ED1D0ADDED120A20EE09
:10381000200AD4ED210A9DED161A00EE810AD4ED9E
:10382000220A9DED1A1A00EE810AD4ED230A9DEDBD
:103830001E1A00EE810A85ED0D0A94ED1D0ADDEDDC
:10384000130A20EE200AD4ED210A9DED171A00EE8E
:10385000810AD4ED220A9DED1B1A00EE810AD4EDF7
:10386000230A9DED1F1A00EE810A85ED0E0A94EDE4
:103870001D0ADDED140A20EE200AD4ED210A9DED8B
:10388000181A00EE810AD4ED220A9DED1C1A00EEF2
:10389000810AD4ED230A9DED201A00EE810A85ED00
:1038A0000F0A94ED260ADDED110A20EE200AD4ED70
:1038B0002A0A9DED151A00EE810AD4ED2B0A9DED22
:1038C000191A00EE810AD4ED2C0A9DED1D1A00EEA6
:1038D000810A85ED100A94ED260ADDED120A20EE2C
:1038E000200AD4ED2A0A9DED161A00EE810AD4EDC5
:1038F0002B0A9DED1A1A00EE810AD4ED2C0A9DEDDB
:103900001E1A00EE810A85ED110A94ED260ADDEDFE
:10391000130A20EE200AD4ED2A0A9DED171A00EEB4
:10392000810AD4ED2B0A9DED1B1A00EE810AD4ED1D
:103930002C0A9DED1F1A01E0BE37863500EE810A84
:1039400085ED120A94ED260ADDED140A20EE200A18
:10395000D4ED2A0A9DED181A00EE810AD4ED2B0A47
:103960009DED1C1A00EE810AD4ED2C0A9DED201A63
:1039700000EE810A85ED130A94ED2F0ADDED110AA0
:1039800020EE200AD4ED330A9DED151A00EE810ACF
:10399000D4ED340A9DED191A00EE810AD4ED350AF2
:1039A0009DED1D1A00EE810A85ED140A94ED2F0A93
:1039B000DDED120A20EE200AD4ED330A9DED161A31
:1039C00000EE810AD4ED340A9DED1A1A00EE810A48
:1039D000D4ED350A9DED1E1A00EE810A85ED150A1B
:1039E00094ED2F0ADDED130A20EE200AD4ED330A00
:1039F0009DED171A00EE810AD4ED340A9DED1B1AD5
:103A000000EE810AD4ED350A9DED1F1A00EE810A01
:103A100085ED160A94ED2F0ADDED140A20EE200A3A
:103A2000D4ED330A9DED181A00EE810AD4ED340A64
:103A30009DED1C1A00EE810AD4ED350A9DED201A89
:103A400000EE810A85ED170A94ED380ADDED110AC2
:103A500020EE200AD4ED3C0A9DED151A00EE810AF5
:103A6000D4ED3D0A9DED191A00EE810AD4ED3E0A0F
:103A70009DED1D1A00EE810A85ED180A94ED380AB5
:103A8000DDED120A20EE200AD4ED3C0A9DED161A57
:103A900000EE810AD4ED3D0A9DED1A1A00EE810A6E
:103AA000D4ED3E0A9DED1E1A00EE810A85ED190A3D
:103AB00094ED380ADDED130A20EE200AD4ED3C0A1D
:103AC0009DED171A00EE810AD4ED3D0A9DED1B1AFB
:103AD00000EE810AD4ED3E0A9DED1F1A00EE810A28
:103AE00085ED1A0A94ED380ADDED140A20EE200A5D
:103AF000D4ED3C0A9DED181A00EE810AD4ED3D0A82
:103B00009DED1C1A00EE810AD4ED3E0A9DED201AAF
:103B100000EE810A85ED1B0A94ED410ADDED110AE4
:103B200020EE200AD4ED450A9DED151A00EE810A1B
:103B3000D4ED460A9DED191A00EE810AD4ED470A2C
:103B40009DED1D1A00EE810A85ED1C0A94ED410AD7
:103B5000DDED120A20EE200AD4ED450A9DED161A7D
:103B600000EE810AD4ED460A9DED1A1A00EE810A94
:103B7000D4ED470A9DED1E1A00EE810A85ED1D0A5F
:103B800094ED410ADDED130A20EE200AD4ED450A3A
:103B90009DED171A00EE810AD4ED460A9DED1B1A21
:103BA00000EE810AD4ED470A9DED1F1A00EE810A4E
:103BB00085ED1E0A94ED410ADDED140A20EE200A7F
:103BC000D4ED450A9DED181A00EE810AD4ED460A9F
:103BD0009DED1C1A00EE810AD4ED470A9DED201AD6
:103BE00000EE810A85ED1F0A94ED4A0ADDED110A07
:103BF00020EE200AD4ED4E0A9DED151A00EE810A42
:103C0000D4ED4F0A9DED191A00EE810AD4ED500A49
:103C10009DED1D1A00EE810A85ED200A94ED4A0AF9
:103C2000DDED120A20EE200AD4ED4E0A9DED161AA3
:103C300000EE810AD4ED4F0A9DED1A1A00EE810ABA
:103C4000D4ED500A9DED1E1A00EE810A85ED210A81
:103C500094ED4A0ADDED130A20EE200AD4ED4E0A57
:103C60009DED171A00EE810AD4ED4F0A9DED1B1A47
:103C700000EE810AD4ED500A9DED1F1A00EE810A74
:103C800085ED220A94ED4A0ADDED140A20EE200AA1
:103C9000D4ED4E0A9DED181A00EE810AD4ED4F0ABC
:103CA0009DED1C1A00EE810AD4ED500A9DED201AFC
:103CB00000EE810A85ED230A21B030BD30B5024601
:103CC0000B46002046E0002141E003EB001494ED98
:103CD000000A01F1120402EB8404D4ED000A20EE84
:103CE000200A012404EB800403EB8404D4ED000AD1
:103CF00001F1360402EB840494ED001A00EE810A0F
:103D0000022404EB800403EB8404D4ED000A01F1E7
:103D10003F0402EB840494ED001A00EE810A0324B0
:103D200004EB800403EB8404D4ED000A01F14804A1
:103D300002EB840494ED001A00EE810A00EBC0044B
:103D40000C44104D05EB840484ED000A491C09293C
:103D5000BBDB401C0928B6DB00200FE002EB800132
:103D600091ED000A074901EB8001D1ED000A30EE28
:103D7000600A02EB800181ED000A401C5128EDDB56
:103D800030BD0000B48E002010B502460023002094
:103D900003E032F810402344401C8842F9DBB3FBB7
:103DA000F1F080B210BD02468A4201DC881A7047E9
:103DB0004FF6FF70801A401C0844F8E738B50446F7
:103DC000254600200090686800788DF8000068683B
:103DD00040788DF80100686840786968097800EBE0
:103DE00001200A49088002236A46AC210020F3F72B
:103DF000B1FC01210648F6F777FDF8F76FFB05499E
:103E0000086005490420F5F76FFB38BDAC3F002082
:103E1000A1FB0200B03F0020009F00FF70B50546E7
:103E20002C4600201C490870207A012829D160689E
:103E30000078012825D1194890F82800432801D19D
:103E4000012000E0002015494979884219D0FCF78B
:103E500015FA662011494871F4F750FB18B110A10A
:103E60000820F3F75DFF0D4800791449C8750B4829
:103E700040798876F4F71AFB18B111A10820F3F7FE
:103E80004FFF0648007928B1237AB02114486268B0
:103E9000F3F760FC70BD00003C4000207853002028
:103EA000707772207361766520696E666F726D61DE
:103EB00074696F6E206661696C0000000854002010
:103EC0006170705F6465746563745F4C52207361E8
:103ED0007665206261636B7570206661696C0000B5
:103EE000184000200121014A1170704798400020BD
:103EF00070B50446254606F0BBFA2B7AA7210020B0
:103F00006A68F3F727FC70BD70B505462C46124869
:103F10000079002811DD6068007818B901200F4988
:103F2000087070BD60680078012813D10123A621B4
:103F300000206268F3F70EFC0CE00123084AA6217A
:103F40000848F3F72BFA01200749086001210748C8
:103F5000F6F7CAFC00BFE4E7785300205C3F00207E
:103F6000853F0020603F0020583F00206D0903007E
:103F700070B504462546686800781549C87008463B
:103F8000C078B0B1002008711248FEF707FE104853
:103F9000C078012802D1F4F74DFF05E00C48C07845
:103FA000022801D1F4F74CFF01210B48F6F79CFCE5
:103FB00006E000210848F6F797FC0648FEF716FED3
:103FC0000123034AD21CA2210020F3F7C3FB70BDDA
:103FD0003C3F0020306604003904030070B50446FD
:103FE0002546686800780B49087008460078012863
:103FF00006D10020084908800848FEF7CFFD02E0FE
:104000000648FEF7F3FD0123024AA5210020F3F73D
:10401000A1FB70BD303F00202E3F00201066040041
:1040200070B505462C46606840786168097840EABA
:10403000012615480079D8B160688078012803D13D
:104040003046F5F769FC1DE06068807848B9304675
:10405000F5F762FC237AA42100206268F3F77AFB6B
:1040600010E0237AA42100206268F3F773FB09E0D3
:1040700060688078022802D06068807810B9304685
:10408000F5F74AFC70BD00007853002008B50446DF
:10409000A146D9F804000078009001236A46AB21BC
:1040A0000020F3F757FB00201C494876F4F7FEF98F
:1040B00018B11BA10D20F3F733FE4FF4FA7505B9C3
:1040C0000EE000BF4FF47A7606B905E0DFF87080A5
:1040D000B7013846C04700BF681E051EF2D100BFB9
:1040E00000BF00BF00BF00BF00BFBFF34F8F00BFC6
:1040F00000BF00BF1348006800F4E06012490843A5
:10410000001D1049086000BF00BF00BFBFF34F8F04
:1041100000BF00BF00BF00BF00BFFDE70854002084
:10412000617070207265737461727420736176655A
:10413000206261636B7570206661696C000000002D
:10414000416604000CED00E00000FA0570B505467C
:104150002C466068067836B1012E0ED0022E17D09C
:10416000032E26D11BE014480079012802D1FCF768
:10417000E1FA01E0FBF710FC1CE00F480079012890
:1041800003D11420FCF7BCFA01E0FBF7A9F911E018
:10419000FDF71AF910B92046FBF794FA0AE0237AE2
:1041A000A12100206268F3F7F9F82046FBF730FA06
:1041B00000E000BF00BF70BD7853002010B504467A
:1041C0000E48007800B910BD0D4800880D490988D7
:1041D000884210DA0A480088401C80B208490880EA
:1041E00008490988884202DB002004490870044815
:1041F0000088FBF7A7FA00BFE5E700009D3E00201E
:104200009E3E0020A03E002070B5044625462B7A35
:10421000A72100206A68F3F7C1F870BD38B50446DD
:1042200000200090254668680078009001236A46C7
:10423000A6210020F3F7B2F838BD70B50446254634
:104240002B7AAD2100206A68F3F7A8F870BD000052
:1042500070B505462C4660680078012818D10D48D5
:104260000078012811D1606840780006616889787B
:1042700040EA01406168C97840EA01206168097933
:10428000084305490860FDF72BF80320034908702F
:1042900070BD0000203F0020283F00202C3F002060
:1042A0002DE9F04106463248007908B9BDE8F081B1
:1042B00034466068077817B1012F55D12AE00020F5
:1042C00007E000F141016268525C294932310A5429
:1042D000401C0628F5DB47256068405D0106681C28
:1042E0006268105C41EA0041A81C105C41EA0020B1
:1042F000E91C515C08431E49C862681D6168095C7D
:10430000281D6268105C41EA002119480186FBF70C
:1043100043FB2AE06068407816490870606880783E
:10432000154908706068C07900066168097A40EA3A
:1043300001406168497A40EA01216068807A01435E
:104340000B488161207A192808DB6068807D6168EC
:10435000497D00EB012000B208490880002008498F
:104360000870FBF7BDF800E000BF00BF00BF9DE78D
:1043700078530020D03E0020D13E0020D23E0020C5
:10438000F83E00200121014A11707047F83F0020DB
:1043900008B50446F3F77BFEF3F78FFEF3F761FEF3
:1043A000A146D9F804000078009001236A46AE21A6
:1043B0000020F3F7CFF94FF4FA7505B90EE000BF0E
:1043C0004FF47A7606B905E0134F4FEA8618404657
:1043D000B84700BF681E051EF2D100BF00BF00BF76
:1043E00000BF00BF00BFBFF34F8F00BF00BF00BFC3
:1043F0000A48006800F4E06009490843001D0749C5
:10440000086000BF00BF00BFBFF34F8F00BF00BFF9
:1044100000BF00BF00BFFDE7816704000CED00E0B6
:104420000000FA0538B5044600200090FBF7B6FD01
:1044300000900F48007988B19DF80000012806D14E
:1044400001236A46A3210020F3F784F90EE001233B
:104450006A46A3210020F2F7A1FF07E001200090A7
:1044600001236A46A3210020F2F798FF38BD00001F
:104470007853002010B5044600210348F6F734FABB
:1044800001200249087010BD6D0903005E3F002045
:104490002DE9FF4780464FF00009002400200090DE
:1044A0000190454605F06EFE012801D1BDE8FF8769
:1044B000FAF77CFF6868016800918088ADF8040015
:1044C0006868807900066968C97940EA01406968CE
:1044D000097A40EA01206968497A40EA0106686879
:1044E000C07A6968897A40EA012701202249087068
:1044F00022490720F4F7F8FF00240AE02048005D75
:104500001DF80410884202D04FF0010903E0601C3E
:10451000C4B2062CF2DB00BF19483238C06AB04280
:1045200007D117483238008EB84202D1B9F1000FD6
:104530001FD013483238C662078602A8F4F76CF918
:1045400000240AE01DF804100D48015502A8015D81
:104550000B482C380155601CC4B2062CF2DB01203C
:1045600008490870F7F70AF806F0AEF908B106F046
:1045700063F900BF9AE7000041400020AF0000FF50
:10458000AA5300204040002038B504460120009086
:1045900001236A46A3210020F2F700FF38BD000086
:1045A0002DE9F0478CB08046454606F08DF908B1FC
:1045B00006F042F96868007B10B90CB0BDE8F087DE
:1045C000F6F7DCFF01204449087044490720F4F75E
:1045D0008BFF4FF0000900240020089009906868C4
:1045E000016808918088ADF8240068688079000629
:1045F0006968C97940EA01406968097A40EA01209E
:104600006968497A40EA01066868C07A6968897A07
:1046100040EA012700BF0AE03148005D08A9095DB2
:10462000884202D04FF0010903E0601CC4B2062C9E
:10463000F2DB00BF2A48801FC06AB04207D1284879
:10464000801F008EB84202D1B9F1000F42D0244839
:10465000801FC66207860AA8F4F7DEF800240AE085
:104660000AA8015D1E482C30015508A8015D1C48B0
:104670000155601CC4B2062CF2DBFCF705FC0020DF
:1046800004900590069007901548801F90F8371009
:1046900090F8362090F83500114B9B1F1B7ACDE91E
:1046A0000030CDE902210E48801FC37982790DA127
:1046B00004A8F8F7B1F904A8F1F7F7FE82465146CD
:1046C00004A811F099F8FAF775FB11F04FF8FAF712
:1046D0004DFB00BF00BF70E741400020AF0000FF6E
:1046E0007E5300202530325825303258253032583C
:1046F000253032582530325825303258000000001D
:10470000704710B50446012110200AF01EFFF6F78D
:1047100071FA10BD10B50446F6F74CFA10BD000052
:1047200010B50548007928B1F3EE0E0AB3EE0E0A73
:1047300011F07CF810BD00007853002010B504463D
:10474000F2F793FA0148F7F73FFF10BD71830300BA
:1047500010B50446F2F78DFA0748006807498861EA
:10476000002008610648F2F711FB03200349486165
:104770000448F7F70BFF10BD04B500404479002052
:10478000D98203007183030010B5F3F7F3F92549CB
:1047900008600846006890F82000032841D00320F4
:1047A000096881F820009FED200A1E48006880ED0E
:1047B000050A9FED1E0A1B48006880ED070A9FED61
:1047C0001B0A1848006880ED060AB7EE000A154873
:1047D000006880ED030A9FED150A1248006880ED1D
:1047E000040A9FED120A0F48006880ED010A9FED50
:1047F0000F0A0C48006880ED000A0020094909688A
:1048000081F821009FED090A0648006880ED020A40
:1048100001200449096881F823000249096881F8E8
:10482000220010BD9C4000200000C8420000000093
:10483000024909680144014A11607047084100209B
:1048400070B58AB004460D462E46202102A8F1F725
:1048500021FEF0B28DF80400300A8DF80500012029
:104860008DF808000D4804900594A189ADF81A1040
:104870000221ADF81E100021ADF81C1001A908910D
:1048800001208DF8180001218DF81910228902A944
:10489000A0690AF017F80AB070BD0000B99A0300C9
:1048A00070B590B006460C461546A07818B90120A0
:1048B0008DF80E0002E0A0788DF80E002088ADF88B
:1048C0000C0000200290607C02A910F093FEA07CF6
:1048D0000DF1090110F08EFEE07B08B1012000E02F
:1048E00000209DF80A1060F3C3018DF80A10207CA7
:1048F00008B1012000E000209DF80A1060F30411C7
:104900008DF80A10207B08B1012000E000209DF8FE
:104910000A1060F300018DF80A10207D08B1022012
:1049200000E001209DF80A1060F342018DF80A10A2
:104930001C2109A8F1F7AEFD607BC0F3001018B987
:10494000607BC0F34010F8B100200090E07C0DF1D6
:10495000010110F04FFE00BF9DF8000020F00F0095
:10496000401C8DF800009DF8000020F0F000103091
:104970008DF8000000BF9DF8020020F00600801CAA
:104980008DF80200CDF838D0607B8DF82400A07B34
:104990008DF82500142104A8F1F77CFD03A80490EC
:1049A00002A80590A088ADF81C00A06820B1E0889E
:1049B000ADF81800A0680890A069002849D0002030
:1049C0000190A0690088ADF82C00A0694088ADF87E
:1049D0002E00A06940680A9001A80D90A169087B8B
:1049E00001A910F007FEA169487B0DF1050110F047
:1049F00001FEA069807A08B1012000E000209DF846
:104A0000061060F3C3018DF80610A069C07A08B1E2
:104A1000012000E000209DF8061060F304118DF8DD
:104A20000610A069007A08B1012000E000209DF87E
:104A3000061060F300018DF80610A069807B08B1B4
:104A4000022000E001209DF8061060F342018DF87D
:104A50000610E06908B1E0690C902B4604AA09A988
:104A60003046AADF10B070BD70B58AB004460E465D
:104A7000202101A8F1F70EFD0020099094F8C6024C
:104A800000EB8001C1EB801004EB400594F8C502F7
:104A9000B8B194F8C522521ED1B294F8C62202EBE6
:104AA0008203C3EB821204EB420501EBC10305F163
:104AB0000A0202EB43000289521C92B2ADF8242094
:104AC00002E0E888ADF824002889ADF8260003202C
:104AD0008DF8040009980590049405480390324627
:104AE00001A90448006809F0EDFE0AB070BD00009D
:104AF000195E03009C4A002010B52DED048BB0EE2A
:104B0000408A9FED270AB0EE409A9FED250AF0EE0D
:104B1000408A2448006890F8220060B1B2EE040A8E
:104B2000C8EE000A1F480068C0ED010A00201D49B8
:104B3000096881F82200B2EE040AC8EE000AF0EE1D
:104B4000609A18480068001DDFED170AB0EE690A88
:104B500003F0C0FAF0EE408A9FED140AF4EEC08A2A
:104B6000F1EE10FA04D29FED0E0AB0EE409A11E079
:104B70009FED0F0AF4EEC08AF1EE10FA04DD9FED0E
:104B80000D0AB0EE409A05E0B0EE680A06F0D4FCDB
:104B9000B0EE409AB0EE490ABDEC048B10BD0000A7
:104BA000000000009C400020CDCC4C3D0000AF43F5
:104BB0000080CF430000C84210B51C200AF02FFC33
:104BC00008B1012010BD0020FCE710B5014600220D
:104BD0000B46002004E00C1D245C1444E2B2401C8F
:104BE000DC788442F7DC9878904201D1012010BD36
:104BF0000020FCE770B505460DB9094C01E0084CF2
:104C0000083409E0204607F0ADF9064606B904E08D
:104C100028467168884700BFF4E700BF70BD0000F8
:104C20007093002010B504462CB901200649487045
:104C30000020FFF7DFFF012C04D10120024988701A
:104C4000FFF7D8FF10BD0000689300202DE9F04762
:104C5000024613468C46D3E90245DCE90267B6EB0F
:104C6000040877EB050002D30120BDE8F08700209F
:104C7000FBE701468878012805D191F8200001283A
:104C800001D100207047886A042802D0486A0428AD
:104C900001D10020F6E70120F4E72DE9FF4F03469C
:104CA0000C46002047E0225CFF2A3ED0C2F3C01928
:104CB00022F080014DF82010B9F1000F0DD05DF801
:104CC000201000BF4FF0A0452E46012707FA01F53E
:104CD000C6F8085500BF00BF0DE05DF8201000BF0A
:104CE0004FF0A0452E46012707FA01F5C6F80C55EE
:104CF00000BF00BF00BF5DF8201001252E46002731
:104D0000BC46B84600BF4FF0A04BDA4645EA460B1A
:104D10004BEA870B4BEA0C2B4BEA084E0AF5E06B8B
:104D20004BF821E000BF00BF03E04FF0FF314DF82A
:104D30002010411CC8B20428B5DB6D461A6800215A
:104D400007E055F8217002F5AC6646F821704E1C5C
:104D5000F1B20429F5DB00BFBDE8FF8F0246002059
:104D600007E0536833F810308B4200D17047431C82
:104D700098B213888342F4DC00BFF7E733B58BB0F9
:104D80000546002000900C9878B100240BE02146E5
:104D90000CA809F032FC28B1009A501C009001A820
:104DA00020F81240641C142CF1D32C2269462846AA
:104DB000F1F757FB0DB030BD10B502460B46002190
:104DC0000DE0506830F811004FF6FF74A04204D196
:104DD000506820F81130002010BD481C81B21088A6
:104DE0008842EEDC0420F7E701460888062808DB45
:104DF0000888B0F5486F06DD08884FF6FF729042CC
:104E000001D0072070474888062808DB4888B0F59D
:104E1000486F06DD48884FF6FF72904201D00720A8
:104E2000F0E708884FF6FF72904208D04888904219
:104E300005D008884A88904201DD0720E2E700207B
:104E4000E0E72DE9F04107460D46144698462088D4
:104E5000801D404502D90C20BDE8F0813846FFF79F
:104E6000C3FF064600BF304600B1F5E700BF05208E
:104E7000218868542088401C208012202188685492
:104E80002088401C208022885119388811F0BBF9F5
:104E900021880844208022885119788811F0B3F9BC
:104EA0002188084420800020D6E7000010B5044681
:104EB00000BF03A292212046F1F7ACF900BF10BD5C
:104EC0002E2E5C2E2E5C2E2E5C626C655F636667F8
:104ED0005C736C6176652E630000000030B587B0AE
:104EE0001C216846F1F7D6FA002000904FF480406C
:104EF00001904FF4A030029001208DF80C004FF685
:104F0000FF70ADF80E0001208DF810000020059014
:104F1000094806906846FCF74DFF044600BF254649
:104F200035B100BF05A2A5212846F1F773F900BFEE
:104F300000BF07B030BD0000AD4E03002E2E5C2E2A
:104F40002E5C2E2E5C626C655F6366675C736C61C1
:104F500076652E6300000000F8B505460C46607AC1
:104F600088B9207A10B91048476801E00E48876870
:104F70002A4639466068FCF787FA064616B130467D
:104F800010F000F90EE0002020720748406948B197
:104F900001208DF80000ADF80250034841696846D1
:104FA000884700BFF8BD00004C9300200246002057
:104FB00003E0064B1B5C1354401C054B1B789842C6
:104FC000F7DB03480078087070470000D0820020AB
:104FD0005A4800200246002003E0064B1B5C135495
:104FE000401C054B1B789842F7DB0348007808709B
:104FF000704700009482002059480020F0B5044614
:105000000D460020002108E014F801C00646471CA8
:10501000F8B20B4F07F806C0491CA942F4DB002187
:1050200008E012F801C00646471CF8B2044F07F822
:1050300006C0491C9942F4DB02490870F0BD00002B
:1050400094820020594800202DE9F0410646DDE910
:10505000064500200F88C7F307280746401CDFF8E5
:105060003CC10CF8078091F800800746401C0CF802
:1050700007804F88C7F307280746401C0CF80780B5
:1050800091F802800746401C0CF807808F88C7F310
:1050900007280746401C0CF8078091F80480074653
:1050A000401C0CF807801788C7F307280746401CE8
:1050B0000CF8078092F800800746401C0CF8078027
:1050C0005788C7F307280746401C0CF8078092F85A
:1050D00002800746401C0CF807809788C7F3072812
:1050E0000746401C0CF8078092F804800746401CD5
:1050F0000CF807801F88C7F307280746401C0CF8E8
:10510000078093F800800746401C0CF807805F88F2
:10511000C7F307280746401C0CF8078093F8028065
:105120000746401C0CF807809F88C7F307280746EE
:10513000401C0CF8078093F804800746401C0CF8CC
:1051400007802788C7F307280746401C0CF807800C
:1051500094F800800746401C0CF807806788C7F366
:1051600007280746401C0CF8078094F80280074681
:10517000401C0CF80780A788C7F307280746401C87
:105180000CF8078094F804800746401C0CF8078050
:10519000DFF80CC08CF80000BDE8F081D082002060
:1051A0005A4800207FB506460C4600200290039026
:1051B000ADF80840ADF80A40009001906A4602A997
:1051C000304690DF054605B100BF284604B070BDEB
:1051D00010B5044621460248FDF7CFFA10BD000085
:1051E000308000207CB5002000900190094800909C
:1051F000094801906846FCF773FE044600BF254647
:1052000035B100BF05A22D212846F1F703F800BFF4
:1052100000BF7CBDD1510300284800202E2E5C2EFB
:105220002E5C2E2E5C626C655F6366675C686F73D4
:10523000742E630070B52DED0A8B04460D4694ED77
:10524000060AB1EE400A10EE101A0846F1F72DFBDF
:1052500041EC1B0BB0EE4B0AF0EE6B0AF7F77CFC4F
:10526000B0EE40AAF0EE60AA51EC1A0BF1F760FB29
:1052700008EE900A94ED000A10EE101A0846F1F7B5
:1052800014FB41EC1B0B94ED030A10EE101A0846B8
:10529000F1F70BFB41EC1C0BB0EE4B1AF0EE6B1A66
:1052A000B0EE4C0AF0EE6C0AF8F70AF8B0EE40AA3D
:1052B000F0EE60AA51EC1A0BF1F73AFB08EE100A77
:1052C00094ED080A10EE101A0846F1F7EEFA41ECD8
:1052D0001B0B94ED070A10EE101A0846F1F7E5FAD9
:1052E00041EC1C0BB0EE4B1AF0EE6B1AB0EE4C0A10
:1052F000F0EE6C0AF7F7E4FFB0EE40AAF0EE60AA19
:1053000051EC1A0BF1F714FB09EE100A9FED100A8D
:1053100028EE000ABDEEC00A10EE100A00B2288086
:105320009FED0B0A28EE800ABDEEC00A10EE100AAF
:1053300000B268809FED060A29EE000ABDEEC00AA1
:1053400010EE100A00B2A880BDEC0A8B70BD000000
:1053500000401C4602781206437842EA03428378F2
:1053600042EA0322C3781A433C4B1A6002791206C0
:10537000437942EA0342837942EA0322C3791A431A
:10538000364B5A60027A1206437A42EA0342837A23
:1053900042EA0322C37A1A43304B9A60427B037B72
:1053A00042EA032212B22E4B1A80C27B837B42EA6E
:1053B000032212B22A4B5A80427C037C42EA032227
:1053C00012B2274B9A80C27C837C42EA0322254B8F
:1053D0001A80427D037D42EA0322234B1A80827D9C
:1053E000224B1A80C27D224B1A70427E037E42EA13
:1053F000032212B21F4B1A80C27E837E42EA03222E
:1054000012B21D4B1A80427F037F42EA032212B27E
:10541000194B5A80C27F837F42EA032212B2164B95
:105420009A8090F8212090F8203042EA032212B2AC
:10543000124B1A8090F8232090F8223042EA03227F
:1054400012B20E4B5A8090F8252090F8243042EA90
:10545000032212B2094B9A80704700007489002021
:1054600084490020B6490020BA490020964900200E
:10547000B2490020804900208A490020904900203C
:1054800002781206437842EA0342837842EA032212
:10549000C3781A433C4B1A6002791206437942EAF8
:1054A0000342837942EA0322C3791A43364B5A6096
:1054B000027A1206437A42EA0342837A42EA0322DC
:1054C000C37A1A43304B9A60427B037B42EA032241
:1054D00012B22E4B1A80C27B837B42EA032212B2A5
:1054E0002A4B5A80427C037C42EA032212B2274BA9
:1054F0009A80C27C837C42EA0322254B1A80427D3B
:10550000037D42EA0322234B1A80827D224B1A80BC
:10551000C27D224B1A70427E037E42EA032212B2FF
:105520001F4B1A80C27E837E42EA032212B21D4BB9
:105530001A80427F037F42EA032212B2194B5A803B
:10554000C27F837F42EA032212B2164B9A8090F800
:10555000212090F8203042EA032212B2124B1A8026
:1055600090F8232090F8223042EA032212B20E4B28
:105570005A8090F8252090F8243042EA032212B293
:10558000094B9A8070470000808900209C490020C8
:10559000B4490020B8490020AE490020B14900209C
:1055A00098490020A2490020A84900202DE9F04F89
:1055B00089B004460F4691464FF0000B2021684603
:1055C000F0F768FF94F8C60200EB8001C1EB801091
:1055D00004EB400594F8C50200EBC00105F10A0098
:1055E00000EB410A94F8C502401C2979884207D192
:1055F00008AB00225146204606F074FC834627E0A3
:1056000094F8C5621FE02879401EB04202D14FF0E5
:10561000000806E0701C00EBC00105F10A0000EB79
:10562000410808AB42465146204606F05BFC10B1EB
:105630004FF0010B0AE0C24694F8C502401C84F802
:10564000C502701CC6B22879B042DCDC00BF00BFC6
:10565000BBF1000F05D101203870002009B0BDE872
:10566000F08F0020387004208DF800000898049016
:105670000394044802904A4669460348006809F0CA
:1056800021F9EBE7195E03009C4A0020F0B50346C0
:10569000002249488446DCE90267DCF80450DCF863
:1056A00010C0A0E8E0104548851C2E6806606D68B3
:1056B0004560B3F90400002801DB054600E04542DF
:1056C0003D4E35613D4801813D480068042841DD7B
:1056D000304600693546ED68A8420DDB3046C068AB
:1056E000384D2D68A84202DA3046C06801E03548DE
:1056F0000068344D286003E049F64040314D286091
:105700002D4805692F48006800F5FA70854205DDCF
:105710002D480068401C2C4D286002E000202A4DD6
:10572000286029480068002800DD0122274D2D68E7
:10573000012D14D1214DB5F90850204EB6F906605F
:10574000A81B002801DB054600E04542CB2D06DA08
:10575000012204E01A480068401C194D286000240A
:105760001A48006850B9012A08D119480068194D33
:105770002D68401BB0F5007F00DD0124A2B914485C
:105780000068884202DD1248006800E00846104DBB
:10579000286010480068884202DA0E48006800E07D
:1057A00008460C4D286003E0094801600948016083
:1057B000064802602046F0BD6C4A0020749200202A
:1057C000844A0020804A00208C4A0020884A002019
:1057D000904A0020944A00202DE9FF4F8BB082466A
:1057E00014461D46BAF90400002801DB014600E01A
:1057F000414209B20A910C99B1F90400002801DB79
:10580000014600E041420FFA81FB7622FE49881EE4
:10581000F0F727FE7622FD49881EF0F722FE762259
:10582000FB49881EF0F71DFE7622FA49881EF0F724
:1058300018FE7622F849881EF0F713FEF249891EF9
:105840000A98A1F87600F148801EA0F876B020886A
:10585000EF49891EA1F876006088EE49891EA1F8FB
:105860007600A088EC49891EA1F8760008A809A94D
:1058700004233C22CDE900101421E548801E02F0EB
:105880003CFC06A807A904233C22CDE90010142102
:10589000E048801E02F031FC04A805A904233C2244
:1058A000CDE900101421DC48801E02F026FCDB4B01
:1058B0004FF4FA723C21D548801E06F04AFA814620
:1058C000B9F1010F02D15020D5490880D54B4FF4D2
:1058D000FA723C21CD48801E06F0F6F90390D048BC
:1058E000B0F90000002809DDCF4B4FF47A723C215B
:1058F000C548801E06F02DFA064608E0CA4B4FF454
:10590000FA623C21C048801E06F023FA0646BE48D3
:10591000801EB0F97600BC49891EB1F96E10401A9C
:1059200010F1320F0FDDB848801EB0F97600BF4984
:10593000B1F9001088420CDAB348801EB0F8760046
:10594000BA49088005E0B048801EB0F87600B74933
:105950000880AD48801EB0F97600B449B1F9001056
:10596000401AB0F57A7F00DD0126A848801EB0F904
:105970007600AA49B1F90010401AB0F5FA6F00DDBF
:105980000126AB4B4FF4FA723C219F48801E06F073
:105990009BF907469D48801EB0F976009F49B1F9F2
:1059A0000010401AB0F5FA7F09DD9848801EB0F962
:1059B00076009C49B1F90010081AC8281FDB9248EC
:1059C000801EB0F976009849B1F90010401AB0F580
:1059D000FA7F09DD8C48801EB0F976009449B1F950
:1059E0000010081AC8280ADB8748801EB0F9760024
:1059F0008E49B1F90010401AB0F5FA7F04DD50204D
:105A00008C4908808C490880012F02D100208A49E6
:105A100008807E48801EB0F976008049B1F90010F8
:105A2000401AB0F57A7F0BDD7748801EB0F976001A
:105A30007D49B1F90010401AB0F57A7F00DD0126EA
:105A40007E4A39B230B20FF0A1FC7C48B0F90000B8
:105A5000002802DD50207A4908806F48801E6D4B77
:105A60009B1E6B4A921E2946009074480FF04CFC16
:105A70007348B0F90000002804DC6E48B0F900005B
:105A800000281CDDBDF92400BDF92010401A822831
:105A900015DABDF91C00BDF91810401A82280EDA7B
:105AA000BDF91400BDF91010401A822807DA012050
:105AB00028806248008810B9022060490880208848
:105AC00010FB00F0618811FB0100A18811FB0100AF
:105AD00002905949B1F90010002910DD0299A1F591
:105AE0008000002801DB014600E04142554A914216
:105AF00005DA5248008810B9022050490880BDF9E3
:105B00002400BDF92010401A672816DABDF91C00E0
:105B1000BDF91810401A67280FDABDF91400BDF955
:105B20001010401A672808DA0121199801804648A8
:105B30000068401C4449086005E000211998018074
:105B400000204149086040480068B0F5C87F03DD87
:105B500001202880394908804FF067083648B0F99D
:105B60000000002801DD40F20648384B1B88012B5D
:105B700040D1274B9B1EB3F96E30DFF894C0ACF1D7
:105B8000020CBCF976C0A3EB0C02002A01DB134621
:105B900000E0534243452DDA1E4B9B1EB3F96E3095
:105BA000DFF870C0ACF1020CBCF976C0A3EB0C01BD
:105BB000002901DB0B4600E04B4243451ADA164B45
:105BC0009B1EB3F96E30DFF850C0ACF1020CBCF98B
:105BD00076C0A3EB0C00002801DB034600E0434243
:105BE000434507DA012028801448008810B90220B4
:105BF000124908801248B0F9000000282ADD104838
:105C00000088401E00B223E0069000207E90002015
:105C1000F69000206E910020E69100202C4A002092
:105C2000244A0020304A00202A4A00201C4A002032
:105C30002E4A0020264A0020284A00200C4A002034
:105C4000164A0020E0930400204A0020144A002055
:105C5000214908802148B0F90000002805DD1F48CF
:105C60000088401E00B21D4908801D48B0F90000A0
:105C7000002805DD1A480088401E00B21849088037
:105C80001848B0F90000002805DD16480088401EBD
:105C900000B2144908801448B0F90000002805DD5E
:105CA00011480088401E00B20F490880288810B1B2
:105CB0005020094908800D48B0F90000002805DD92
:105CC0000A480088401E00B2084908802888084910
:105CD00008800FB0BDE8F08F164A0020184A002057
:105CE0001A4A0020244A0020264A0020284A002080
:105CF000144A002030B59FB004460D467C2168460A
:105D0000F0F7C8FBADF8025003208DF800000194B5
:105D10000448006818B168460249096888471FB0FE
:105D200030BD0000984A00202DE9F04104460D46A0
:105D3000164694F8C60200EB8001C1EB801004EB1C
:105D4000400840460DF078FC0746E7B3D4F8CC0293
:105D5000062838D204F53470D4F8CC1200EBC11008
:105D6000468004F53471D4F8CC2201EBC211081D31
:105D700076224146F0F775FB45B1002104F53470F9
:105D8000D4F8CC2200EBC210017007E0022104F528
:105D90003470D4F8CC2200EBC210017004F53470DA
:105DA000D4F8CC1200EBC110C767D4F8CC02401C69
:105DB000C4F8CC020549D4F8CC020968884202D163
:105DC00020460CF009FBBDE8F0810000A04A00204D
:105DD0002DE9F041A0B004460D46164694F8C602DF
:105DE00000EB8001C1EB801004EB400840460DF051
:105DF00023FC074657B17C22064901A8F0F731FB86
:105E0000ADF80660029501A8B84700BF20B0BDE814
:105E1000F0810000FC6804002DE9F04105460C46C5
:105E200016462746002087F8C802324629463846DB
:105E3000FFF7CEFF31463846FFF75CFFBDE8F08143
:105E4000F0B589B004460E464FF4BA612046F0F72B
:105E500021FB202101A8F0F71DFB31461E480068F8
:105E600008F006FD054600BF284608B109B0F0BDA0
:105E700000BFA4F8CA620020C4F8CC0284F8C702AC
:105E800084F8C60284F8C50294F8C60200EB8001CB
:105E9000C1EB801004EB400794F8C6020F4901EBF8
:105EA00080000068386002208DF804000120ADF801
:105EB00014003968CDF8161004940948039032464E
:105EC00001A90548006808F0FDFC054615B9012048
:105ED00084F8C8022846C9E79C4A00207E92002028
:105EE000195E03001CB518213348F0F7D3FA0021DE
:105EF00031482C3880F84C1080F8491080F84D104B
:105F000080F84A1080F84E1080F84B1080F8461048
:105F100080F8481080F84710002027492C3981F874
:105F20004400002124482C3880F845102348224999
:105F30002C3948602248086000208862032103460B
:105F40000122CDE900101146072009F052F9032083
:105F500009F0D7F9042009F0D4F9052009F0D1F9A6
:105F6000062009F0CEF90021032009F03DFB0021B5
:105F7000042009F039FB0021052009F035FB002140
:105F8000062009F031FB0021072009F02DFB03203A
:105F90000CF045FA0121072009F026FB03200CF044
:105FA0003EFAF5F7C7F9074A07A14FF47A70F4F7FC
:105FB000C1FC0EF023F81CBDC47A00207D2404002F
:105FC000E5240400E17103006472765F6C736D5F19
:105FD0007370695F6572726F725F7265706F7274F1
:105FE0000000000038B50446134890F84900E8B1B5
:105FF0006946114806F02DFD9DF8000000F00100F3
:1060000088B10E4800210160818001460A4805F0F0
:10601000D9FF0A48008820800848408860800748E7
:106020008088A08005E04FF0FF3038BD4FF0FF3092
:10603000FBE70020F9E70000987A0020E87A0020CA
:106040000146054802680A6042684A6002890A817E
:10605000807A887200207047DC7A00202DE9F041B8
:10606000054600260024474890F84A0000B1B61DB6
:10607000444890F8490000B1B61D424890F84B00E2
:1060800000B1B61D3F4890F84800012800D1B61D68
:1060900018213D48F0F7FEF9F2B23B49394806F0C5
:1060A000BAF90746781C18B94FF0FF30BDE8F08107
:1060B000002D64D0334890F84A0098B104EB4400B6
:1060C000314931F81000E88004EB440001EB400056
:1060D0004188298104EB44002B4901EB4000818871
:1060E0006981641C274890F8490090B104EB440092
:1060F000254931F81000288004EB440001EB4000F2
:106100004088688004EB440001EB40008088A88050
:10611000641C1C4890F84B0098B104EB44001A49E9
:1061200031F81000A88104EB440001EB40004188E5
:10613000E98104EB4400144901EB40008188298285
:10614000641C104890F84800012818D104EB440062
:106150000D4901EB40004078000404EB44010A4A79
:1061600012F8111040EA012004EB440102EB410156
:10617000C978084300EBC00101EB00106861002002
:1061800094E70000987A0020E87A00203EB50020CD
:1061900001900025002402A9214806F08CF9012372
:1061A0006A463B211E4806F028FB9DF8000000F0DF
:1061B000E000E0280CD10021194806F0EAF81E2082
:1061C0000CF056F90621164806F0E3F8601E3EBDB5
:1061D0009DF8080008B301A9114805F053FF1048C5
:1061E00090F8490008B1E01C84B20D4890F84A00CC
:1061F00008B1E01C84B20A4890F84B0008B1E01CDA
:1062000084B2074890F84800012801D1E01C84B20C
:10621000BDF8040090FBF4F085B22846D7E70000F3
:10622000987A002010B50649064805F01FFF04487B
:1062300000786A2802D04FF0FF3010BD0020FCE744
:1062400090410020987A002038B50024FF2000906B
:1062500001236A46002138200DF004F90446601C31
:1062600018B19DF80000802802D04FF0FF3400E004
:106270000024204638BD0520704700001CB5F5F706
:1062800037F80020032103460122CDE90010114612
:10629000072008F0AEFF032009F033F800210320A7
:1062A00009F0A2F90021042009F09EF9002105203F
:1062B00009F09AF90021062009F096F9002107203B
:1062C00009F092F918211348F0F7E4F80021114879
:1062D0002C3880F84C1080F8491080F84D1080F868
:1062E0004A1080F84E1080F84B1080F8461080F865
:1062F000481080F84710002006492C3981F84400E6
:10630000002104482C3880F84510002001492C3920
:1063100088621CBDC47A00207CB50121072009F0E9
:1063200063F903250124002000902346024601461C
:106330000190284608F05DFF00BF18211548F0F7CE
:10634000A9F8002113482C3880F84C1080F8491027
:1063500080F84D1080F84A1080F84E1080F84B10ED
:1063600080F8461080F8481080F84710002009494E
:106370002C3981F84400002106482C3880F845105B
:10638000002004492C398862F4F7B2FFF4F7D2FFF9
:1063900000207CBDC47A002010B51A491A4805F0C7
:1063A00065FE184800786A2802D04FF0FF3010BD13
:1063B0000121154806F042FA4FF4FA60124988624A
:1063C00000BF1249104806F028FA0F48806A401EA4
:1063D0000D4988620D48007818B10846806A002887
:1063E000EFD10948806A10B94FF0FF30DFE707218D
:1063F000054806F0F3FB0221034806F041FC0020AB
:10640000D5E7000090410020987A002091410020BB
:1064100010B54FF4FA604B49886200BF4A494948B9
:1064200006F0F5FB4748806A401E464988624648A8
:10643000007818B90846806A0028EFD14148806A80
:1064400010B94FF0FF3010BD40493E4805F0BAFD8D
:106450003F48002101604160816000203D49087093
:1064600047E04FF4FA603749886200BF3649354843
:1064700006F0CDFB3348806A401E324988623248BC
:10648000007818B90846806A0028EFD12D48806A44
:1064900010B94FF0FF30D6E72C492A4805F092FD9D
:1064A00000202D4908701BE028492B4A127831F949
:1064B000120006F069F826482749097800EB8100A8
:1064C000D0ED000A30EE200A21482349097800EB7C
:1064D000810080ED000A20480078401C1E490870A9
:1064E0001D4800780328DFDB1A480078401C194952
:1064F0000870184800780528B3DB0020154908709B
:1065000016E013481349097800EB810090ED000A6A
:10651000F1EE040A80EE201A0D480E49097800EBCE
:10652000810080ED001A0B480078401C0949087072
:10653000084800780328E4DB0221024806F0F0FB5B
:10654000002080E7987A00209941002092410020A5
:10655000007B00209A4100209B41002010B52DEDCA
:10656000048B4FF4FA608549886200BF84498348F0
:1065700006F04DFB8148806A401E80498862804851
:10658000007818B90846806A0028EFD17B48806AF5
:1065900020B94FF0FF30BDEC048B10BD794977482E
:1065A00005F010FD78480021016041608160002005
:1065B0007649087047E04FF4FA607049886200BF7E
:1065C0006F496E4806F023FB6C48806A401E6B4999
:1065D00088626B48007818B90846806A0028EFD1B5
:1065E0006648806A10B94FF0FF30D4E765496348C8
:1065F00005F0E8FC0020664908701BE06149644A28
:10660000127831F9120005F0BFFF5F486049097840
:1066100000EB8100D0ED000A30EE200A5A485C49B8
:10662000097800EB810080ED000A59480078401C91
:1066300057490870564800780328DFDB5348007834
:10664000401C52490870514800780528B3DB0020EF
:106650004E49087016E04C484C49097800EB81001F
:1066600090ED000AF1EE040A80EE201A46484749F0
:10667000097800EB810080ED001A44480078401C46
:1066800042490870414800780328E4DB00203F4974
:1066900008702EE03C483D4A127800EB820090EDF5
:1066A000000A3C48394A127800EB8200D0ED000A1B
:1066B00030EE600A10EE101A0846F0F7F6F841ECDA
:1066C000190BB0EE490AF0EE690AF7F77DF8B0EE63
:1066D000408AF0EE608A51EC180BF0F729F92E4948
:1066E0002A4A127841F8220028480078401C27499D
:1066F0000870264800780328CCDB01202749087061
:1067000000202249087023E023482049097800EB43
:10671000810090ED000ADFED220AB4EEE00AF1EE0E
:1067200010FA0DD31C481949097800EB810090ED4F
:10673000000ADFED1C0AB4EEE00AF1EE10FA02DD09
:1067400000201649087011480078401C0F49087055
:106750000E4800780328D7DB0021084806F0E0FA4D
:106760000021064806F03AFA0721044805F06FFFB9
:106770000621024805F0C0FF00200CE7987A0020AF
:1067800099410020924100200C7B00209A4100207A
:106790009B410020007B0020187B002098410020B6
:1067A0000000B4420080D44410B54FF4FA604B4965
:1067B000886200BF4A49494805F062FF4748806A3D
:1067C000401E464988624648007818B90846806AE3
:1067D0000028EFD14148806A10B94FF0FF3010BD5A
:1067E00040493E4805F018FC3F48002101604160E7
:1067F000816000203D49087047E04FF4FA60374956
:10680000886200BF3649354805F03AFF3348806A50
:10681000401E324988623248007818B90846806ABA
:106820000028EFD12D48806A10B94FF0FF30D6E72D
:106830002C492A4805F0F0FB00202D4908701BE088
:1068400028492B4A127831F9120005F091FE2648AA
:106850002749097800EB8100D0ED000A30EE200ACC
:1068600021482349097800EB810080ED000A204887
:106870000078401C1E4908701D4800780328DFDBA3
:106880001A480078401C19490870184800780528F3
:10689000B3DB00201549087016E013481349097846
:1068A00000EB810090ED000AF1EE040A80EE201A60
:1068B0000D480E49097800EB810080ED001A0B4865
:1068C0000078401C09490870084800780328E4DB78
:1068D0000121024805F05FFF002080E7987A002040
:1068E0009941002092410020007B00209A41002025
:1068F0009B41002010B52DED048B864800210160DE
:106900004160816000208449087049E04FF4FA60DA
:106910008249886200BF8249804805F0B1FE7F4805
:10692000806A401E7D4988627D48007818B9084613
:10693000806A0028EFD17948806A20B94FF0FF3093
:10694000BDEC048B10BD7749744805F065FB002051
:10695000754908701BE07349734A127831F91200C7
:1069600005F006FE6B487049097800EB8100D0ED18
:10697000000A30EE200A67486B49097800EB810075
:1069800080ED000A68480078401C67490870664836
:1069900000780328DFDB60480078401C5E490870FF
:1069A0005D4800780528B1DB00205B49087016E0DF
:1069B00058485949097800EB810090ED000AF1EE42
:1069C000040A80EE201A53485349097800EB8100ED
:1069D00080ED001A50480078401C4F4908704E481E
:1069E00000780328E4DB00204B4908702EE049487A
:1069F000494A127800EB820090ED000A4B48464A63
:106A0000127800EB8200D0ED000A30EE600A10EE42
:106A1000101A0846EFF749FF41EC190BB0EE490A8E
:106A2000F0EE690AF6F7D0FEB0EE408AF0EE608A2A
:106A300051EC180BEFF77CFF3D49374A127841F8CB
:106A4000220035480078401C3349087032480078ED
:106A50000328CCDB00203049087023E034482E495D
:106A6000097800EB810090ED000ADFED320AB4EE08
:106A7000E00AF1EE10FA0DD32D482749097800EB12
:106A8000810090ED000ADFED2C0AB4EEE00AF1EE91
:106A900010FA02DD0020294908701F480078401CC8
:106AA0001D4908701C4800780328D7DB00211B48CB
:106AB00005F071FE0021194805F0C9FD1F48007856
:106AC000012810D10121154805F031FFFF201C4994
:106AD0000870124805F01AFF19480078012816D0EE
:106AE0004FF0FF302CE701210C4805F020FFFF207C
:106AF00013490870094805F009FF1148007801287A
:106B000002D04FF0FF301BE74FF0FF3018E70020B6
:106B100016E700000C7B00209A410020987A0020A4
:106B200099410020924100209B410020007B0020E1
:106B3000187B0020007C124800E62A49984100207A
:106B400091410020F8B504460026144890F84C0006
:106B5000A04221D014B1012C04D101E0002504E0B1
:106B6000012502E04FF0FF3600BF00BF16B14FF025
:106B7000FF30F8BD2946094806F082F86946074803
:106B800006F056F89DF80000A84202D04FF0FF3002
:106B9000EFE7024880F84C403046EAE7987A002058
:106BA000F8B5054600261A4890F84900A8422DD0AD
:106BB000082D11D2DFE805F004061010080A0C0EAB
:106BC00000240CE001240AE0042408E0052406E087
:106BD000062404E0072402E04FF0FF3600BF00BFA8
:106BE00016B14FF0FF30F8BD2146094805F0F6FF19
:106BF0006946074805F0B1FF9DF80000A04202D0A9
:106C00004FF0FF30EFE7024880F849503046EAE79E
:106C1000987A0020F8B504460026144890F84400FD
:106C2000A04221D014B1012C04D101E0002504E0E0
:106C3000012502E04FF0FF3600BF00BF16B14FF054
:106C4000FF30F8BD2946094806F051F86946074863
:106C500006F02FF89DF80000A84202D04FF0FF3058
:106C6000EFE7024880F844403046EAE7987A00208F
:106C70002DE9FF4F8BB08B4600200A900190914880
:106C800090F846100B98814274D00B98082873D264
:106C9000DFE800F0040772721C31465B0024002517
:106CA0006EE0012401254FF0060ABBF1010F00D16F
:106CB00001260D98012800D101270E9808B14FF048
:106CC00001081898012800D1814659E001240425C3
:106CD0004FF0060ABBF1040F00D101260D980428DD
:106CE00000D101270E9808B14FF00108189801282B
:106CF00000D1814644E0012405254FF0060ABBF18E
:106D0000050F00D101260D98052800D101270E9806
:106D100008B14FF001081898012800D181462FE0F2
:106D2000012406254FF0060ABBF1060F00D101260B
:106D30000D98062800D101270E9808B14FF00108E0
:106D40001898012800D181461AE0012407254FF048
:106D5000060ABBF1070F00D101260D98072800D1C4
:106D600001270E9808B14FF001081898012800D1AA
:106D7000814605E0A4E0FFE74FF0FF300A9000BF36
:106D800000BF0A9820B14FF0FF300FB0BDE8F08F80
:106D900021464C4805F026FB09A94A4805F012FB9C
:106DA0009DF82400A04202D04FF0FF30EDE7002C08
:106DB00073D05146434805F0ECFA07A9414805F065
:106DC000BDFA9DF81C00504502D04FF0FF30DCE7C3
:106DD000012E11D131463B4805F0B1FB06A93948D7
:106DE00005F079FB9DF81800B04201D0B01ECCE749
:106DF0000198C01C80B20190012F11D13946314851
:106E000005F083FA05A92F4805F04BFA9DF8140008
:106E1000B84201D0B81EB8E70198C01C80B20190FA
:106E2000B8F1010F12D14146264805F0D4F904A962
:106E3000244805F09CF99DF81000404502D04FF021
:106E4000FF30A2E70198C01C80B20190B9F1010F98
:106E500012D149461B4805F00BFA03A9194805F061
:106E6000D3F99DF80C00484502D04FF0FF308CE775
:106E70000198C01C80B201901248019905F0F7FA00
:106E800002A9104805F0D6FABDF808100198814211
:106E900003D04FF0FF3078E7FFE72946094805F0B7
:106EA0004DF908A9074805F00AF99DF82000A84205
:106EB00002D04FF0FF3068E702490B9881F8460096
:106EC0000A9862E7987A0020F8B50446002614482C
:106ED00090F84D00A04221D014B1062C04D101E05D
:106EE000002504E0062502E04FF0FF3600BF00BF9A
:106EF00016B14FF0FF30F8BD2946094805F0FCFBFC
:106F00006946074805F0CDFB9DF80000A84202D075
:106F10004FF0FF30EFE7024880F84D403046EAE797
:106F2000987A0020F8B5054600261A4890F84A00DD
:106F3000A8422DD0082D11D2DFE805F0040610106C
:106F4000080A0C0E00240CE001240AE0042408E0E6
:106F5000052406E0062404E0072402E04FF0FF3693
:106F600000BF00BF16B14FF0FF30F8BD2146094801
:106F700005F06DFB6946074805F02BFB9DF8000006
:106F8000A04202D04FF0FF30EFE7024880F84A50AD
:106F90003046EAE7987A0020F8B5044600261448FF
:106FA00090F84500A04221D014B1012C04D101E099
:106FB000002504E0012502E04FF0FF3600BF00BFCE
:106FC00016B14FF0FF30F8BD2946094805F0CAFB5D
:106FD0006946074805F0A9FB9DF80000A84202D0C9
:106FE0004FF0FF30EFE7024880F845403046EAE7CF
:106FF000987A0020F8B505460F461646002E01DDAA
:10700000062E02DB4FF0FF30F8BD454890F84B00EC
:10701000A84278D0062E7DD2DFE806F07C03102748
:1070200030444DB10620009001236A4629213820C2
:107030000FF0A6FA044600E000246BE09DB1FF20AB
:10704000009001236A46292138200CF00BFA0446EF
:10705000601C18B19DF80000062802D04FF0FF34E4
:1070600002E0002400E0002454E0009501236A4679
:107070000A2138200FF084FA04464BE0FF200090EC
:1070800001236A460A2138200CF0ECF90446601C02
:1070900018B19DF80000A84202D04FF0FF3400E084
:1070A000002437E087B301211D4805F077FC1D4916
:1070B0001B4805F08CFC0421194805F085FBFF20D6
:1070C000009001236A460321154805F096FB002134
:1070D000134805F079FB9DF80000012802D04FF01D
:1070E000FF3091E700210E4805F0EBFB01210C4831
:1070F00005F056FA01210A4805F0CAFB00240848A9
:1071000080F84B5005E006E0FFE70024044880F8D3
:107110004B5000BF01E0002076E7204674E70000F6
:10712000987A002084410020F8B5044600261448CF
:1071300090F84700A04221D014B1012C04D101E005
:10714000002504E0012502E04FF0FF3600BF00BF3C
:1071500016B14FF0FF30F8BD2946094805F0B4FCE0
:107160006946074805F092FC9DF80000A84202D04D
:107170004FF0FF30EFE7024880F847403046EAE73B
:10718000987A0020F8B504460026144890F8480084
:10719000A04220D01CB1012C03D1012504E0002520
:1071A00002E04FF0FF3600BF00BF16B14FF0FF30D6
:1071B000F8BD2946094805F0A0FC6946074805F0D6
:1071C00054FC9DF80000A84202D04FF0FF30EFE7DA
:1071D000024880F848403046EAE70000987A0020EC
:1071E00000B589B0202101A8EFF754F910480068D4
:1071F00048B10F480FA1026801A8F5F70DFC01A9DD
:107200001420F0F78DFD1048006848B10E480FA11A
:10721000026801A8F5F700FC01A91420F0F780FD31
:107220000020034908600849086009B000BD00005B
:10723000884100207370695F77726974655F657259
:10724000722C25640D0A00008C4100207370695F68
:10725000726561645F6572722C25640D0A0000001E
:107260001CB51F480021816081810121C17300206C
:107270001B4988731B4848601B4808600020032195
:1072800003460122CDE9001011460B2007F0D9FF7B
:1072900000210B2008F0DAF9C8200BF0CFF801210B
:1072A0000B2008F0D3F90D2008F043F800210D2041
:1072B00008F0CCF90F2008F03CF801210F2008F06D
:1072C000C5F9C8200BF0BAF8F1F758FC0EF046FBF0
:1072D0000446601C10B94FF0FF301CBD0020FCE7D5
:1072E000347B0020AD300400D130040070B5054679
:1072F0001848807B48B3184800210160818002F063
:107300007FFC0446601C10B94FF0FF3070BD12487E
:10731000801C02F086FC0446601C10B94FF0FF3060
:10732000F4E70D48001D02F08DFC0446601C10B906
:107330004FF0FF30EAE70848008828800648408878
:10734000688005488088A88002E04FF0FF30DDE7C4
:107350000020DBE7347B0020A44100201CB5002086
:10736000032103460122CDE9001011460B2007F04E
:1073700068FF0D2007F0DDFF0C2007F0DAFF0E207C
:1073800007F0D7FF0F2007F0D4FF00210D2008F0F1
:107390005DF900210C2008F059F900210E2008F0B9
:1073A00055F900210F2008F051F900210B2008F0B9
:1073B0004DF900201CBD00001CB500200321034630
:1073C0000122CDE9001011460B2007F03AFF012100
:1073D0000B2008F03BF90D2007F0ABFF00210D203A
:1073E00008F034F90F2007F0A4FF01210F2008F066
:1073F0002DF9F1F7C3FB094800218160818101214A
:10740000C1730020054988730EF0A8FA0446601C79
:1074100010B94FF0FF301CBD0020FCE7347B00208A
:107420003EB505466348807BA84270D025B1012D4A
:107430001ED0022D1BD16BE000200EF0ABF80446ED
:10744000601C10B94FF0FF303EBD684602F070FC82
:107450000446601C10B94FF0FF30F5E79DF80000BE
:1074600010B14FF0FF30EFE70020524988739EE0E3
:1074700001200EF08FF80446601C10B94FF0FF3069
:10748000E2E7684602F054FC0446601C10B94FF075
:10749000FF30D9E79DF80000012802D04FF0FF30FF
:1074A000D2E706200EF04AF80446601C10B94FF0EF
:1074B000FF30C9E702A802F0FFFB0446601C10B9C8
:1074C0004FF0FF30C0E79DF80800062802D04FF0CB
:1074D000FF30B9E702200EF00BF80446601C10B92B
:1074E0004FF0FF30B0E701A802F0BEFB0446601C7D
:1074F00010B94FF0FF30A7E79DF80400022802D032
:107500004FF0FF30A0E701202A4988734FE04FE099
:1075100001200EF03FF80446601C10B94FF0FF3018
:1075200092E7684602F004FC0446601C10B94FF074
:10753000FF3089E79DF80000012802D04FF0FF30AE
:1075400082E702200DF0FAFF0446601C10B94FF0EC
:10755000FF3079E702A802F0AFFB0446601C10B9C7
:107560004FF0FF3070E79DF80800022802D04FF07E
:10757000FF3069E701200DF0BBFF0446601C10B925
:107580004FF0FF3060E701A802F06EFB0446601C7C
:1075900010B94FF0FF3057E79DF80400012802D0E2
:1075A0004FF0FF3050E702200249887300BF00BF50
:1075B000002049E7347B00201CB50020032103464E
:1075C0000122CDE900101146122007F026FE1320FB
:1075D00007F0A3FE142007F0A0FE0021132008F0FE
:1075E00018F80021142008F014F80021122008F0E7
:1075F00010F8052007F0BAFC0121122008F009F864
:10760000052007F0B3FC104A10A14FF47A70F3F78D
:1076100091F9F1F752F9134800210160416081604E
:10762000C16011480F4948601048086000210D48AA
:10763000C17300200B4988730BF05CFD08B100207A
:107640001CBD4FF0FF30FBE73D780300716D635FB9
:107650006969635F6572726F725F7265706F727471
:1076600000000000247B0020B5240400192504003C
:1076700001460248C089088000207047247B002012
:107680007CB5044601208DF80000134806236A46A5
:10769000012146683820B047054615B94FF0FF3044
:1076A0007CBDBCB19DF800009DF8011040EA0120AE
:1076B00000B220809DF802009DF8031040EA0120EE
:1076C00000B260809DF804009DF8051040EA01209A
:1076D00000B2A0800020E3E7247B002010B50BF06F
:1076E00009FD08B1002010BD4FF0FF30FBE704207A
:1076F00070471CB50020032103460122CDE900108C
:107700001146122007F089FD132007F006FE142011
:1077100007F003FE0021132007F07BFF0021142057
:1077200007F077FF0021122007F073FF00201CBD37
:1077300010B50121122007F06CFFF1F7BEF80448E4
:10774000002181608181C17300200149887310BDCF
:10775000247B0020F8B505460E464FF0FF37002E7B
:1077600001DD052E02DB4FF0FF30F8BD3248807B93
:10777000A8425CD0012E06D0022E18D0032E2ED0A7
:10778000042E53D13BE085B1062000902A48012306
:107790006A462921D0F800C03820E047044614B9D1
:1077A0004FF0FF30E1E7002700E000273EE0A5B101
:1077B000FF200090204801236A462921D0F804C008
:1077C0003820E04704461CB19DF80000062802D08E
:1077D0004FF0FF30C9E7002700E0002726E00095C2
:1077E000154801236A460A21D0F800C03820E04736
:1077F000044614B94FF0FF30B7E7002716E0FF202A
:1078000000900D4801236A460A21D0F804C03820B0
:10781000E04704461CB19DF80000A84202D04FF09A
:10782000FF30A2E700270448857300BF01E0002075
:107830009BE7384699E70000247B002000B589B01B
:10784000202101A8EEF726FE1048006848B10F4835
:107850000FA1026801A8F5F7DFF801A91520F0F7DC
:107860005FFA1048006848B10E480FA1026801A8ED
:10787000F5F7D2F801A91520F0F752FA00200349D4
:1078800008600849086009B000BD00009C41002064
:107890006969635F77726974655F6572722C2564CC
:1078A0000D0A0000A04100206969635F7265616490
:1078B0005F6572722C25640D0A00000070B50546E4
:1078C0000C464FF4803000FA04F1284600F03CFBEF
:1078D00070BD70B505460C464FF4A07000EB8400F7
:1078E00086B23146284600F049FB70BD2DE9F047CD
:1078F00004460D4616461F464FF4803000FA05F840
:107900004FF4A07000EB85001FFA80F926F07F4647
:107910004146206808F040F94146206808F02DF9FA
:107920004946206808F01FF932462946206808F0C9
:107930000AF94146206808F026F91FB1414620683F
:1079400008F030F9BDE8F08710B50446206808F06B
:10795000FFF810BD2DE9F04303460C461646587952
:10796000284941F820605879274901EBC000007987
:1079700018B108221046BDE8F08321881868C0F8C5
:10798000081500BF93F90450A77828463946002807
:1079900008DB4FEA417C4FEA1C68DFF870C00CF846
:1079A00000800BE04FEA417C4FEA1C69DFF860C0C1
:1079B00000F00F08A8F104080CF8089000BF00BF01
:1079C00093F90410084600280DDB00BF00BF00F04B
:1079D0001F070125BD404709BF0007F1E027C7F891
:1079E000005100BF00BF00BF00BF01205979064D04
:1079F00005EBC10108715879294641F83030002261
:107A00001046B8E7044B0020084B002000E400E0DB
:107A100018ED00E010B5014691F90400002807DBDD
:107A200000F01F0301229A40024B440943F824202E
:107A300000BF10BD00E200E070B505460C462246CE
:107A40000221284600F08CFA70BD10B504464FF4B0
:107A50008271204600F092FA10BD10B50446002154
:107A6000206808F0AAF810BD10B50446042120686B
:107A700008F0A3F810BD2DE9F84F044688461546D6
:107A800099464FF4803000FA08FA4FF4A07000EBEA
:107A900088001FFA80FB25F07F455146204600F004
:107AA00053FA206808F054F806464146206808F06A
:107AB0003FF8009032464146206808F044F85946A5
:107AC000206808F050F8314600980EF0BAFA012804
:107AD00006D1102008F038FB5946206808F043F81A
:107AE000206808F035F80646314628460EF0A9FA17
:107AF00007465146206808F046F8012F0FD16A1C4E
:107B00004146206808F01FF8102008F01DFB20688F
:107B100008F01EF8B04225D00D20BDE8F88F2A46A7
:107B20004146206808F00FF8206808F011F8064672
:107B3000681E31460EF085FA07466FF07F40A0EBD5
:107B40000900B84201D20D20E7E75FB96A1C41463F
:107B5000206807F0F8FF206807F0FAFFB04201D074
:107B60000D20DAE701225146204600F0F9F9002005
:107B7000D3E72DE9F04F85B00746DDE90E65109C8F
:107B8000601E32F8109032F810C000B20490601EEF
:107B900000B20390601E35F810000290601E35F8A8
:107BA000108000B20190601E00B20090601E58E08C
:107BB00032F810B0A0F1010A32F81AE0DDF848A05E
:107BC000F244D3454BDB32F810B0A0F1010A32F891
:107BD0001AA00AF57A7AD34541DA35F810B0A0F147
:107BE000010A35F81AE0DDF848A0F244D34536DB47
:107BF00035F810B0A0F1010A35F81AA00AF57A7A22
